:100000004D434C46030002000000000002000000C7
:100010000300000001000000FFFFFFFF00000000E0
:10002000000000000000007200000000010000005D
:1000300000100000349E030000C0030038090000D7
:1000400090A604006555020001000000FFFFFFFFBD
:10005000FFFFFFFF000000000000000000000000A4
:100060000000000000000000000000000000000090
:100070000000000000000000000000000000000080
:10008000000000003C000000000000000000000034
:10009000F46E0800100000000000000014000100D1
:1000A0000000000000000000000000000000000050
:1000B00000000000000000000000000000F08AF8CE
:1000C000002000F091F9002070471046704710B5ED
:1000D000C1B20BA000F075F8012010BD014608A0C8
:1000E00000F06FB800F080F9FFF7E8FF05A000F01E
:1000F00061F84FF4967000F077F9FFF7F7FF000012
:10010000256300003E3E3E5445455F50616E696385
:10011000286469766973696F6E206279207A6572E6
:100120006F293C3C3C0A00001A4AD2F88C300A463F
:100130000146B320184738B5184B174AD3E90014C5
:10014000174BC3E9001442B10020694600901068C3
:10015000FFF7EAFF48B9009838BD124929B1124AA1
:100160001AB1106801EB800038BD00F03DF90F496D
:100170000F4800B1006882000648D0F88C304FF07C
:100180000040984739F055FE0548D0E9000105F0D8
:10019000CAF900000010000000000000C06F080055
:1001A000C06F0800D81904002C680200D819050097
:1001B00030680200524AD2F88C300A4601460520C7
:1001C00018470FB410B503A90298FFF7F3FF10BC4E
:1001D0005DF814FB70B5044615460E4649A0FFF7BE
:1001E000F0FF2A46314652A0FFF7EBFF214652A00E
:1001F000FFF7E7FFBDE8704055A0E2E72DE9F84FB3
:10020000102A15468846074601D9012600E0002637
:100210004FF010044FF000090FB1384601E016B15D
:100220004DA0FFF7CEFF35B15EB12A4641464DA045
:10023000FFF7C7FF09E017B14FA0FFF7C2FF4FA0BC
:1002400048E017B14CA0FFF7BCFFA54200D22C46F6
:100250002EB149464DA0FFF7B4FF09F11009002760
:1002600005E018F807104BA0FFF7ABFF7F1CA74273
:10027000F7D3102C06D22EB1C4F1100000EB4000D1
:1002800000F02BF845A0FFF79CFF0027BA460FE0CF
:1002900018F80700A0F120015F2900D32E20CDF827
:1002A00000A069468DF800003DA0FFF78AFF7F1C83
:1002B000A742EDD36EB1102C03D2C4F1100000F0B0
:1002C0000CF838A0FFF77DFF2D1BA044BDD1BDE881
:1002D000F88F20A0BDE8F84F73E710B5044603E09F
:1002E0003148FFF76EFF083C082CF9D2002C06D0ED
:1002F000C4F10800BDE810402B49084461E710BD77
:10030000001000000A232323230A2323232320543D
:10031000525553544C4554204153534552540A238B
:1003200023232320536F757263653A200000000079
:1003300025733A25750A000023232323204578706E
:1003400072657373696F6E3A2025730A00000000AE
:10035000232323230A0000006D656D6F72792064EA
:10036000756D7000202825702C202564206279741A
:100370006573293A0A0000003A2000005B6C656E44
:1003800067746820697320305D0A00007C20257046
:10039000207C200025327820000000007C20000016
:1003A00025730000207C0A0028AE03000248D0F824
:1003B0008C10072008470000001000000249D1F807
:1003C0008C2001460620104700100000054B30B479
:1003D000D3F88C4013460A460146A44630BC0E2092
:1003E00060470000001000000249D1F88C2001464F
:1003F0000420904700100000FEB5064CDDE90856C9
:10040000D4F88C408DE8680013460A4601461B204C
:10041000A047FEBD001000000FB410B503A902985C
:1004200000F004F810BC5DF814FB0000034AD2F899
:100430008C300A46014605201847000000100000D5
:100440000249D1F88C2001461E2010470010000000
:10045000034AD2F88C300A4601461C201847000097
:1004600000100000F07FA0E80000A0E301001EE300
:100470000EF0A0011EFF2FE1F07FB0E80100B0E117
:100480000100A00301001EE30EF0A0011EFF2FE1FA
:10049000012020E0030012E32100001A032010E2F3
:1004A0000300C0E30310C1E304C090E404309104EE
:1004B0000600000A032022E28221A0E1FF34E0E3EB
:1004C0003322A0E1043091E402C08CE1023083E1E8
:1004D00004402DE50140A0E3044484E1044884E1A4
:1004E00004204CE003005CE10C20C20184031201F3
:1004F00004C0900404309104F8FFFF0A0C0CA0E142
:100500002CC4A0E1010050E3030C50212334A001CE
:10051000F9FFFF0AFF3003E2200C63E004409DE492
:100520001EFF2FE1030010E30600000A0120D0E4C3
:100530000130D1E4010052E303005221F8FFFF0A29
:10054000030042E01EFF2FE104502DE504402DE59D
:100550000120A0E3022482E1022882E103C001E23B
:100560000310C1E3044090E4045091E402005CE312
:100570001700000A2D00008AFFC4C4E325045CE1D3
:10058000023044E00430C3E10700001A823313E074
:10059000045091040600001A04C02CE0050C5CE134
:1005A0000800001A044090E4F2FFFFEA2554A0E19D
:1005B000370000EAFF34D3E33100001A0050D1E5E0
:1005C00024CCA0E1320000EA24CCA0E1FF5005E2F7
:1005D0002F0000EA04C8A0E1023044E02CC8A0E1EA
:1005E0000430C3E125085CE10E00001A823313E0F9
:1005F000045091040400001A04C02CE005085CE1DA
:100600000600001A044090E4F1FFFFEA0338B0E16D
:100610001B00001AB050D1E124C8A0E11C0000EA80
:100620000558A0E124C8A0E12558A0E1180000EA7F
:10063000FFC004E2250C5CE1023044E00430C3E179
:100640000700001A823313E0045091040600001AD8
:1006500004C02CE005045CE10600001A044090E4AC
:10066000F2FFFFEA255CA0E1090000EAFF0014E3C5
:100670000300000A045091E424C4A0E1FF54C5E340
:10068000030000EA0000A0E304409DE404509DE460
:100690001EFF2FE1FF200CE2FF0005E2010050E306
:1006A000020050212CC4A0012554A001F8FFFF0A2C
:1006B000000042E004409DE404509DE41EFF2FE151
:1006C000012051E21EFF2F013600003A010050E1E7
:1006D0002200009A020011E12300000A0E0211E339
:1006E0008111A0010830A0030130A013010251E3E1
:1006F000000051310112A0310332A031FAFFFF3A5C
:10070000020151E3000051318110A0318330A0314A
:10071000FAFFFF3A0020A0E3010050E10100402071
:1007200003208221A10050E1A1004020A3208221CA
:10073000210150E12101402023218221A10150E12A
:10074000A1014020A3218221000050E32332B011F7
:100750002112A011EFFFFF1A0200A0E11EFF2FE1FE
:100760000100A0030000A0131EFF2FE1010851E3C8
:100770002118A0211020A0230020A033010C51E358
:100780002114A02108208222100051E32112A0216F
:1007900004208222040051E303208282A12082905F
:1007A0003002A0E11EFF2FE1000050E30000E01343
:1007B000728F00EA000051E3FAFFFF0A03402DE9BF
:1007C000BEFFFFEB0640BDE8920003E0031041E0EE
:1007D0001EFF2FE1000051E34300000A01C020E0AA
:1007E00000106142012051E22700000A0030B0E110
:1007F00000306042010053E12600009A020011E13E
:100800002800000A0E0211E38111A0010820A003B4
:100810000120A013010251E3030051310112A03164
:100820000222A031FAFFFF3A020151E303005131E5
:100830008110A0318220A031FAFFFF3A0000A0E32E
:10084000010053E10130432002008021A10053E167
:10085000A1304320A2008021210153E12131432016
:1008600022018021A10153E1A1314320A201802175
:10087000000053E32222B0112112A011EFFFFF1A52
:1008800000005CE3000060421EFF2FE100003CE13D
:10089000000060421EFF2FE10000A033CC0FA0013A
:1008A000010080031EFF2FE1010851E32118A02160
:1008B0001020A0230020A033010C51E32114A0211B
:1008C00008208222100051E32112A021042082225C
:1008D000040051E303208282A120829000005CE3A7
:1008E0003302A0E1000060421EFF2FE1000050E350
:1008F0000201E0C30201A0B3208F00EA000051E32F
:10090000F9FFFF0A03402DE9B3FFFFEB0640BDE806
:10091000920003E0031041E01EFF2FE1021121E2EB
:10092000000000EA023123E230402DE98140A0E1DD
:100930008350A0E1050034E10200300100C09411B1
:1009400002C09511C4CAF011C5CAF0118C00000A8A
:10095000A44AA0E1A55A74E0005065B2060000DA8E
:10096000054084E0022020E0033021E0000022E086
:10097000011023E0022020E0033021E0360055E39F
:100980003040BD881EFF2F81020111E30116A0E156
:1009900001C6A0E321168CE10100000A000070E20C
:1009A0000010E1E2020113E30336A0E123368CE1FB
:1009B0000100000A002072E20030E3E2050034E1A9
:1009C0006900000A014044E220E075E2050000BA37
:1009D00012CEA0E1320590E00010A1E2130E90E0EB
:1009E0005315B1E0060000EA205045E220E08EE217
:1009F000010052E313CEA0E102C08C23530590E026
:100A0000C31FB1E0025101E20200005A00C07CE2C3
:100A10000000F0E20010E1E2010651E30F00003AAD
:100A2000020651E30600003AA110B0E16000B0E117
:100A30006CC0A0E1014084E2842AA0E1010572E3D8
:100A40006B00002A02015CE3A0C0B0010000B0E22C
:100A5000041AA1E0051081E13040BDE81EFF2FE13E
:100A60008CC0B0E10000B0E00110A1E0010611E38C
:100A7000014044E2F2FFFF1A000031E31430A013FA
:100A80003430A0030010A0010000A0030120A0E169
:100A9000010852E32228A02110304322010C52E326
:100AA0002224A02108304322100052E32222A02158
:100AB00004304322040052E302304322A230433088
:100AC000A23143E0202053E2070000AA0C2092E26A
:100AD000040000DA14C082E20C2062E2110CA0E1F2
:100AE0003112A0E1040000EA142082E220C062D2A8
:100AF0001112A0E1301C81D11002A0D1034054E0BA
:100B0000041A81A0051081A13040BDA81EFF2FA1AD
:100B10000440E0E11F4054E20F0000AA0C4094E2C0
:100B2000060000CA144084E2202064E23004A0E100
:100B3000110280E1311485E13040BDE81EFF2FE154
:100B40000C4064E2202064E23002A0E1110480E164
:100B50000510A0E13040BDE81EFF2FE13104A0E107
:100B60000510A0E13040BDE81EFF2FE1000034E396
:100B7000013623E201162102014084020150451290
:100B80008FFFFFEAC4CAF0E1C5CAF0111D00000AD8
:100B9000050034E1020030010400000A00C094E1C5
:100BA0000310A0010200A0013040BDE81EFF2FE1AC
:100BB000030031E10010A0130000A0133040BD1865
:100BC0001EFF2F11A4CAB0E10400001A8000B0E19A
:100BD0000110B1E0021181233040BDE81EFF2FE17A
:100BE000014594E2011681323040BD381EFF2F319D
:100BF000025101E27F1485E30F1681E30000A0E3B8
:100C00003040BDE81EFF2FE1C4CAF0E10310A0117F
:100C10000200A011C5CAF0010130A0110020A011EE
:100C2000014690E10356920103003101021781133E
:100C30003040BDE81EFF2FE1000030E30010A003AC
:100C40001EFF2F0130402DE9014BA0E3324084E22A
:100C50000050A0E30010A0E386FFFFEA000030E3AD
:100C60000010A0031EFF2F0130402DE9014BA0E32F
:100C7000324084E2025110E2000060420010A0E322
:100C80007CFFFFEA8020B0E1C211A0E16110A0E189
:100C9000020EA0E1FF341212FF0433130E132112CF
:100CA0001EFF2F11000032E3FF0433131EFF2F013C
:100CB00030402DE90E4DA0E3025101E20211C1E3E3
:100CC0006CFFFFEA012090E11EFF2F0130402DE96B
:100CD0000050A0E3060000EA012090E11EFF2F0172
:100CE00030402DE9025111E20100005A000070E28B
:100CF0000010E1E2014BA0E3324084E221CBB0E1FD
:100D000044FFFF0A0320A0E3ACC1B0E1032082123C
:100D1000ACC1B0E103208212AC2182E0203062E25B
:100D200010C3A0E13002A0E1110380E13112A0E183
:100D3000024084E037FFFFEA00C0E0E3020000EA7F
:100D400001C0A0E3000000EA01C0A0E304C02DE55B
:100D500081C0A0E1CCCAF0E183C0A0E1CCCAF0110F
:100D60000E00000A04D08DE281C090E183C09201A0
:100D700003003111020030010000A0031EFF2F010B
:100D8000000070E3030031E1030051510200500103
:100D9000C30FA021C30FE031010080E31EFF2FE14C
:100DA00081C0A0E1CCCAF0E10100001A01C690E1C7
:100DB0000400001A83C0A0E1CCCAF0E1E8FFFF1AEA
:100DC00003C692E1E6FFFF0A04009DE41EFF2FE147
:100DD00000C0A0E10200A0E10C20A0E101C0A0E160
:100DE0000310A0E10C30A0E1FFFFFFEA01402DE974
:100DF000D4FFFFEB000050E3000070430140BDE86A
:100E00001EFF2FE108E02DE5F7FFFFEB0100A00337
:100E10000000A01308E09DE41EFF2FE108E02DE58F
:100E2000F1FFFFEB0100A0330000A02308E09DE4E8
:100E30001EFF2FE108E02DE5EBFFFFEB0100A09383
:100E40000000A08308E09DE41EFF2FE108E02DE5EF
:100E5000DEFFFFEB0100A0930000A08308E09DE40B
:100E60001EFF2FE108E02DE5D8FFFFEB0100A033C6
:100E70000000A02308E09DE41EFF2FE1000053E3E3
:100E8000000052030400001A000051E30000500368
:100E90000010E0130000E013BA8D00EA08D04DE224
:100EA00000602DE9140000EB04E09DE508D08DE220
:100EB0000C00BDE81EFF2FE1F0472DE920909DE5D5
:100EC0000280A0E103A0A0E10060A0E10170A0E128
:100ED000190000EB980103E00020A0E1984085E0B4
:100EE0009A3222E0055082E0044056E00550C7E007
:100EF000300089E8F047BDE81EFF2FE1F8432DE9F7
:100F000020909DE50060A0E10170A0E10280A0E1D9
:100F10000340A0E13C0100EB900403E0904885E031
:100F2000913828E0055088E0044056E00550C7E0BD
:100F3000300089E8F843BDE81EFF2FE1F04F2DE9AE
:100F4000004070E20050E1E2000051E30060E0E3A5
:100F50000040A0A10150A0A10060A0A3000053E3A5
:100F600014D04DE2980000BA000053E304C0A0E1A1
:100F700005B0A0E102A0A0E10310A0E10280A0E181
:100F80000470A0E10590A0E14000001A050052E1C4
:100F90005200009A0200A0E1370200EB000050E38B
:100FA000203060123433A0111A80A01115908311E3
:100FB0001470A0112848A0E10410A0E10900A0E1EC
:100FC000BEFDFFEB0410A0E100B0A0E10900A0E12C
:100FD000F7FDFFEB08A8A0E12AA8A0E19A0B00E02A
:100FE0002728A0E1011882E1010050E10700009AE2
:100FF000081091E001304BE20300002A010050E1AB
:1010000002B04B82081081800000008A03B0A0E18A
:10101000019060E00900A0E10410A0E1A7FDFFEB52
:101020000410A0E10050A0E10900A0E1E0FDFFEB09
:10103000950A0AE00778A0E12778A0E1011887E186
:1010400001005AE10600009A088091E0013045E273
:101050000200002A08005AE1025045820000008A7E
:101060000350A0E10B3885E10040A0E3000056E307
:101070000300A0E10410A0E10100000A000070E2FA
:101080000010E1E214D08DE2F04FBDE81EFF2FE129
:10109000050053E10040A0830430A081F2FFFF8AE5
:1010A0000300A0E10C108DE508C08DE5F20100EB16
:1010B000005050E20C109DE508C09DE57F00001A2D
:1010C0000B0051E10C005A210040A0830140A09385
:1010D0000130A0930540A0910430A081E2FFFFEA17
:1010E000000052E30300001A0210A0E10100A0E397
:1010F00072FDFFEB0080A0E10800A0E1DE0100EB43
:10110000003050E23400001A08A8A0E1099068E01D
:101110002AA8A0E12858A0E10140A0E30510A0E121
:101120000900A0E165FDFFEB0510A0E100B0A0E122
:101130000900A0E19EFDFFEB9A0B00E02728A0E14B
:10114000011882E1010050E10600009A081091E0C8
:1011500001304BE2A400002A010050E102B04B82B2
:1011600008108180A000009A012060E00200A0E148
:101170000510A0E10C208DE550FDFFEB0C209DE556
:101180000090A0E10510A0E10200A0E188FDFFEBC6
:10119000990A0AE00778A0E12778A0E1011887E121
:1011A00001005AE10600009A088091E0013049E20E
:1011B0000200002A08005AE1029049820000008AD9
:1011C0000390A0E10B3889E1A7FFFFEA0660E0E1A8
:1011D000002072E20030E3E262FFFFEA1883A0E140
:1011E00020B063E2394BA0E137BBA0E12858A0E171
:1011F0000510A0E10400A0E119B38BE11773A0E191
:101200002EFDFFEB0510A0E10030A0E10400A0E1FD
:1012100004308DE566FDFFEB08A8A0E104309DE5F4
:101220002AA8A0E19A0300E02B28A0E1011882E19E
:10123000010050E10600009A081091E0012043E20D
:101240006F00002A010050E10230438208108180C3
:101250006B00009A019060E00900A0E10510A0E198
:1012600004308DE515FDFFEB0510A0E10040A0E185
:101270000900A0E14EFDFFEB9A0409E00BB8A0E1E4
:101280002BB8A0E101188BE1010059E104309DE584
:101290000700009A081091E0012044E20300002AB0
:1012A000010059E102404482081081800000008A58
:1012B0000240A0E1019069E0034884E196FFFFEA63
:1012C000203065E23A83A0E1118588E13B23A0E16B
:1012D0003733A0E12898A0E10910A0E10200A0E1C5
:1012E0001BB583E10C208DE5F4FCFFEB0C209DE5A4
:1012F0000030A0E10910A0E10200A0E104308DE57A
:101300002BFDFFEB0848A0E104309DE52448A0E157
:10131000940300E02B28A0E1011882E1010050E1D4
:101320001AA5A0E10600009A081091E0012043E20E
:101330003100002A010050E1023043820810818010
:101340002D00009A01C060E00C00A0E10910A0E1AE
:1013500008108DE9D9FCFFEB08C09DE50020A0E155
:101360000910A0E10C00A0E10C208DE510FDFFEBC1
:101370000C209DE5920404E00BB8A0E12BC8A0E18D
:1013800001C88CE10C0054E104309DE50600009A90
:1013900008C09CE0011042E21500002A0C0054E154
:1013A0000220428208C08C801100009A031882E15A
:1013B000912A83E00C4064E0030054E10700003A06
:1013C0000040A0130140A003170552E10040A09384
:1013D00001400482000054E30130A00122FFFF0A13
:1013E000013041E20040A0E31FFFFFEA03B0A0E1AB
:1013F0005CFFFFEA0120A0E1EBFFFFEA0230A0E181
:10140000CFFFFFEA0230A0E191FFFFEAF04F2DE9A4
:10141000000053E30CD04DE20370A0E10080A0E196
:101420000150A0E10260A0E10240A0E10090A0E133
:1014300001A0A0E13A00001A010052E14800009A20
:101440000200A0E10C0100EB000050E320A06012BC
:1014500038AAA0111640A01115A08A112458A0E1A5
:101460001890A0110510A0E10A00A0E193FCFFEB89
:101470000510A0E10070A0E10A00A0E1CCFCFFEBA8
:101480000488A0E12888A0E1980700E02938A0E1BD
:10149000011883E1010050E10700009A041091E077
:1014A000012047E20300002A010050E10270478258
:1014B000041081800000008A0270A0E101A060E0B9
:1014C0000A00A0E10510A0E17CFCFFEB0510A0E103
:1014D0000060A0E10A00A0E1B5FCFFEB960808E07F
:1014E0000998A0E12998A0E1011889E1010058E1DB
:1014F0000500009A044091E0013046E2CC00002A49
:10150000040058E102604682C900009A070886E19B
:101510000060A0E30610A0E10CD08DE2F04FBDE822
:101520001EFF2FE1010053E10060A0830600A081AF
:10153000F7FFFF8A0300A0E1CF0000EB009050E22C
:101540004200001A050057E1080056210060A08300
:101550000160A0930100A0930960A0910600A08102
:10156000EBFFFFEA000052E30300001A0210A0E1C3
:101570000100A0E351FCFFEB0040A0E10400A0E16A
:10158000BD0000EB003050E27400001A04A8A0E196
:10159000055064E02AA8A0E12478A0E10160A0E35E
:1015A0000710A0E10500A0E144FCFFEB0710A0E15B
:1015B0000080A0E10500A0E17DFCFFEB9A0800E0BF
:1015C0002938A0E1011883E1010050E10600009AEA
:1015D000041091E0012048E29700002A010050E148
:1015E00002804882041081809300009A01B060E07C
:1015F0000B00A0E10710A0E130FCFFEB0710A0E119
:101600000050A0E10B00A0E169FCFFEB950A0AE0A5
:101610000998A0E12998A0E1011889E101005AE1A7
:101620000500009A044091E0013045E28400002A60
:1016300004005AE1025045828100009A080885E1C1
:101640000610A0E10CD08DE2F04FBDE81EFF2FE1A7
:10165000203069E23623A0E1177982E13523A0E149
:101660003833A0E12748A0E10410A0E10200A0E186
:10167000155983E104208DE510FCFFEB04209DE566
:1016800000B0A0E10410A0E10200A0E148FCFFEBE3
:1016900007A8A0E12AA8A0E19A0B00E02538A0E164
:1016A000011883E1010050E11669A0E10300009AEE
:1016B000071091E001204BE26800003A02B0A0E17F
:1016C000013060E00300A0E10410A0E104308DE5EA
:1016D000FAFBFFEB04309DE50020A0E10410A0E13F
:1016E0000300A0E104208DE531FCFFEB04209DE523
:1016F000920A0AE00558A0E12558A0E1011885E109
:1017000001005AE10300009A071091E0013042E223
:101710004D00003A0320A0E10B0882E1904685E0ED
:1017200001A06AE005005AE10600003A0060A0133B
:101730000160A003180954E10060A09301600682D3
:10174000000056E372FFFF0A0060A0E3010040E2E0
:101750000610A0E10CD08DE2F04FBDE81EFF2FE196
:101760001443A0E120B063E2356BA0E138BBA0E1F7
:101770002478A0E10710A0E10600A0E11893A0E101
:1017800015B38BE1CDFBFFEB0710A0E10080A0E1DA
:101790000600A0E106FCFFEB04A8A0E12AA8A0E156
:1017A0009A0800E02B38A0E1011883E1010050E124
:1017B0000600009A041091E0013048E22C00002A53
:1017C000010050E102804882041081802800009AC4
:1017D000015060E00500A0E10710A0E1B7FBFFEBBE
:1017E0000710A0E10060A0E10500A0E1F0FBFFEB25
:1017F0009A0605E00BB8A0E12BB8A0E101188BE137
:10180000010055E10700009A041091E0013046E222
:101810000300002A010055E1026046820410818025
:101820000000008A0360A0E1015065E0086886E1DD
:101830005AFFFFEA0360A0E133FFFFEA0280A0E164
:1018400069FFFFEA0350A0E17BFFFFEA01005AE1D4
:101850000220428207108180AEFFFF8AACFFFFEAC0
:10186000010050E102B04B820710818093FFFF8A94
:1018700091FFFFEA0380A0E1D4FFFFEA1C10A0E380
:10188000010850E32008A02110104122010C50E370
:101890002004A02108104122100050E32002A021C2
:1018A0000410412208208FE20000D2E7010080E00E
:1018B0001EFF2FE1040302020101010100000000EC
:1018C0000000000000207047704746F6DC10C0F2B0
:1018D0000800017819B10120CFF6FF70704780B57C
:1018E0006F460121017000F051F9002080BD704762
:1018F000084611461A4600F000B8F0B503AF2DE9CE
:101900000007ADF5805D82B046F61C280646C0F2A1
:1019100008081446D8F800000D4647F81C0C684625
:1019200000214FF4805221F022EF05F00F00022E2B
:1019300008BF05282FD1204643F20F0510F8041FD9
:10194000CFF6FF7542788378C07841EA022143EAF6
:10195000002041EA0042B2F5805F63D8E678A378C0
:101960006178207843EA062340EA012040EA0341F7
:10197000684600F038F99DF882109DF8810040EA31
:10198000012040F67C7188424CD86846012100F065
:1019900059F8054646E00625012ECFF6FF7508BF2B
:1019A00007283FD1204643F20F0510F8041FCFF659
:1019B000FF7542788378C07841EA022143EA00202B
:1019C00041EA0046B6F5805F2CD8E378A2786178CA
:1019D000207842EA032240EA012040EA02416846B8
:1019E000324600F000F99DF882109DF8810040EA2F
:1019F000012040F67C71884214D86846002100F02E
:101A000021F8054675B9E378A2786178207842EA32
:101A1000032240EA0120694640EA0240324600F0D3
:101A2000E2F80025D8F8000057F81C1C401A01BF46
:101A300028460DF5805D02B0BDE8000708BFF0BD87
:101A400003F054FDF0B503AF2DE9000F89B046F661
:101A50001C280546C0F208088946D8F8000006266A
:101A60000890CFF6FF7695F8821095F8810040EA4D
:101A7000012ABAF1000F544618BF05F18304B9F1E9
:101A8000010F77D8287806280BD0042815D0022813
:101A90005AD102211422C3F2000101F1E040079261
:101AA00014E004204022CAF20000079202300490A1
:101AB0000220C3F20000011D09E002202022C3F22F
:101AC0000000811C04200792CAF2000004904FEA33
:101AD000C20B06A8039204225B4601F0A5FA064653
:101AE000002E47D1049805AA594601F073FA46F62C
:101AF0001C280646C0F20808E6BB05985146DDF8EA
:101B00000C8000220023CDE90080204600F0E0F8A0
:101B100006462EBBDDE9051002F0D4F90646FEB9F3
:101B200006980021002205F14104013502F023FB53
:101B30000698B9F1010F09D1294642462346CDF84E
:101B4000008002F0DCFB08E0043613E007A90091F6
:101B500029464246234602F04BFB064606B90026BC
:101B6000059800F064F9069802F027F946F61C285B
:101B7000C0F20808D8F800000899401A01BF3046A2
:101B800009B0BDE8000FF0BD03F0B0FC80B56F46B2
:101B900082B045F2BF5045F2A85145F2B653C0F2AB
:101BA00002000090C0F20201C0F2020304201022E1
:101BB00000F03EF802B080BDF0B503AF4DF804BDB3
:101BC0000E4600210446FEF743FC05462EB925B11A
:101BD00028460021224621F0CAED28465DF804BBC4
:101BE000F0BDFEF72DBC22F0DBBC22F0C5BC22F01C
:101BF000CFBCD0B502AF84B0044645F20060C0F25D
:101C0000020045F2B653CDE90004C0F20203CDE96B
:101C1000021245F2F551C0F2020106205C2200F0EA
:101C200007F84CF638102146C0F20300FEF724EC0A
:101C3000F0B503AF2DE9000B84B046F61C290D4624
:101C4000C0F208090828D9F800101C46039116466E
:101C50009FBF4CF20C01C0F20301096881421DD8FC
:101C6000D7F8088000F025F8024645F22960C0F256
:101C70000200002C009608BF0446002D08BF054650
:101C800045F218602146C0F202002B46FEF7C4FB65
:101C900007F10C0140460291FEF7C8FBD9F800009D
:101CA0000399401A02BF04B0BDE8000BF0BD03F079
:101CB0001DFC0138062882BF45F25F60C0F20200B9
:101CC000704745F29061C0F2020151F82000704760
:101CD000F0B503AF2DE9000F85B092460546002010
:101CE000BA68CFF6FF7000F106081E460C46002ABF
:101CF00000F08880F968002900F08480887E8007E1
:101D000000F185808868D2000392824200F28780C9
:101D1000002C2046294618BF0120002D18BF0121A4
:101D200011EA000808BF0B24002E3046514618BFA8
:101D30000120BAF1000F18BF01210840049008BF2C
:101D40000D26012106EB040BC8F200015846FFF7EF
:101D500033FF8146B9F1000F4FD045F2B961B8F1B8
:101D6000000FC0F20201484618BF2946224621F062
:101D7000ECEB049845F2AC61C0F202013246002857
:101D800009EB040018BF514621F0DEEBFB6800258B
:101D9000CFF6FF7505F10A08186800F1C041132954
:101DA00027D8BC687F220120C0F20B0200FA01F1A3
:101DB00011421ED0D3F884200021CDE9000148460D
:101DC00059462346FEF718FBFA680028A84610D1AA
:101DD0004FF04040946210620120D0614FF0000843
:101DE000039850609069D2F88410516240F400303A
:101DF00090614846FFF7F5FE04E00020CFF6FF7043
:101E000000F10C08404605B0BDE8000FF0BD45F2FA
:101E1000C4610120C0F202012522FFF7EAFE45F26B
:101E2000C4610120C0F202012C22FFF7E2FE30B1B2
:101E3000817EC90718BF02F0F2BA02F0A5BB704755
:101E4000F0B503AF2DE9000F81B092460246907EB7
:101E50009B46800740F18B82880000F19182C80088
:101E600003D4107BC00700F09482D6690820CFF617
:101E7000FF70012EC0F2778202F1200300251C685A
:101E80008C4204D001350C33B542F8DB6BE26E1C9A
:101E900000F06982BBF1000F00F08482D3F8089053
:101EA000BAF1000F03D0DBF80060B14503D9CBF8DD
:101EB0000090083057E216684025CAF20005AE428D
:101EC00011DC06F1C045132D5ED8012404FA05F596
:101ED0007D24C0F20904254256D0596850464A462E
:101EE000FFF781FE3CE23025CAF20015AE4230DD3C
:101EF000A6F12145413D022D30D33123CAF2001312
:101F00009E424CD03223CAF200139E4240F02B82F4
:101F1000D2F8842041F23103CDF20003994240F31C
:101F20004A8141F23223CDF20003994200F0FA8156
:101F300041F23213CDF20003994200F0F68141F2F2
:101F40003203CDF20003994240F00D8202F1080005
:101F5000F0E1A6F12044413C022C56D240F241224D
:101F6000CCF2000291421EBF40F24122CDF20002AB
:101F7000914206D040F24112CDF20002914240F06F
:101F8000F281D3F80480E3E13023CAF200039E42D9
:101F90003ED03123CAF200039E4240F0E481D2F8E1
:101FA000842041F23003CDF20003994240F3908047
:101FB00041F23123CDF20003994200F00D8141F24C
:101FC0003113CDF20003994200F01F8141F2310339
:101FD000CDF20003994240F0C681D2F80C80404611
:101FE00003F0CAFF0730C11700EB5170DBF8001097
:101FF000C010884240F2AC8145F2D66140F20270D6
:10200000C0F20201FF22FFF7F4FDAE4240F0AB81C7
:10201000D2F8842040F22F73CCF2000399422BDCDB
:1020200040F22F53CCF20003994278DC40F2303377
:10203000CCF20003994200F0198140F23043CCF217
:102040000003994240F08F81D2F81C80404603F093
:1020500093FF0730C11700EB5170DBF80010C01080
:10206000884240F2758145F2D66140F20270C0F2BA
:102070000201B022FFF7BDFD40F22F13CDF20003A5
:10208000994272DC40F23073CCF20003994200F0C6
:10209000048140F63003CCF20003994240F06381A2
:1020A000D2F82C80404603F067FF0730C11700EBE1
:1020B0005170DBF80010C010884240F2498145F2AF
:1020C000D66140F20270C0F20201D422FFF791FD06
:1020D00040F23123CCF20003994200F0AF8040F28D
:1020E0003113CDF20003994240F03D81D2F81880BF
:1020F000404603F041FF0730C11700EB5170DBF899
:102100000010C010884240F2238145F2D66140F2AF
:102110000270C0F202014FF48D72FFF76AFD40F2C7
:102120003053CCF20003994200F0CE8040F230638D
:10213000CCF20003994240F01681D2F82480404648
:1021400003F01AFF0730C11700EB5170DBF80010E5
:10215000C010884240F2FC8045F2D66140F2027025
:10216000C0F20201C222FFF744FD40F23023CDF25B
:102170000003994200F0BF8040F23013CDF200031B
:10218000994240F0F080D2F81080404603F0F4FE0F
:102190000730C11700EB5170DBF80010C010884207
:1021A00040F2D68045F2D66140F20270C0F20201E0
:1021B0009522FFF71EFD40F23223CCF20003994234
:1021C00000F0B68040F23213CDF20003994240F0A5
:1021D000CA8002F11400ADE0D2F81480404603F04A
:1021E000CBFE0730C11700EB5170DBF80010C010B8
:1021F000884240F2AD8045F2D66140F20270C0F2F2
:10220000020140F21112FFF7F4FCD2F810804046B0
:1022100003F0B2FE0730C11700EB5170DBF800107D
:10222000C010884240F2948045F2D66140F20270BC
:10223000C0F202014FF48472FFF7DBFCD2F81C807D
:10224000404603F099FE0730C11700EB5170DBF8F0
:102250000010C01088427BD945F2D66140F202706E
:10226000C0F2020140F22312FFF7C3FCD2F818803B
:10227000404603F081FE0730C11700EB5170DBF8D8
:102280000010C010884263D945F2D66140F2027056
:10229000C0F20201A722FFF7ACFCD2F8288040462A
:1022A00003F06AFE0730C11700EB5170DBF8001035
:1022B000C01088424CD945F2D66140F20270C0F29B
:1022C0000201CB22FFF795FCD2F82080404603F0B4
:1022D00053FE0730C11700EB5170DBF80010C0103F
:1022E000884235D945F2D66140F20270C0F202014F
:1022F000B922FFF77EFCD2F81480404603F03CFE82
:102300000730C11700EB5170DBF80010C010884295
:102310001ED945F2D66140F20270C0F202019E223F
:10232000FFF767FC02F10C0004E002F1240001E079
:1023300002F11800D0F80080404603F01DFE07307F
:10234000C11700EB5170DBF80010C010884232D882
:10235000B8F1000F04D04046514603F0CFFF81464C
:102360000020CBF8009001B0BDE8000FF0BD45F2B1
:10237000D66140F20270C0F202015022FFF739FC30
:1023800045F2D66140F20270C0F202015622FFF718
:1023900030FC45F2D66140F20270C0F202015E22CA
:1023A000FFF727FC45F2D66140F20270C0F202014D
:1023B0007422FFF71EFC45F2D66140F20270C0F2B3
:1023C000020140F24F12FFF714FCF0B503AF2DE904
:1023D000000F81B004465CB3A07E800720D5206842
:1023E0004021CAF20001884226DC00F1C0411329D5
:1023F00000F2B980012202FA01F17D22C0F2090245
:10240000114200F0B080D4E920200021FFF7EFFB5B
:1024100004F1200000216022FFF7E9FB0020E061C9
:1024200000204FF0FF316060C4E90310C4E90500EB
:1024300001B0BDE8000FF0BD3021CAF200118842A2
:1024400041DDA0F121414139022942D33121CAF2B3
:102450000011884200F092803221CAF200118842B5
:1024600040F01D81D4F88450A84658F8080F08B1F0
:1024700003F091FDE86808B103F08DFD2E4656F893
:10248000240F08B103F087FDA86A08B103F083FDAB
:10249000E86A08B103F0C1FC686B08B103F07BFD8A
:1024A000686908B103F077FDA86908B103F073FD0E
:1024B00040460021142221F05AE93046002114221E
:1024C00021F054E9A4E7A0F12042413A022A80F029
:1024D0009080E069D4F88480012822DB40F2412911
:1024E00040F2411A40F2412B04F124060025CDF2BE
:1024F0000009CDF2000ACCF2000B56F8040C484556
:1025000018BF504505D0584506D1306803F043FD4B
:1025100002E0306803F063FDE06901350C36854266
:10252000EBDB04F12000002160220025FFF75FFBB8
:10253000E56103F0DFFC4046002109F014F90028B2
:102540003FD000F06FFD6FF31F3041283FF468AFBC
:1025500000F068FD45F622010020C0F202014FF4B0
:10256000FA72FFF746FB3021CAF20001884242D0DE
:102570003121CAF20001884240F09180D4F88450A1
:10258000E86918B103F007FD0020E861A86918B1F7
:1025900003F001FD0020A861E86818B103F0FBFC1E
:1025A0000020E860686918B103F0F5FC002068615C
:1025B000286900283FF42CAF03F0EDFC00202861CF
:1025C00026E74046002109F0A9F8002848D000F08D
:1025D00029FD6FF31F3041283FF422AF00F022FDA8
:1025E00045F622010020C0F2020140F2FD12FFF781
:1025F00000FB884253D1D4F88450286918B103F005
:10260000CAFC00202861686918B103F0C4FC0020EE
:102610006861A86918B103F0BEFC0020A861E869F0
:1026200018B103F0B8FC0020E861286A18B103F083
:10263000B2FC00202862686A18B103F0ACFC0020EC
:102640006862A86A18B103F0A6FC0020A862E86AD4
:1026500000283FF4DDAE03F09EFC0020E862D7E6E0
:102660004046002109F06DF888B100F0DBFC6FF303
:102670001F3041283FF4D4AE00F0D4FC45F62201CF
:102680000020C0F2020140F20522FFF7B2FA4046F4
:10269000C4F8848003F0E6FFC4F88000C0E645F685
:1026A00022010020C0F2020140F25322FFF7A1FAFA
:1026B000F0B503AF2DE9000F8DB046F61C2980461A
:1026C000C0F208098845D9F800000C904FF00000CE
:1026D0000B90CDE9090000F03283D8F8182012F4ED
:1026E000003F40F03683887E800740F13C83D00372
:1026F00000F14383D8F8000031230C68CAF20013BC
:1027000084422AD03026CAF2000606F18075AC4217
:1027100008BFB04221D04226CAF20006B04218D00B
:102720004126CAF20006B04210D03126CAF2000695
:10273000B04208BF9C4210D045F2357140F6090006
:10274000C0F2020140F2C522FFF753FA03F110066E
:1027500001E003F11106B442EED1D8F808604D68EB
:10276000B54200F2148342F40032C8F81820D8F8B9
:102770000C20CE683240C8F80C20CA6908925A1C56
:10278000944201BFD8F88420D1F884301B691361CA
:1027900000220592089A012AC0F21E82002201F14D
:1027A000200B049200220692002203920022029241
:1027B00000224FF0010A002501920791844203D1C3
:1027C000DBF80060584659E04122CAF2000290420C
:1027D00030D03122CAF20002904215D03022CAF223
:1027E0000002904240F0D08105EB4500DBF800602C
:1027F00040F2301201EB8000CDF200022030964210
:102800003CD040F2302234E005EB4500DBF80060BC
:1028100041F2301201EB8000CDF2000220309642EE
:102820001FDC40F23112CDF20002964226D041F276
:1028300031021EE0DBF8006005EB450040F241127A
:10284000CDF20002964201EB80001EBF40F24142F1
:10285000CFF20002964200F120000FD040F2412258
:1028600007E041F23112CDF20002964206D041F269
:102870003122CDF20002964240F08681424652F863
:102880001C3F03EB430902EB8902566040F2311210
:102890000068CDF2000290421BDD41F23012CDF211
:1028A0000002904241DC40F24022CDF20002904210
:1028B0007ADC40F23212CDF20002904250D040F267
:1028C0004112CDF20002904200F0058140F2302228
:1028D00041E040F22F52CCF2000290424ADD40F635
:1028E0002F02CCF20002904200F39F8040F230525F
:1028F000CCF20002904200F0188140F23062CCF23B
:102900000002904200F0CE8040F23072CCF2000221
:10291000904240F04581D8F884002C4600F128060A
:10292000D1F8840000F1280512E141F23122CDF204
:102930000002904256DC41F23112CDF20002904288
:1029400000F0BA8041F23212CDF20002904200F063
:10295000A98041F23122CDF20002904240F0208164
:10296000D8F884002C4600F11406D1F8840000F158
:102970001405EDE040F24022CCF20002904266DD08
:1029800040F24122CCF20002904200F09F8040F2DF
:102990003032CCF20002904266D040F23042CCF2AB
:1029A0000002904274D0FBE040F24122CDF20002DE
:1029B000904200F0A68041F23102CDF20002904236
:1029C0005CD041F23202CDF20002904240F0E88049
:1029D000D8F884002C4600F10806D1F8840000F1F4
:1029E0000805B5E041F23222CDF20002904245D016
:1029F00040F24142CFF20002904271D041F23232B5
:102A0000CFF20002904240F0CB8008F11C00DBF8CE
:102A1000042000EB89008260DBF80820C260D8F84F
:102A20001C000130C8F81C00AEE040F63002CCF2C9
:102A30000002904200F0838040F23012CDF200029A
:102A4000904239D040F23112CDF2000209E040F25A
:102A50003122CCF2000290421AD040F23222CCF263
:102A60000002904240F09C80D8F884002C4600F18F
:102A70001806D1F8840000F1180569E0D8F8840040
:102A80002C4600F10C06D1F8840000F10C055FE043
:102A9000D8F884002C4600F11C06D1F8840000F11F
:102AA0001C0555E0D8F884002C4600F12406D1F826
:102AB000840000F124054BE0D8F884002C4600F196
:102AC0001006D1F8840000F1100541E001202C46E9
:102AD00009AD039019E02C460BAD0120069014E0DF
:102AE000DBF8043008F11C0000EB89001A46019263
:102AF0008360D8F81C000130C8F81C000120029047
:102B000042E001202C4606900AAD2868DBF80460FC
:102B1000002803D003F03FFA00202860304603F07D
:102B20000AFB0028286020D1ECE0D8F884002C466D
:102B300000F12006D1F8840000F1200508E0D8F863
:102B400084002C4600F12C06D1F8840000F12C05FD
:102B5000306818B103F01FFA00203060286803F0D5
:102B6000EAFA0028306000F0B48008F11C01254624
:102B700001EB89018860DBF80800C860D8F81C0008
:102B80000130C8F81C0007990898824529DA0135F8
:102B90000AF1010A0BF10C0BD8F800000C680DE6E5
:102BA00008F11C00009500EB8905D8F88400049C0E
:102BB0002044A860DBE901163246FFF714F8DBF881
:102BC000080034440799E860D8F81C00009D0130E3
:102BD000C8F81C000494D7E7002200244FF0000B33
:102BE0000BE0019946F61C29D8F80000C0F208094C
:102BF0000591DDF818B0DDE90224A0F12141413949
:102C0000022922BFA0F120404138012833D8D8F84A
:102C10008450C5B3002A4BD005980138042847D802
:102C200045F64001C0F2020151F8200008F0D1FD44
:102C30000646EEB32846314608F083FD824630460C
:102C400006F0A7FFBAF1000F32D02CB1099979B381
:102C5000284608F088FD58B3BBF1000F07D00B9948
:102C600039B30A9A2AB3284608F0CCFC00B32846A8
:102C700008F03FFCE0B1D8F81800002440F4003020
:102C8000C8F8180032E000F0CDF900F0CBF96FF38E
:102C90001F3041280CD10B9808B103F0A0F90A9815
:102CA00008B103F09CF909980C24CFF6FF740CE0EE
:102CB0000B9911B1084603F092F90A9808B103F094
:102CC0008EF901240998CFF2100478B103F063F96A
:102CD0000CE000F0A7F96FF31F30412861D10C24FC
:102CE00046F61C29CFF6FF74C0F20809D9F8000097
:102CF0000C99401A01BF20460DB0BDE8000FF0BD91
:102D000002F0F4FB00F08EF90B9808B103F067F9BC
:102D10000A9808B103F063F9099846F61C29C0F235
:102D20000809002818BF03F036F900F07BF96FF3AB
:102D30001F30412841D10C24CFF6FF74D6E745F26D
:102D4000357140F60900C0F202014FF42A72FEF715
:102D500050FF45F2357140F60900C0F2020140F221
:102D6000AD22FEF746FF45F2357140F60900C0F28C
:102D7000020140F2B222FEF73CFF45F2357140F607
:102D80000700C0F2020140F2B722FEF732FF45F21F
:102D9000357140F60900C0F202014FF43372FEF7BC
:102DA00028FF00F03FF945F2357140F60900C0F206
:102DB000020140F2C632FEF71CFF45F2357140F6C3
:102DC0000900C0F2020140F2AF32FEF712FF00002C
:102DD000F0B503AF2DE900070546002040F20A09CF
:102DE000C5F88000E861402090460E46CAF2000017
:102DF000CFF6FF79864215DC06F1C040102849D88D
:102E0000DFE800F0A1D595A59B0909D5D5D5D5D585
:102E1000D5D5D5D58B00A8F58070B0F5407F40F2B0
:102E20009B80C4E03020CAF2001086421DDDA6F16E
:102E30002140413802281DD33120CAF200108642B9
:102E400033D03220CAF20010864240F0B080A8F59C
:102E50008070B0F5E06F00F2AA8049F221114FF0C6
:102E6000000AC0F200014C2082E0A6F12041413965
:102E7000022938D2A8F1C000B0F5A87F00F29780EF
:102E800008F07FFA0446002C00F08F80204603F003
:102E9000E9FB3DE03020CAF20000864225D0312017
:102EA000CAF20000864240F08280B8F5007F7ED3EF
:102EB000B8F5806F4FF0000048F4806198BF0120A2
:102EC000B1F5406F4FF0000108BF01214FF0000A3B
:102ED00018F03F0F6BD1084369D049F203414420F9
:102EE000C0F2000144E0864261D1A8F58070B0F5DF
:102EF000706F5CD806F0AAFB0446002C55D013F086
:102F0000C4F90146204606F0F3FB002853D05820B0
:102F1000C5F880004FF0000A2EE0B8F1800F18BF0E
:102F2000B8F5807F1BD0B8F1C00F18D03FE0A8F1F2
:102F30005000B0F5D87F0FD939E0A8F1C000B0F546
:102F4000507F09D933E0B8F5805F05D92FE0A8F1AB
:102F50007000B0F5C87F2AD818F0070027D108F113
:102F6000070043F6CF71C0F200014FF0010AC0081C
:102F7000C5F8800088470446C5F88440ACB1BAF172
:102F8000000F05D0D5F8802020460021FEF72FFE47
:102F90004FF000094FF0FF30C5E90069C5E9028034
:102FA000C5E90499C5F8189001E009F102094846FD
:102FB000BDE80007F0BD204606F0AAFB45F2E3712C
:102FC0000020C0F2020140F28962FEF712FE0021E9
:102FD000FEF7F2BDF0B503AF4DF8048D0E46044682
:102FE000882000219046FEF7E7FD05467DB1284682
:102FF00000218822FEF7FBFD284621463246FFF7D6
:10300000E7FE04463CB12846FEF7EBFD06E00C2443
:10301000CFF6FF7402E00024C8F8005020465DF8A7
:10302000048BF0BD00207047F0B503AF2DE9000F11
:1030300087B046F61C2B0390C0F2080B40F20A0E34
:10304000DBF800000D4606900020CDE904000120C9
:10305000C5F20000CFF6FF7E854224DD42F230103B
:10306000C7F20000854242DD45F24000C7F2000091
:10307000854200F3828043F62F00C7F200008542AC
:1030800000F3E38043F24000C7F20000854200F302
:10309000678142F23110C7F20000854200F0818161
:1030A00042F6300078E140F2CF30C1F200008542B4
:1030B0003DDCBF20C1F20000854240F38A8040F22F
:1030C0000F10C1F20000854200F3E380A5F18050AB
:1030D000C038102800F21085012101FA00F0072104
:1030E000C0F20101084240F0968100F005BD40F2B7
:1030F0002F20C6F22100854256DD40F22F20C6F275
:103100006100854200F3928040F22F20C6F2410018
:10311000854200F3098140F23020C6F22100854249
:1031200000F00F8140F23020C6F2310006E10F209E
:10313000C1F20040854263DD0120C3F200008542F8
:1031400040F3E880A5F140500238042800F2D8820C
:103150000292DFE810F005003C0314032F03F30292
:10316000042A40F0C9840221032001904FF0400A54
:103170004FF01409CAF200018DE343F62F10C7F295
:103180003100854272DC46F62F00C7F2000085420E
:1031900000F3EF8045F24100C7F20000854200F0E5
:1031A000008145F63000F7E0A5F1A0400238042880
:1031B00000F2A6800292DFE810F00500D502B90205
:1031C000CE02B202052A40F0978498464FF01409C7
:1031D000B2E243F24100C8F2000085426ADD45F2E6
:1031E0004100C8F20000854200F3EE8043F2420045
:1031F000C8F20000854200F0EF8044F2420068E02F
:103200000F20C1F20020854269DD0F20C1F200309D
:10321000854200F3E9801020C1F20020854200F0D1
:10322000FA8040F21010C1F20020F1E041F24000BB
:10323000C7F20000854200F38A8040F23020C6F2D7
:10324000610085427DD04120A6E044F23010C7F2F3
:103250000000854200F3988043F63000C7F200007A
:10326000854200F09E8044F2410095E045F62F1023
:10327000C7F25100854200F39C8043F63010C7F23C
:103280003100854200F08D8044F63010C7F24100D5
:1032900084E040F20F20C1F20000854200F3AE80CE
:1032A00040F21010C1F20000854200F0B48040F2FC
:1032B000D010ABE03220C8F20000854200F06C82F2
:1032C00041F24200C8F20000854200F0858042F2DF
:1032D0004200C8F2000085427ED000F00DBC40F2F2
:1032E000D030C1F2000085421EBF1020C1F2001094
:1032F000854200F0908040F21010C1F2001087E08B
:103300003020C6F2000085421BD040F23010C6F2D9
:10331000000013E01020C1F2004085427BD040F253
:103320001010C1F2004073E040F23020C6F24100BC
:10333000854206D040F23020C6F25100854240F06E
:10334000DB83012A00F2D8834FF0060C49E041F2FA
:103350004100C7F20000854223D042F241001BE049
:1033600043F24100C7F2000085421AD043F2311007
:1033700012E046F63000C7F20000854211D042F656
:103380003010C7F2210009E044F23110C7F200000A
:10339000854206D044F63000C7F20000854240F076
:1033A000AB8342F00100032840F0A6834FF0070CE6
:1033B00017E045F63010C7F251008542F1D046F6CD
:1033C0003010C7F26100E9E745F24200C8F20000A0
:1033D000854201D0102019E0062A40F08D834FF07D
:1033E000080C4FF0000A1DE01020C1F200308542A9
:1033F00011D040F21010C1F2003009E040F210206C
:10340000C1F20000854206D040F2D020C1F2000097
:10341000854240F07183012A00F26E834FF0010C67
:103420004FF0100A40F22F200021C6F22100854201
:1034300022DC40F20F20C1F20000854242DD40F262
:103440000F10C1F2002085427CDD0F20C1F2004048
:10345000854240F3C8802F20C6F20000854200F369
:10346000D7811020C1F20040854200F00F8140F268
:103470001010C1F2004006E143F23010C7F2000024
:10348000854240DD45F62F00C7F2000085426EDD23
:1034900043F62F10C7F23100854240F3B48045F661
:1034A0002F10C7F25100854200F3BC8143F6301063
:1034B000C7F23100854200F0C18144F63010C7F2F6
:1034C0004100B9E11220C1F20000854266DC44F2FD
:1034D0004100C8F20000854200F3C68041F242007C
:1034E000C8F2000085421EBF42F24200C8F200004E
:1034F000854200F0D18043F24200C8F200008542CC
:1035000000F0CA809DE141F24000C7F20000854210
:1035100052DC40F22F20C6F25100854200F3C280F7
:1035200040F23020C6F2210085421EBF40F230201A
:10353000C6F23100854200F0818140F23020C6F2AF
:10354000410079E10F20C1F2001085426DDC40F2AC
:103550001020C1F2000085421EBF40F21030C1F2BF
:103560000000854200F0928040F2104089E044F271
:103570003010C7F20000854266DC43F23110C7F21A
:103580000000854200F0B78043F63000C7F200002B
:10359000854200F0538144F24100A1E040F20F1057
:1035A000C1F20000854200F32081A5F18050C038AF
:1035B00003286BD3132021E142F23010C7F2000040
:1035C00085427EDC41F24100C7F20000854200F0F6
:1035D0008C8041F63000C7F20000854200F02E8159
:1035E00042F241007CE040F21010C1F2002085421E
:1035F0001EBF1020C1F20030854247D040F21010AB
:10360000C1F200303FE045F63000C7F200008542CD
:103610001EBF46F63000C7F20000854200F00E8162
:1036200042F63010C7F2210006E11020C1F200106E
:1036300085421EBF40F21010C1F20010854225D015
:103640001020C1F200201EE044F23110C7F2000049
:10365000854250D044F63000C7F20000854200F0A9
:10366000ED8045F241003BE044F24200C8F2000028
:1036700085421EBF45F24200C8F2000085420BD0D1
:103680001020C1F20000854240F0DB800220CAF227
:10369000000000F10E01D4E03020CAF2001000F169
:1036A0001201CEE040F23020C6F2510085421EBF2A
:1036B00040F23020C6F26100854200F0BF80412018
:1036C0000EE042F23110C7F20000854213D042F6FC
:1036D0003000C7F20000854200F0B08043F24100A4
:1036E000C7F20000854240F0AC803020CAF20010E2
:1036F00000F11101A5E03020CAF20010411CA0E049
:1037000040F61000C4F20000854240F0F581012A25
:1037100000F2F2814FF0100A4FF0040CB6E7052AD0
:1037200040F0EA8198464FF0400921E0052A40F038
:10373000E38198464FF0200940201AE0042A40F027
:10374000DB8102204FF0000ACAF20000011D0320B5
:103750004FF0400947E0052A40F0CE8198464FF0EF
:10376000300905E0052A40F0C78198464FF01C0952
:10377000002000904FF0050A4FF0010BB0E0042A42
:1037800040F0BA8102204FF0400ACAF20000811CCA
:1037900003204FF0200926E0062A029240F0AC8177
:1037A00030204FF00009CAF20010811C08204FF0B1
:1037B000000A18E0042A40F09F8102204FF0000A1E
:1037C000CAF20000C11C03204FF030090BE0042AAC
:1037D00040F0928102204FF0400ACAF20000411CE2
:1037E00003204FF01C09019055E040F21010C1F287
:1037F000000085423FF44AAF40F21310C1F20000CE
:10380000854202BF0220CAF2000000F1110118E057
:103810003020C6F20000854210D040F23010C6F2CF
:10382000000009E045F63010C7F25100854205D08E
:1038300046F63010C7F26100854202D13021CAF24B
:10384000001144F23110CDE901C2C7F200008542F7
:1038500019D043F23110C7F2000085420FD042F276
:103860003110C7F20000854213D1A3F50070B0F506
:10387000007F00F2418113F03F000AD03CE1B3F534
:10388000006F06D038E143F48060B0F5406F40F03F
:1038900033814FF0000905AA0C46084619469846A0
:1038A000FFF798FB86464146BEF1000F40F02481A9
:1038B00040F21040C1F2000085420BD104AA20461C
:1038C000FFF788FB014629B105980C46FEF7AFFAD1
:1038D000A6460DE14FF0000BCDF800A0DDF804A0E6
:1038E000982000210026FEF767F90446002C00F01E
:1038F000EB80204600219822FEF779F9029BC4E96B
:10390000005A002BA3F10100C4E90239C4E904867E
:1039100008BF02260528A6610FD8C1B22F2222FABD
:1039200001F1009AC90709D045F67041C0F20201C1
:1039300051F820000643A66100E0009A3020C6F24C
:10394000000085420ED1012B05D81020002B08BFA6
:1039500020203043A0615846BBF1000F18BF4FF440
:10396000C0200EE040F21041BBF1000F5846C1F2FA
:10397000000118BF4FF4C0208D42E06102D140F435
:103980000020E0610026DDE90410C4E91D624FF06B
:10399000FF32C4E9086004F1280046C00F20C1F2DC
:1039A0000040854219DD40F60F00C4F20000854258
:1039B00040DC6FF040502844062853D246F683017D
:1039C000D020C0F20201002202F048F90646002E83
:1039D00077D0304603F056FC66E040F20F20C1F28B
:1039E0000000854212DCBF20C1F20000854243DDA9
:1039F000A5F18050C038032852D340F21010C1F214
:103A0000000085424CD040F213103BE00F20C1F281
:103A10000020854216DD0F20C1F20030854234DCE3
:103A20001020C1F2002085423AD040F21010C1F2BD
:103A3000002033E06FF0A0402844062868D202F04E
:103A400003FF2FE040F21020C1F2000085421EBFAC
:103A50001020C1F20010854222D040F21010C1F2B5
:103A600000101BE01020C1F20040854218D040F247
:103A70001010C1F2004011E01020C1F20000854298
:103A80000ED01320C1F2000008E01020C1F2003077
:103A9000854205D040F21010C1F20030854203D1BA
:103AA00003F0C8F8064666B12663BBF1010F039820
:103AB000046017D1204600F04EF888B1204600F08F
:103AC000CAF82046FEF78DF80598FEF7B0F904987D
:103AD000FEF7ADF90A20CFF6FF7000F1020E07E005
:103AE00003980468204600F06BFD50BB4FF0000EB9
:103AF00046F61C2BC0F2080BDBF800000699401AB2
:103B000001BF704607B0BDE8000FF0BD01F0EEFC4C
:103B100040F61000C4F200008542C5D146F683018C
:103B20004FF4BC70C0F20201002202F097F8064682
:103B3000002EC6D0304600214FF4BC72FEF757F875
:103B4000B2E745F6540140F60140C0F2020140F2EE
:103B50009E52FEF74EF8F0B503AF4DF8048D82B0DB
:103B600046F61C280546C0F208080024D8F80000D4
:103B700001902869C11DC808B4EBD10F009005D091
:103B80000021FEF719F80446002C43D0686A50B1B2
:103B90006968032907D16B464FF040412246FEF782
:103BA0004FF900284ED128686FF040510144062992
:103BB00016D36FF0A041014405291CD82D6B00F0ED
:103BC0000DFC01462846002202F051FE98B945F648
:103BD000D5310020C0F202014FF45472FEF709F80B
:103BE0002D6B009E00F0FAFB034628462146324624
:103BF00003F028FBE8B15CB1009A204600210025C3
:103C0000FDF7F5FF207820702046FDF7EAFF04E07D
:103C1000002502E00C25CFF6FF75D8F800000199C9
:103C2000401A01BF284602B05DF8048BF0BD01F0D8
:103C30005DFC45F6D5310020C0F2020140F263324E
:103C4000FDF7D7FF45F6D5310020C0F2020140F262
:103C50003B32FDF7CEFFB0B502AF04460F2120681E
:103C6000C1F20041256B884211DD40F20F71C4F2B0
:103C70000001884224DC6FF04051014406294AD2F9
:103C8000284603F05EFB284602F0C7F887E040F2C2
:103C90000F21C1F2000188421BDD0F21C1F200217A
:103CA000884229DC0F21C1F2001188425FDC40F21A
:103CB0001021C1F2000188426ED040F2104153E061
:103CC0006FF0A041014406292FD2284602F02CFFB4
:103CD00065E0BF21C1F2000188423FDDA0F18051C3
:103CE000C039032958D340F21011C1F200018842B3
:103CF00052D040F2131137E00F21C1F20031884257
:103D00003FDC1021C1F20021884245D040F2101161
:103D1000C1F200213EE01021C1F2004188423BD0B7
:103D200040F21011C1F2004134E040F21071C4F2CF
:103D30000001884230D040F61001C4F200018842F0
:103D400030D1D5F8740100289DD00021F422FDF770
:103D50004EFFD5F8740102F060F894E71021C1F22B
:103D60000001884218D01321C1F2000112E0102195
:103D7000C1F2001188420FD040F21011C1F20011BF
:103D800008E01021C1F20031884205D040F2101144
:103D9000C1F20031884205D1284603F07EF80020A8
:103DA0002063B0BD002DFAD045F6E5310020C0F209
:103DB00002014FF42672FDF71CFFB0B502AF40F6CA
:103DC0000341044600F02BF8606A08B1FEF72FF8B3
:103DD000A06A08B1FEF72BF8206840F21071C4F217
:103DE0000001884210D1D4F88000FDF7FAFE0025CA
:103DF000C4E92055C4F88850D4F88C00FDF7F1FED2
:103E0000C4E92355C4F894502046FFF724FF204608
:103E100000F0EEFB2046BDE8B040FDF7E2BED0B5B5
:103E200002AF0C4618B100F0BCFB48B1D0BD45F65E
:103E3000F2312046C0F2020140F22D52FDF7D9FEC8
:103E400045F6F2312046C0F2020140F23352FDF74E
:103E5000D0FEB0B502AF40F605410446FFF7DFFFE4
:103E60006068052821D0606A10B3E06910F4802FE3
:103E70001ED0216840F21072C4F20002914211D1AA
:103E8000D4F88000FDF7ADFE0025C4E92055C4F844
:103E90008850D4F88C00FDF7A4FEC4E92355C4F87B
:103EA0009450E06920F40030E06100202062B0BD51
:103EB00045F6AD0140F60540C0F2020140F21C6239
:103EC000FDF797FE012200F000B8F0B503AF4DF802
:103ED00004BD0D4640F6064116460446FFF79FFF17
:103EE000206A08B1002E67D1606805281FBF2068CE
:103EF00040F21041C1F20001884267D0E06910F43D
:103F0000003F6DD1400309D5606AFEF75EFA204696
:103F100000F07AF8E06920F48020E061002D47D0BD
:103F2000A069E96861EA0000013063D12968402096
:103F3000CAF2000081420EDC3020CAF20000814249
:103F40001BD03120CAF20000814214D13020CAF2C5
:103F50000010421C1FE04120CAF20000814215D02F
:103F60004220CAF20000814205D13020CAF200107E
:103F700000F112020FE0606A12E0606A3023CAF2B8
:103F8000001302689A4208BF016009E03020CAF2BB
:103F9000001000F11102606A0368934200D10160D1
:103FA0002946FEF785FB20B9E06940F48020E061F6
:103FB00000205DF804BBF0BD45F6094140F606401F
:103FC000C0F2020140F24362FDF713FE45F60941DB
:103FD00040F60640C0F2020140F24C62FDF709FED5
:103FE00045F6094140F60640C0F2020140F2526235
:103FF000FDF7FFFD45F6094140F60640C0F202011B
:1040000040F26162FDF7F5FDB0B502AF0168046BE7
:10401000B1F1405F12DD40F60F00C4F200008142B2
:1040200028DC6FF04050084406284ED2002C00F0E7
:1040300087802046BDE8B04003F083B940F20F20EE
:10404000C1F20000814221DD40F20F10C1F20010E8
:1040500081422ADC40F21020C1F2000081421EBFE2
:1040600040F21040C1F20000814234D01020C1F271
:1040700000102EE06FF0A0400844062831D2002C3A
:1040800067D02046BDE8B04002F06EBCA1F1805080
:10409000C03803281FD31020C1F2000081421AD07B
:1040A00040F21010C1F2000013E040F21010C1F213
:1040B000001081421EBF1020C1F2002081420AD0B0
:1040C00040F21010C1F2002003E040F21070C4F280
:1040D000000081421FD154B32046BDE8B04002F039
:1040E00097BE40F61000C4F20000814213D1CCB359
:1040F000D4F8745135B12846F42101F0D8FE284691
:1041000001F08BFE204600214FF4BC72FDF76FFDDD
:1041100020782070B0BD002C08BFB0BD45F62E4100
:104120000020C0F2020140F20B32FDF762FD45F6BD
:104130002E410020C0F2020140F20232FDF759FD8B
:1041400045F62E410020C0F202014FF43172FDF716
:1041500050FD45F62E410020C0F2020140F2B62289
:10416000FDF747FD45F62E410020C0F202014FF455
:104170003872FDF73EFDD0B502AF40F6037104463C
:10418000FFF74DFE206A012804BF2046FFF761FEBD
:104190006068032818D1E06910F4003F03D120467D
:1041A000FFF757FEE069400318D52046FFF7D3FC20
:1041B000E067D4E90701002940F40030E06100D055
:1041C000D0BD01202062D0BD45F6C11140F603707C
:1041D000C0F2020140F65532FDF70BFD45F6C11164
:1041E00040F60370C0F2020140F65E32FDF701FDB9
:1041F000F0B503AF2DE9000B0E4640F602711D46E7
:1042000090460446FFF70BFEE06F78BB8DB3D7F8FE
:104210000890B9F1000F2CD0E068D9F80010814265
:1042200003D21020CFF6FF7020E0606803282AD167
:10423000A07F800731D5206A012838D12068A0F1FD
:104240004050023804283CD8206B3146424603F0E7
:1042500029F800283FD0206B29464A4603F025F86C
:10426000002842D02046FFF7F4FD0020BDE8000BF7
:10427000F0BD45F6012140F60270C0F2020140F6A1
:10428000BE32FDF7B6FC45F6012140F60270C0F2E1
:10429000020140F6C432FDF7ACFC45F6012140F6C0
:1042A0000270C0F2020140F6C932FDF7A2FC45F6E9
:1042B000012140F60270C0F2020140F6CE32FDF755
:1042C00098FC45F6012140F60270C0F2020140F66A
:1042D0001442FDF78EFC45F6012140F60270C0F253
:1042E000020140F6DD32FDF784FC45F6012140F67F
:1042F0000270C0F2020140F6E332FDF77AFCF0B53D
:1043000003AF2DE9000794B046F61C2A0546C0F21B
:10431000080A0C46DAF8000040F6017113902846AE
:1043200098469146FFF77BFD40200290EE6FDEB984
:1043300002A803AB0090284621464A46FFF758FFE3
:1043400006468EB9B8F1000F1AD0BA6843F271066A
:10435000E868CFF6FF76904206D103A94046FDF704
:1043600044FC002808BF0646DAF800001399401AFA
:1043700001BF304614B0BDE80007F0BD01F0B6F84B
:1043800045F6282140F60170C0F2020140F62E42A7
:10439000FDF72FFC00207047D0B502AF46F6E014C1
:1043A000C0F20804207858B945F29530C0F20000F8
:1043B00001F013FC01F0C3F8012803D101202070A3
:1043C0000120D0BD072045F6C931CFF6FF70C0F2FD
:1043D000020141F2F132FDF70CFC0000A0F1405166
:1043E000023904290DD9A0F1A0400238042884BF65
:1043F00000207047DFE800F0030B0D0F110002F002
:10440000DFB9DFE801F0030406080A00F7E702F06D
:10441000DCB902F0DFB902F0E2B902F0E5B9D0B5DB
:1044200002AF044654B1D4F8800010B1204600F029
:1044300006F82046BDE8D040FDF7D3BBD0BDF0B5AF
:1044400003AF2DE9000F81B004462F212068CAF286
:104450000011884218DD4021CAF20011884227DC91
:104460003021CAF2001188427BD03121CAF20011FA
:10447000884218D03221CAF20011884269D1D4F89A
:10448000840003F09AFE70E0A0F120414139022936
:1044900013D33021CAF20001884262D03121CAF21E
:1044A0000001884255D1D4F8840003F0F7FF5CE0A6
:1044B000A0F12140413802284BD2D4F8840006F004
:1044C00084FF0025C4E92055E069012840DB40F263
:1044D000402840F2412940F2412B04F12406CDF25C
:1044E0000008CCF20009CDF2000B4FF0000A56F89C
:1044F000041C46F8045C414508DC494514D040F2F0
:104500004112CDF2000291420AD018E0594507D07D
:1045100040F24142CFF20002914210D130460CE00D
:10452000306801F05CFD02E0306801F034FD0AEB18
:104530004A00356004EB800028300560E0690146E0
:104540000828A8BF08210AF1010A0C368A45CEDBEB
:10455000E561D4F8840004F11C0558B1FDF741FB76
:1045600008E0D4F8840005F0D3F804F11C0500201D
:10457000C4E92000284600216C2201B0BDE8000FEC
:10458000BDE8F040FDF733BBD0B502AF04463CB107
:104590002046FFF754FF2046BDE8D040FDF721BB81
:1045A000D0BD4CF21001C0F203010968002904BF1C
:1045B000002070478A68824204BF01207047F4E7F8
:1045C000B0B502AF05460C2000210024FDF7F4FA37
:1045D00050B14CF2100104608560C0F203014A68DA
:1045E00042601060486001E04FF0FF342046B0BDEB
:1045F0004CF2100C0146C0F2030CDCF8000030B1A4
:10460000826803688A420CD0002B1846F8D180B526
:104610006F4645F688410020C0F202013722FDF7BF
:10462000E8FA191D002B08BF0CF1040142680A606A
:10463000D0E900121160FDF7D4BAF0B503AF2DE94F
:10464000000B82B0814600F095FA46F6E418002887
:10465000C0F20808C8F8000000F0FD8046F6E81532
:104660000021C0F20805022907D12846102100F0D8
:10467000B2FB03210028F6D0DDE001311329F2D38B
:1046800046F2B8400024C0F2020000F1080555E9E6
:104690000212D5E90036D8F80000009600F0F5F9CE
:1046A000002840F0D08001341435122CEFD900F0EE
:1046B00061FA46F608280028C0F20808C8F8000089
:1046C00000F0D48046F2E9160522C0F2020610235B
:1046D0003146CDF8009000F0D8F90546002D40F0A5
:1046E000D08046F20A26D8F8000009F11001C0F285
:1046F0000206009131460222012300F0C6F9054668
:10470000002D40F0D88046F22026D8F8000009F1AC
:104710001101C0F20206009131460222012300F08D
:10472000B4F90546002D40F0E08046F23426D8F872
:10473000000009F11201C0F2020600913146022286
:10474000012300F0A2F90546002D40F0E88046F272
:104750004D26D8F8000009F11401C0F202060091BC
:1047600031460322042300F090F90546002D40F065
:10477000F08046F25D26D8F8000009F11801C0F279
:104780000206009131460322042300F07EF905461B
:10479000002D40F0F88009F15406D8F8005030465A
:1047A0001FF0B4ED009646F26E26431CC0F20206DE
:1047B00028463146012200F068F90546002D40F0F8
:1047C000FC8046F28C26D8F8000009F16501C0F2A1
:1047D0000206009131460222012300F056F90546F7
:1047E000002D40F0048146F2A826D8F8000009F117
:1047F0006801C0F20206009131460322042300F052
:1048000044F90546002D40F00C8146F2C625D8F843
:10481000000009F16C01C0F2020500912946032253
:10482000042300F032F90446002C40F0148102B059
:10483000BDE8000BF0BD45F64D714FF40072C0F2BB
:104840000201FDF7D6F945F64D7140F20D22C0F296
:104850000201FDF7CEF90C2045F64D71CFF6FF7041
:10486000C0F202014FF4FC72FDF7C3F90C2046F2CE
:10487000D611CFF6FF70C0F2020140F21A22FDF706
:10488000B8F946F2F61046F2D61445F2B653C0F225
:104890000200C0F20204CDE90006C0F202030620C5
:1048A00021464FF40872FDF7C3F92846214640F22D
:1048B0002122FDF79EF946F2F61046F2D61445F293
:1048C000B653C0F20200C0F20204CDE90006C0F205
:1048D00002030620214640F22722FDF7A9F92846C7
:1048E00021464FF40A72FDF784F946F2F61046F2BB
:1048F000D61445F2B653C0F20200C0F20204CDE96C
:104900000006C0F202030620214640F22E22FDF7E7
:104910008FF92846214640F22F22FDF76AF946F228
:10492000F61046F2D61445F2B653C0F20200C0F2B9
:104930000204CDE90006C0F202030620214640F23F
:104940003522FDF775F92846214640F23622FDF75B
:1049500050F946F2F61046F2D61445F2B653C0F2BC
:104960000200C0F20204CDE90006C0F202030620F4
:1049700021464FF40F72FDF75BF92846214640F2BD
:104980003D22FDF736F946F2F61046F2D61445F20E
:10499000B653C0F20200C0F20204CDE90006C0F234
:1049A00002030620214640F24322FDF741F9284642
:1049B00021464FF41172FDF71CF946F2F61046F24B
:1049C000D61445F2B653C0F20200C0F20204CDE99B
:1049D0000006C0F202030620214640F24B22FDF7FA
:1049E00027F9284621464FF41372FDF702F946F2E3
:1049F000F61046F2D61445F2B653C0F20200C0F2E9
:104A00000204CDE90006C0F202030620214640F26E
:104A10005222FDF70DF92846214640F25322FDF7B8
:104A2000E8F846F2F61046F2D61445F2B653C0F254
:104A30000200C0F20204CDE90006C0F20203062023
:104A4000214640F25922FDF7F3F82846214640F26C
:104A50005A22FDF7CEF846F2F61045F2B653C0F2F0
:104A60000200C0F20203CDE9000546F2D615C0F2FD
:104A70000205062029464FF41872FDF7D9F82046A2
:104A8000294640F26122FDF7B4F8F0B503AF2DE9F5
:104A9000000F83B046F61C2B9046C0F2080B05466B
:104AA000DBF8000001AA0290284699460E4600F065
:104AB000A7F8044624B10820CFF6FF7084424DD1F8
:104AC00048460021FDF778F882460C20CFF6FF70AB
:104AD000BAF1000F22D0B96850464A46FDF783F874
:104AE0000C20CFF6FF700438844219D1304600F014
:104AF00059F90446ECB128462146012200F0B7F8E6
:104B000005462046FDF76DF80C24002DCFF6FF7406
:104B100024D005F1140080E8000708E004461DE0F9
:104B2000019CE06908B1FDF75CF8C4E9069A00242D
:104B300014E046F2F62046F29C3145F2B653C0F23C
:104B400002000090C0F20201C0F20203062040F20F
:104B5000A312FDF76DF80C24CFF6FF74DBF800000C
:104B60000299401A01BF204603B0BDE8000FF0BD16
:104B700000F0BCFCB0B502AF82B0202000210025BF
:104B8000FDF71AF804462CB30120C4E90250204670
:104B900040F8145FA06146F68300C0F2020000F006
:104BA00001F90028206128D146F2844046F23941BB
:104BB00045F2B653C0F202000090C0F20201C0F20A
:104BC000020306204FF4F672FDF732F82046FDF797
:104BD00008F811E046F24D4046F2394145F2B6532D
:104BE000C0F202000090C0F20201C0F202030620EF
:104BF00040F2E312FDF71CF80024204602B0B0BDDD
:104C0000F0B503AF4DF8048D82B0804608461546D6
:104C100000F0C8F808240646CFF6FF747EB140467F
:104C20003146002200F023F828603046FCF7D9FF17
:104C30002868B8B1C068022808BF002412E046F214
:104C4000F62046F2E42145F2B653C0F2020000908D
:104C5000C0F20201C0F20203062040F28B12FCF700
:104C6000E7FF0434204602B05DF8048BF0BDF0B5D8
:104C700003AF2DE9000F83B00D4690468146002D0D
:104C800000F08B8028462E211FF05EEA8346BBF1A0
:104C9000000F05D000204FF0010A0BF8010B03E0D4
:104CA0004FF0000B4FF0020AB9F1000F35D04E461D
:104CB00056F8144F00E02468002C06D020692946DD
:104CC000FBF7E6EB0028F6D121E0B8F1010F62D145
:104CD00020200021FCF770FF0446A4B3284600F012
:104CE00061F80028206141D020460021C4E9029AE1
:104CF00040F8141FA061D9F81400206000280EBFEE
:104D000009F1180030680430046034606660A14620
:104D1000BBF1000F5D46B5D13FE046F2343046F2BC
:104D2000233145F2B6534FF00009C0F20200C0F241
:104D30000201CDE90009C0F2020303204FF4B4726E
:104D4000FCF776FF29E046F2463046F23D3145F267
:104D5000B653C0F202000090C0F20201C0F202039A
:104D600006204FF49F72FCF763FF14E046F27330A5
:104D700046F23D3145F2B653C0F202000090C0F257
:104D80000201C0F2020306204FF4A272FCF750FFAA
:104D90002046FCF726FF4FF00009484603B0BDE867
:104DA000000FF0BDF0B503AF4DF8048D80461FF045
:104DB000AEEA451C002100262846FCF7FDFE04460D
:104DC0002CB1204641462A46FCF70DFF26463046C8
:104DD0005DF8048BF0BD102908BF00F019B880B54C
:104DE0006F4682B046F2486046F2346145F2B653EF
:104DF000C0F202000090C0F20201C0F202030620DD
:104E00003D22FCF715FF0620CFF6FF7002B080BDF3
:104E1000F0B503AF2DE9000796B046F61C2A05460B
:104E2000C0F2080A1026DAF8000002AA1590002045
:104E3000CDE906008021CDE90400CDE902064FF05E
:104E40002040FEF7C7F8044684B146F26D6046F292
:104E50005A6145F2B653C0F20200CDE90004C0F237
:104E60000201C0F20203062054223CE0029846F2FE
:104E70009C62C0F2020210211023CDE9006046F2CC
:104E80008C60C0F20200FCF723FF98B1002446F2C8
:104E90006D6046F25A6145F2B653CFF6FF74C0F228
:104EA0000200CDE90004C0F20201C0F202030620B4
:104EB0005D2218E0029804AA03AB4FF04041FCF7D2
:104EC000BFFF0446ECB146F26D6046F25A6145F20E
:104ED000B653C0F20200CDE90004C0F20201C0F2F4
:104EE000020306206522FCF7A3FEDAF800001599FC
:104EF000401A01BF204616B0BDE80007F0BD00F023
:104F0000F5FA0298FCF793FF0DF120090024002127
:104F100020224846CDE91244CDE910441EF026EC8B
:104F200046F2AC614846C0F202011022FCF75BFE7B
:104F300009F1100004A91022FCF755FE0DF14008FC
:104F4000484620211023424600F016F828464146E4
:104F50001022FCF748FE15F8060F02236978AA789C
:104F600040EA0120052161F31F3063F39F12AA700C
:104F70002870000A6870B8E7F0B503AF2DE9000F9C
:104F800085B046F61C2646F2BC6AC0F20806A1F1BE
:104F9000010C36684FF0000B0496C0F2020A10F8BC
:104FA000019BEE460BEB09040229E4B21AF8045007
:104FB0000AD36446064616F8018B013C85EA0805CB
:104FC000EDB21AF80550F6D10EF80B500BF1010BAB
:104FD000BBF1100FE6D110460F2B8CBF10221A46E2
:104FE0006946FCF700FE46F61C20C0F20800006887
:104FF0000499401A02BF05B0BDE8000FF0BD00F0F3
:1050000075FAF0B503AF2DE9000F8DB00D464AF6E5
:1050100022618246C0F2020100201EF0A6E9BAF128
:10502000000F00F0338146F29400854240F03E814B
:1050300046F6182046F61421C0F20800C0F2080116
:10504000C0F800A045F24000504408604CF638100B
:10505000C0F20300FBF706EA002840F03B814CF663
:10506000981545F2300046F6920BC0F203052E1853
:1050700045F22C0005AC05EB00084FF00009C0F22A
:10508000020B04964FF0FF30FBF798F92846514683
:1050900045F240021EF058EA45F23100032105F8BE
:1050A0000090304600F8021B294680F8019080F8F5
:1050B0000090687A11F8082F42EA00208A78C978AF
:1050C00042EA01212A4640EA0140214600F078F9EF
:1050D000010A45F22D02A9544146020E01F8020BC5
:1050E00000284A704FEA10420A700ED046F684013A
:1050F00045F2B6530620C0F202014522C0F2020377
:10510000CDF800B0FCF794FDB7E0EB78AA786978A9
:10511000287842EA032240EA012040EA02414FF6A1
:105120000270814221D04FF60170814247D146F68C
:105130000C20C0F208000068FCF7D9FB45F23100F2
:10514000042105F80090304645F2400200F8021BA9
:10515000294680F8019080F8009050461EF0F4E94E
:10516000FBF724F9FCF7B0FB8CE746F61020C0F201
:105170000800006878B946F2BC70C0F20200FFF780
:105180005CFAFCF79FFB46F61020C0F208000146CF
:10519000086801300860284610F8081F42788378B4
:1051A000C07841EA022146F60C22C0F2080243EA26
:1051B000002041EA00402146FCF787FB13E0284627
:1051C00010F8082F43788678C07842EA03222346F5
:1051D00046EA002042EA004246F60C20C0F20800EF
:1051E0000068FCF785FB010A45F22D0B05F80B1052
:1051F0004146030E01F8020B000C22464B7008706A
:105200002946687A11F8083F43EA00208B78C9786C
:1052100043EA012140EA0140294600F06EF8D8B186
:1052200046F6B20046F6840145F2B653C0F20200DB
:1052300000900620C0F202016522C0F20203FCF7D2
:10524000F7FC40460E2105F80B9000F8021BFF21E9
:10525000049E417001700CE0049E45F2310005F897
:1052600000900421304600F8021B80F8019080F87D
:10527000009046F6920BC0F2020B5046294645F2CA
:1052800040021EF062E9FBF791F8FBE646F64300A8
:1052900046F6340145F2B653C0F202000090C0F267
:1052A0000201C0F2020306207A2210E046F65C01F9
:1052B00045F2B653C0F20201C0F20203CDE9001577
:1052C00046F634010290C0F2020106208022FCF76B
:1052D000AFFC0FE045F22D0030210AF8001045F236
:1052E0002C005044242100F8021BFF214170017062
:1052F000FBF75CF80120FBF777F8F0B503AF2DE979
:10530000000F40F2060C0029CFF6FF7C53D0131D8E
:10531000002206244FF00F094FF00108A61F0CF1E0
:10532000040E09FA06F5054025FA06F6072E43D8BD
:1053300008FA06F616F0230F35D116F00C0F11D12E
:1053400016F0C00F38D001EBC20693F800B093F806
:1053500001E093F802A0DD7806F810BFF57086F83A
:1053600002A01EE01D4613F803EC15F8046D95F835
:1053700002A0ED7801F8146001EB4406F57086F8A0
:1053800002A086F801E001EBC20693F800A093F8B2
:1053900001E09D7893F803B006F810AFB57086F879
:1053A00003B086F801E0013208330434042AB5D38F
:1053B0004FF0000E00E0E6467046BDE8000FF0BD7D
:1053C000F0B503AF2DE9000F40F20608002ACFF632
:1053D000FF7800F0868002F12C0E4FF0000C4FF0A9
:1053E0000F090026012409FA0CF3034023FA0CF5F7
:1053F00008F10403072D75D804FA05F515F0E00F40
:105400002DD115F0050F62D115F00A0F6AD002EB0D
:10541000C6031D4693F80DA015F80CBF95F8028041
:10542000ED7801F836B001EBC60B8BF803508BF822
:1054300002808BF801A013F8108F5D7893F802A01A
:10544000DB788BF805500BF1040505F8028B40F270
:105450000608CFF6FF7885F800A06B7037E002EB06
:10546000C6031D4615F80C8F95F801A095F802B0FB
:10547000ED7848EA0A284BEA052548EA054515B1C2
:1054800041F836500FE001EBC6084FEA1E6501F8FF
:1054900036E088F803504FEA1E4588F802504FEA7C
:1054A0001E2588F8015013F810BF01EBC60593F8CC
:1054B000018093F802A0DB7805F804BFEB7085F853
:1054C00002A085F8018040F20608CFF6FF78013689
:1054D0000CF1040C0EF5A05E042EFFF484AF002343
:1054E00000E043461846BDE8000FF0BD80B56F46AA
:1054F0000F2046F6D301CFF6FF70C0F202012C2236
:10550000FCF777FB80B56F4682B000200421019044
:1055100001A81DF0C8FE46F61C200199C0F2080043
:10552000016002B080BDB0B502AF0C460546FEF783
:1055300033FFFFF7E7FF28462146FFF762FD80B5FE
:105540006F4600F007F818B101F0F8FA012080BDAD
:10555000002080BD41F6DC104FF4A831C0F20700F6
:1055600000F000B8B0B502AF46F620250024C0F226
:10557000080500282C7024D04FF200020024C0F649
:10558000FF728B1803F1704393421AD810F0030294
:1055900017D146F624224318C0F208020839906257
:1055A0000124C2E9003000239060036040F8041F2A
:1055B000C0E90133C0E903334461D36000F003F86C
:1055C0002C702046B0BD2DE9F04103AF0446002CFD
:1055D00071D046F62428201DC0F2080800211422AC
:1055E000D8F80C5000261EF0C2E8002D4FD02068DD
:1055F0002E463168884250D006F10C0138BF06F1C2
:1056000008010D68002DF3D1666030682168814281
:105610002CBFF460B4607069002848D1D8F80C0041
:1056200086423FD0706881688E4212D009B14A69C3
:105630001AB3B068844203D1304600F0B8FA344659
:1056400060680121416100214068416100F099FAE0
:1056500019E0C16809B14A697AB1F068844203D19E
:10566000304600F08EFA3446606801214161002125
:105670004068416100F09BFA05E0012204464A615E
:105680000021726141616668002EC4D10FE00120E3
:105690006660C8F80C40606109E0306920613461DF
:1056A000BDE8F081012141617269002AFBD0D8F880
:1056B0000C0001214161BDE8F0812DE9F04303AF09
:1056C00081B0054646F62020C0F208000078012887
:1056D00023D1142D38BF142515F00300C0F10400A8
:1056E00018BF0544CDB146F62428C0F20808D8F802
:1056F0000C1091B10C462068A84213D004F10801A7
:1057000038BF04F10C0109680029F3D100E02068DA
:10571000A84207D26468002CF9D10024204601B0C9
:10572000BDE8F083204600F04BF8204650F8041DF9
:1057300041F0010101602168491B1B2915D900F1C5
:10574000080445602D19A1F108002E4646F8040F03
:105750000ED0286844F001014FF0000910F0010F4D
:1057600008BF24F00101296005E000F10804D5E735
:1057700000254FF00109286820F00100286030461C
:10578000FFF721FFB9F1000F01D0002002E03068DF
:10579000284408300028C1D0D8F800108142BDD973
:1057A000D8F804108142B9D8016805F1080242F026
:1057B000010311F0010F08BF22F001030360ADE700
:1057C0002DE9F04F03AF81B0002800F01B81026883
:1057D00082B146F62421C0F20801C96805E001F152
:1057E000080338BF01F10C03196819B10B68934223
:1057F000F5D100E000210A6981420DD162B146F67F
:105800002421C0F20801CB68834203D041688B6831
:1058100083421ED0CA601DE0814208BF002A11D118
:105820000246014652F8084F2CB1C36873B31946BB
:105830008B68002BFBD1CC6801F10802CCB14FF092
:10584000000826E00A4611698142FBD10069106117
:10585000D8E08A6081689160816801B14A60C1685E
:10586000D160C16801B14A604168516040695061CE
:10587000C8E046F624234FF00108C0F2080303F104
:1058800010048C60C3F82480596102E04FF00008D6
:1058900001464B6863604B6823B19E68B14205D1F5
:1058A0009C6004E046F62423C0F20803DC604B69E8
:1058B000814219D046682EB1B568854214BFF160A7
:1058C000B16004E046F62425C0F20805E9604569A8
:1058D0004D6185681560C268CA604E60826802B119
:1058E0005160C06800B14160012B7AD146F6242B8B
:1058F0002246C0F2080BDBF80C00A0426FD04FF03C
:10590000010A4FF0000922465069012867D1154667
:1059100055F8040F81688A422AD04A693AB9C1F819
:1059200014A0C0F8149000F042F9286881688A68D1
:1059300012B15369012B12D1CB6873B35E69012E8A
:105940002BD012B15669012E09D10846C3F814A014
:10595000C1F8149000F015F9286881688A684369D5
:105960004B61C0F814A0C2F814A000F020F92EE09A
:10597000C1684A693AB9C1F814A0C0F8149000F09F
:1059800000F92868C1688B6813B15A69012A07D1E8
:10599000CA6812B15369012B11D1C1F8149018E0F3
:1059A000CA6812B15669012E09D10846C3F814A07D
:1059B000C1F8149000F0FBF82868C168CA68436910
:1059C0004B61C0F814A0C2F814A000F0DAF80BF193
:1059D0000C052A68DBF80C0082427FF495AF0120A9
:1059E0005061B8F1000F0DD0606828B181688C4219
:1059F00006D10021816005E046F62420C0F20800AF
:105A00000021C16001B0BDE8F08F2DE9F04F03AF78
:105A100081B0044646F62020C0F208000078012834
:105A200012D146F62426C0F208067168A1420BD8AE
:105A30003068A04208D9254655F8082D12F0010F0C
:105A400002D014F0030F02D001B0BDE8F08F22F0B5
:105A50000109A9F10808414515D8404513D998F81E
:105A6000002012F0010F0ED1A9F10400FFF7A8FEEB
:105A700059F8040C454654F8041C0844083049F809
:105A8000040CD6E90001AA465AF8042F0AF10409C9
:105A900009EB0204A14229D8A04227D9207810F0AE
:105AA000010F20D1A04658F804BF4046FFF788FEFA
:105AB00004EB0B003168083081420BD971688142D8
:105AC00008D8016849F0010211F0010F08BF29F060
:105AD00001020260DAF80000D8F80010084408302B
:105AE000CAF8000002E049F001002060286820F0B8
:105AF00001002860504601B0BDE8F04FFFF763BDDC
:105B0000B0B502AF044646F62020C0F20800007887
:105B1000012804D12CB154F8040C884206D100208D
:105B2000B0BD0846BDE8B040FFF7C7BD46F6242229
:105B30000020C0F208025368A34221D81268A24292
:105B40001ED90846FFF7B9FD05460020002D08BF05
:105B5000B0BD54F8042C55F8041C914288BF11467E
:105B6000B0EB910F08D088082946224652F8043B32
:105B7000013841F8043BF9D12046FFF746FF28469B
:105B8000B0BD98B1C1688A68C26002B15060426815
:105B90004A6022B19368834205D1916004E046F6E1
:105BA0002422C0F20802D16088604160704798B139
:105BB0008168CA68826002B1506042684A6022B15E
:105BC0009368834205D1916004E046F62422C0F236
:105BD0000802D160C8604160704746F65021C0F2AB
:105BE00008010860704746F65022C0F208021268A9
:105BF00022B180B56F469047012080BD4FF0FF3045
:105C000070474CF2B801C0F20301096808474CF232
:105C1000C002C0F20302126810474CF2CC01C0F27D
:105C2000030109680847B0B502AF46F6642504468B
:105C3000C0F208052A6812B12046002190474CF2B4
:105C4000D400C0F203000168204688472A6822B1C8
:105C500000200121BDE8B0401047B0BD2DE9F0475C
:105C600003AF82B0044690468A46012C37DB46F6E5
:105C70005C2946F65421C0F20809C0F20801D9F89F
:105C80000050012008705DB146F658215246C0F21E
:105C90000801434608700020009000202146A847D4
:105CA0004CF2BC005146C0F2030042460368204655
:105CB0009847D9F80060054636B10120214600908A
:105CC000284652464346B047B4F5006F08DD3DB163
:105CD00046F66920C0F208000078287000E0002530
:105CE000284602B0BDE8F0872DE9F04703AF82B047
:105CF00004461E4690460D4664B3012D32DB46F63F
:105D0000602AC0F2080ADAF800C0BCF1000F07D020
:105D100000200021CDE9006020462A464346E047A6
:105D20004CF2C4002946C0F203004246D0F800C03D
:105D300020463346E047DAF800C08146BCF1000F48
:105D400012D001204946CDE9006020462A4643464C
:105D5000E04709E028464146324602B0BDE8F04738
:105D6000FFF77CBF4FF00009484602B0BDE8F0875E
:105D70002DE9F04F03AF83B0D7F81890044698464A
:105D800015468A46002C40D0012D4FF00006A8BFD2
:105D9000554536DB46F6602BC0F2080BDBF8006099
:105DA0003EB100200021CDE9009020462A4643461E
:105DB000B0474CF2BC004146C0F203004A460368BB
:105DC0002846984706467EB13046214652461DF089
:105DD000BCEB2046514600F06AF84CF2C800C0F215
:105DE0000300016820468847DBF800C0BCF1000FC3
:105DF00007D001203146CDE9009020462A4643468F
:105E0000E047304603B0BDE8F08F284641464A4699
:105E100003B0BDE8F04FFFF721BFB0B502AF46F6C3
:105E200064250446C0F208052A6812B12046002104
:105E300090474CF2C800C0F2030001682046884732
:105E40002A6822B100200121BDE8B0401047B0BD52
:105E5000FFF733BCFFF754BEFFF7D7BD80B56F46E1
:105E600082B00346012001AA0191C0F60000194644
:105E7000FAF7ACFA002808BF012002B080BD80B557
:105E80006F4646F66820C0F20800017871B901211A
:105E90000170FFF75FFB48B146F65D60C0F200009D
:105EA000FFF79BFEBDE8804000F048BE80BDF0B526
:105EB00003AF81B046F669260A46C0F20806002AFA
:105EC00035780AD0411C134601F00F0401F8015C3B
:105ED000254401311135013BF6D1E9B21DF050EAFC
:105EE0002918002818BF01F13F05357001B0F0BD39
:105EF000704770477047002070472DE9F04103AFAD
:105F0000984615460E46044612F026FAD0F804C00C
:105F1000204631462A464346BDE8F041604746F6F2
:105F2000E800C0F202007047B0F5803F0AD3B0F13C
:105F3000807F19D346F6FC01000EC0F20201085C16
:105F40001830704710F47F4F1FBF000A46F6FC015F
:105F5000C0F20201085C1CBF0830704746F6FC0125
:105F6000C0F20201085C704746F6FC01000CC0F26A
:105F70000201085C10307047416851B1D0B502AFE2
:105F800000684C1E50F82400FFF7CEFF00EB4410D1
:105F9000D0BD00207047B0B502AF0446CCB1206838
:105FA00068B1A1688900FFF782FF254615F8100F38
:105FB00010F0020F04BF2068FFF72FFF01E004F18B
:105FC0001005204614212D68FFF771FF15F0010F11
:105FD00000D1B0BD2046BDE8B040FFF71EBFD0B530
:105FE00002AF044684B1206828B1217C11F0020F71
:105FF00008BFFFF712FF206910F0010F05D140F430
:106000000040206100202060D0BD2046BDE8D04087
:10601000FFF703BF002114221EF0BABAD0B502AFB9
:1060200082B046F683011420C0F20201002200244F
:10603000FFF714FE38B1C0E900440121C0E9024471
:106040000446016106E003207121412200230094EF
:10605000FFF74EFF204602B0D0BD2DE9F04303AF5D
:1060600081B08046B1F1807F07DB4FF0000903204B
:1060700078217222CDF800903AE098F8100010F0E4
:10608000020F2ED1880046F68301C0F202010022E1
:106090000026FFF7E3FD8146B9F1000F2FD0D8F8B5
:1060A00000E0BEF1000F26D0D8F8040081100129CD
:1060B0002FDB4B1C4FEA810C49467046D0E9006249
:1060C000013BD0E902541030C1E90062012BC1E963
:1060D000025401F11001F1DCD8F804000EEB8C0E33
:1060E00018E04FF000090320CDF8009078216922D4
:1060F0000023FFF7FDFE484601B0BDE8F083032012
:106100007821412200230096FFF7F2FE4FF00009AC
:10611000F1E7494610F00300EDD0012807D002282E
:106120001CBFDEF808008860DEF804004860DEF876
:1061300000000860DFE7B0B502AF05465DB1FFF7CC
:106140006DFF04463CB12046294600F020F818B9FE
:106150002046FFF744FF00242046B0BDF0B503AF52
:1061600081B004460D46A068A8420DDA20462946B3
:10617000FFF773FF064636B1206808B1FFF74DFE02
:106180002660A56000E00024204601B0F0BD2DE9A6
:10619000F04303AF81B088468146C1453AD0D8F874
:1061A0000410D9F80800814205DD4846FFF7D6FF04
:1061B00070B3D8F80410D8F800208B10D9F800007C
:1061C000012B0FDB591C92E8680001390129D468C2
:1061D00002F1100280E86800C46000F11000F2DCF7
:1061E000D8F8041011F003030BD0012B05D0022BBB
:1061F0001CBF916881605168416011680160D8F8E6
:106200000410C9F80410D8F80C00C9F80C0001E01B
:106210004FF00009484601B0BDE8F083B0B502AFC9
:1062200005460C46A868002804DC28460121FFF733
:1062300095FF48B10020002CE8602868046018BF72
:10624000012401206C60B0BD0020B0BD2DE9F047F5
:1062500003AF92460D460646BAF1000F02D04FF04A
:10626000000906E0FFF7DAFE8146B9F1000FCA46E1
:106270003FD0A5B36C1E012000EB9408DAF80800AB
:10628000A108814204DB50464146FFF767FF50B347
:1062900004F003000021CAF80480CAF80C1006E0DC
:1062A000DAF80010A8F1010841F828000320C143E2
:1062B00000203DB116F8012B013D013142EA0020DA
:1062C000F7D1EDE7DAF80400012814DBDAF8001062
:1062D000043951F820201AB90138FADC00E0002016
:1062E000CAF8040007E0B9F1000F02D04846FFF7F2
:1062F00076FE4FF0000A5046BDE8F087B0B502AF19
:106300000C460546FFF738FE0146C81D0E31C21780
:106310000F2900EB52704FEAE00038BFB0BD411EBC
:10632000CA172B6801EB927222F003029B588A1A5B
:106330000139D200B1F1FF3F23FA02F204F8012B38
:10634000EED1B0BD024648685368181A18BF7047AE
:1063500008681168A0F1040C0439012BBCBF0020AF
:1063600070475A1E5CF8230051F8233083421346CD
:10637000F3D04FF0FF3088BF0120704710B50446BE
:106380005CB351B3D4F80CE04FF0FF30BEF1000F16
:1063900008BF0120CB689E451ED14FF0010CBEF115
:1063A000000F08BF4FF0FF3C4B68D4F804E09E4557
:1063B00012DC10DBAEF101035A1C012A16DB0A685D
:1063C00052F823E0226852F82320724588BF10BD9E
:1063D000A3F10103F0D2604610BD002918BF0121CE
:1063E000002C18BF4FF0FF31084610BD002010BD33
:1063F0002DE9F04103AF0D460446002D29DB61680D
:106400006E09B1EB551F17DC06F10108A068864242
:1064100005DB20464146FFF7A1FED0B16168B142DD
:1064200008DC206800EB8100A8EB01018A00002154
:106430001DF09CE9C4F80480226805F01F010120CA
:1064400000FA01F152F82630194342F82610BDE84F
:10645000F0810020BDE8F08100290DDB4268B2EB3D
:10646000511F09DD00684A0901F01F0150F82200A0
:10647000C84000F00100704700207047002915DB7C
:1064800043684A099A4211DA11F01F0110D0531CD7
:1064900043604FF0FF3303FA01FC036853F8221006
:1064A00021EA0C0143F82210426802E00020704704
:1064B0004260012A07DB0168043951F822300BB928
:1064C000013AFADC42600120704719B1416809B114
:1064D000012100E00021C16070476FF0030303EB6E
:1064E000820351F803C0C35863450CD1023A002A15
:1064F00007DB51F822C050F82230634503D1013A3E
:10650000F7DA002070474FF0FF3088BF0120704756
:10651000B0B5A2F1010CB3F1FF3F0DDCACEB03040D
:1065200001EB840E5C1EDEF80050B5B90134AEF10B
:10653000040EB4F1FF3FF6DB012B08DB00EB8C040B
:1065400054F823503DB95D1E022B2B46F8DABDE806
:10655000B040FFF7C2BF0120B0BD4FF0FF30B0BD6B
:10656000D0B502AF46F66C24C0F20804206810B91A
:106570000AF006FA2060D0BD2DE9F04103AF82B0E9
:1065800047F2E35547F2D951C0F20005C0F20001CD
:106590002A462B46044605F0F8F80646C6B900F030
:1065A00032F88046B8F1000F0FD047F2D95220469A
:1065B000C0F2000241462B46009505F0E9F8064678
:1065C0002EB1404600F00DF802E0002600E04646FD
:1065D000304602B0BDE8F08108B100F014B80020E8
:1065E0007047D0B502AF044604F110020C202146DA
:1065F00011F0F9F920461821FFF759FC2046BDE8B3
:10660000D040FFF70ABCB0B502AF82B046F68301B6
:106610001820C0F2020100220025FFF71FFB0446EC
:10662000ACB1256046F66C25C0F20805286810B9A3
:106630000AF0A6F928600021E060616004F1100210
:1066400000692146A0600C2011F0BEF907E02A2065
:106650006421412200230095FFF74AFC00242046D4
:1066600002B0B0BDB0B502AF86B070B305F067F848
:10667000054655B3FFF7D2FC044634B328462146FD
:10668000002203F0ADFCE8B12046FFF775FC0730AF
:10669000C11700EB51700021C010029001A80490B6
:1066A00002200390FF208DF8040002A813F041FEA1
:1066B00041000120102214F022FA05462046FFF77F
:1066C0006AFC03E02046FFF766FC0025284606B07A
:1066D000B0BD80B56F4684B0F86803900020CDE966
:1066E0000100B868009000F002F804B080BDB0B5B9
:1066F00002AF82B00D46144628462146019301F0B0
:10670000C1F9FFF72DFFD0F804C021467869009049
:106710002846D7E90323E047BD6804464CB101A9E8
:10672000204600F03BF82860204600F043F80120A6
:1067300001E00020286002B0B0BD2DE9F04303AFB6
:1067400083B014460D46029300F02EF8019098B1E4
:106750003A6901A802A900F01BF880B1D7F81480AB
:10676000DDF80490FFF7FCFEC668284621464A463D
:106770004346B047044604E04FF0FF3404E04FF0D6
:10678000FF34019800F016F8204603B0BDE8F0830E
:1067900046F6FC13C0F2020312F091B846F6FC1262
:1067A000C0F2020213F0F0B946F6FC10C0F202008B
:1067B00014F05FBA46F6FC11C0F2020113F062B8A1
:1067C00046F64C20C0F20200704746F69820C0F210
:1067D0000200704746F6E420C0F20200704746F619
:1067E0003030C0F20200704746F67C30C0F2020042
:1067F0007047C0680FF028BDC0680EF0C6BBC26805
:10680000084611460FF0B1BCC0680AF084BCC068ED
:106810000AF0E7BCC268084611460AF038BDC068F5
:106820000AF0ACBCC0680BF0DEBBC0680EF032BB37
:10683000C268084611460BF08EBCC0680BF02FBC36
:10684000002118221DF0A4BED0B502AF46F6830188
:106850001820C0F202010022FFF700FA044624B11A
:106860002046002118221CF082EF2046D0BDB0B592
:1068700002AF82B00D460221044600F0CFF9206835
:10688000A84218D020B1406C10B1E068FFF7C5FAFB
:106890002560607A10F0010F0DD1686C58B16969FC
:1068A0000022616146F68301C0F202010025FFF774
:1068B000D5F9E060E0B1206968B100254FF0FF3103
:1068C000F8220723CDE9005400F0D2FB10F1020FAB
:1068D00001D0012813DB607A10F0010F06D1206887
:1068E0000169204602B0BDE8B0400847012506E036
:1068F00006208021412200230095FFF7F9FA28465F
:1069000002B0B0BD43691847F0B503AF81B004468B
:106910000D4620681646816841290BDB46F6830048
:1069200046F6C832C0F20200C0F20202002111F0A5
:10693000A9FA2068826920462946904705462068C2
:106940000EB181683160016A31B120468847204626
:10695000022100F05FF92068426C0021E0681CF021
:1069600006EF284601B0F0BDD0B502AF044620685E
:10697000E8B1006A40B12046022100F054F918B98C
:106980002068016A20468847206880B1406C70B159
:10699000E06860B12046042100F045F938B921686B
:1069A000E068496CFFF783FAE068FFF736FA206980
:1069B00008B100F045FB2046002118221CF0D6EE5D
:1069C0000120D0BDB0B502AF0C460021182205460B
:1069D0001CF0CCEE28462146BDE8B04000F000B8DF
:1069E0002DE9F04703AF82B08A46BAF1000F814625
:1069F0001CBFDAF8000000280BD100260620009604
:106A00006E216F220023FFF773FA304602B0BDE813
:106A1000F087D9F80010814202D04FF0000805E05D
:106A200048460421D9F80C8000F0F4F84846FFF7F6
:106A30009BFFD44649469CE87D007DC1DAF80C00F6
:106A400000B3D9F80000426CE2B1B8F1000F02D0F7
:106A5000C9F80C8011E046F683011046C0F202012D
:106A600000220026FFF7FAF88046B8F1000FC9F8B7
:106A70000C8024D0D9F80000426CDAF80C104046A3
:106A80001CF062EDDAF81400C9F81400DAF810000E
:106A900020B100F0A3FAC9F8100058B1D9F80000ED
:106AA000C2692AB14846514602B0BDE8F0471047D6
:106AB0000126AAE74846FFF757FF0026A5E706206C
:106AC0006E21412200969DE72DE9F04703AF86B085
:106AD0006C4691468A460546204600211822984673
:106AE00000261CF044EE2046012100F093F879695D
:106AF0002046FFF7BCFE80B1059B684629465246FA
:106B0000984748B1684649464246FFF7FDFE0646AB
:106B1000002E18BF012600E000266846FFF724FF7C
:106B2000304606B0BDE8F087D0B502AF0446FFF7A7
:106B30001BFF2046BDE8D040FFF76FB980B56F4618
:106B400000F004F8BDE8804000F01CBA7047B0B512
:106B500002AF0446FFF793F9206800F08DFD012194
:106B60002246054600F04DFF30B3206800F03DFDA1
:106B7000206800F0BBFD0121224600F042FFD8B1A1
:106B80006168D1B122688A4208BFB0BD084600F0F2
:106B900073FD48F201012A4600F033FF60B16068DE
:106BA00000F023FD606800F0A1FD48F201012A46D3
:106BB000BDE8B04000F025BF0020B0BD022100F0CC
:106BC000E3BE012100F0E0BED0F800C0DCF818C040
:106BD00060470068006970470068C0687047006CD3
:106BE00070470068704708B18068704780B56F468D
:106BF00082B00020A221009006209F220023FFF7F0
:106C000077F94FF0FF3002B080BD002814BF006854
:106C1000002070478268114381607047826822EAD1
:106C200001018160704780680840704700218C2214
:106C30001DF0AEBCD0B502AF46F683018C20C0F289
:106C400002010022FFF70AF8044624B12046002181
:106C50008C221CF08CED2046D0BD00002DE9F047C1
:106C600003AF82B00446B86999460E4628B1B0F128
:106C7000FF3F05D1D4F808A006E04FF0000A01E07C
:106C80004FF0010AC4F808A02068C6B130B1204610
:106C9000E56D00F0BDF8C4F808A0E5652660306A2F
:106CA000A0B146F683010022C0F202010025FEF7E2
:106CB000D5FF2066002800F08E80206809E0D8B952
:106CC0000025062000957B2183228DE00020206690
:106CD0003046B1680022C4E91612017C11F0400F61
:106CE0000AD02046002100220023002500F0B2F83F
:106CF000002800F0758020684068102808D801211D
:106D000001FA00F040F20211C0F2010108420AD17A
:106D100046F6830046F6F032C0F20200C0F20202EC
:106D2000002111F0AFF82046D7F81480FFF751FF8B
:106D300010F0100F35D12046FFF74BFF0721C0F2AE
:106D40000F010840052844D8DFE800F02B2B05038D
:106D50000355002020652046FFF73EFF11280ADB7F
:106D600046F6830046F64E42C0F20200C0F202022E
:106D7000002111F087F804F11005B8F1000F07D0D9
:106D80002046FFF729FF0246284641461CF0DCEB6F
:106D90002046FFF721FF024604F1200029461CF09F
:106DA000D4EB2068B9F1000F04BF017C11F0200F73
:106DB00007D046692046494642465346B04740B14F
:106DC000206800210125E160616640680138A06605
:106DD0000DE000250BE006207B214122009503E019
:106DE000009506207B2186220023FFF781F82846A4
:106DF00002B0BDE8F0870020B8F1000F2065D0D0C8
:106E00002046FFF7E9FE024604F120004146C6E7AE
:106E1000B0B502AF0446206868B1C16911B120461F
:106E20008847A8B1254655F8600F30B12168096A36
:106E3000FFF73DF801E004F16005286808B1FEF7AE
:106E4000ECFF204600218C221CF090EC0120B0BD0C
:106E50000020B0BDD0B502AF82B0046864B1E46A6E
:106E600084B1A0470446B4F1FF3F13D100240620AB
:106E70007C21852200940AE00024062000947C21D5
:106E8000832204E00024062000947C218422002335
:106E9000FFF72EF8204602B0D0BDD0B502AF0446B1
:106EA0003CB12046FFF7B4FF2046BDE8D040FEF7D6
:106EB000B4BFD0BD0A460168096911F0800F0DD139
:106EC000D0B502AF82B0836D934205D0012A09DBB1
:106ED00011F0080106D0826501240BE00121002396
:106EE000FFF7B8BF002406207A21822200230094F5
:106EF000FEF7FEFF204602B0D0BDF0B503AF81B073
:106F00000D46044625B3286810B32046FFF780FFDE
:106F1000204629468C221CF018EB286E88B1286880
:106F2000006A70B146F683010022C0F20201002619
:106F3000FEF794FE206600B32A68296E126A1CF0E0
:106F400004EB2868417C11F0040F0CD1012607E006
:106F5000002606200096A3216F220023FEF7C8FF1B
:106F6000304601B0F0BDD0F82CC0284608210022E0
:106F7000234601B0BDE8F04060470620A32141222E
:106F80000096EAE780B56F46FFF71AFCFFF7DFFDD2
:106F900046F6CC4047F2C262C0F20200C0F20202E2
:106FA00048F2010100F02DFD46F6D64046F6E142DA
:106FB000C0F20200C0F2020248F2010100F021FD1D
:106FC000FFF708FCFFF7C3FDFFF709FCFFF7BFFD64
:106FD000FFF70AFCBDE88040FFF7B9BDB0B502AFCE
:106FE0000546286848B3C06838B346F683012820B0
:106FF000C0F2020100220024FEF730FEF0B1044688
:1070000028682060A86810B1816801318160A060A3
:10701000E86810B1816801318160E0600020C4E956
:1070200005002946286920612868C26820469047E3
:10703000002803DC204600F003F800242046B0BD01
:10704000D0B502AF044694B1206818B1016909B106
:1070500020468847A06808B118F03AFFE06808B1F8
:1070600018F036FF2046BDE8D040FEF7D6BED0BDB2
:1070700080B56F4682B080B3D0F800C0BCF1000F7D
:107080001CBFDCF864E0BEF1000F26D0B1F1FF3F79
:107090001CBFDCF800C08C4514D1016951B1B2F1BC
:1070A000FF3F12D0114010D100208921009006200E
:1070B000942204E0002089210090062095220023DC
:1070C000FEF716FF4FF0FF3011E0D7E9022C19460A
:1070D0006346F04710F1020F09D10020892100908A
:1070E000062093220023FEF703FF6FF0010002B099
:1070F00080BD2DE9F04F03AFA1B09B4616460C466C
:107100008146BBF1000F03D0C9F800B0012002E0B6
:10711000D9F800B00020D7F8188074B35846FFF7AC
:107120005EFD0546812D0ADB46F6830046F6F142F8
:10713000C0F20200C0F20202002110F0A3FEB5422C
:107140001FDA09F1040A594642465046FFF78FFB01
:10715000002873D0504621463246FFF7D3FB002863
:107160006CD009F14C0409F1500150462246FFF75A
:10717000CBFB002862D0266818E008BB09F11C068A
:1071800054E0812E0AD346F6830046F60C52C0F234
:107190000200C0F20202002110F074FE09F150005A
:1071A000214632461CF0D0E9C9F84C60802E07D049
:1071B00009EB0600C6F18002503000211CF0D6EA2F
:1071C00009F1500501A900202A5C82F036020A5418
:1071D00001308028F8D109F11C0659464246304654
:1071E000FFF745FB50B35846FFF7F9FC01AC0246E8
:1071F00030462146FFF786FB00B30020295C81F072
:107200005C01215401308028F8D109F13404594639
:1072100042462046FFF72BFB80B15846FFF7DFFCC4
:1072200001A902462046FFF76DFB38B109F10400C1
:107230003146FFF7D5FB08B1012000E0002021B066
:10724000BDE8F08F2DE9F04103AF82B00E461C4639
:10725000904605465EB154B105F11C00FFF7F0FA07
:1072600005F13400FFF7ECFA281DFFF7E9FA0020DA
:1072700031460090284642462346FFF73AFF02B0C7
:10728000BDE8F081D0B502AF044604F11C00FFF761
:10729000D7FA04F13400FFF7D3FA201DBDE8D0403F
:1072A000FFF7CEBA0430FFF72DBB2DE9F04103AF55
:1072B00092B00446261D90460D4601A911AA3046FB
:1072C000FFF722FB98B104F134013046FFF788FB49
:1072D00068B1119A01A93046FFF714FB38B1304666
:1072E00029464246FFF710FB08B1012000E00020CC
:1072F00012B0BDE8F081B0B502AF0D46044604F10E
:107300001C0005F11C01FFF75DFBC0B104F1340066
:1073100005F13401FFF756FB88B1201D291DFFF749
:1073200051FB60B104F1500005F1500180221CF0C6
:107330000CE9E86CE064286820600120B0BD002002
:10734000B0BDD0B502AF044604F11C00FFF70CFB42
:1073500004F13400FFF708FB201DFFF705FB204672
:107360000021D022BDE8D0401DF012B9B0B502AF67
:10737000054605F11C000C46FFF74CFC05F13400F6
:107380002146FFF747FC281D2146BDE8B040FFF726
:1073900041BCF0B503AF81B046F683010546C0F2AB
:1073A0000201E42000220024FEF758FC064666B1E4
:1073B0000420C6E90044C6E9020406F11400346161
:1073C000FFF760FF6E616C620124204601B0F0BDE2
:1073D0002DE9F04103AF0C460546FFF7DAFFD8B1BF
:1073E0006669D5F81480344654F8140B454645F8C0
:1073F000140B2846FFF746FF28462146FFF77BFF80
:1074000050B1F16829B1726808F1040011F055FA21
:1074100010B10120BDE8F0810020BDE8F081D0B5B9
:1074200002AF446904F11400FFF78BFFE06840B13C
:10743000616811B1FEF73BFDE068FEF7EEFC00204D
:10744000E0602046BDE8D040FEF7E7BCD0B502AF13
:1074500040690C46C16859B1043011F02CFA02465B
:1074600032B1204640F2573118F01EFD0120D0BD48
:107470000020D0BDD0B502AF0C464069A1681430E1
:1074800021F48071FFF772FF20464FF48071FFF7FF
:10749000C1FB48F2D550C0F2000060610120D0BDB0
:1074A000F0B503AF81B04669184614460D46FFF7A4
:1074B000ACFBFFF798FB00280CDB206045B106F120
:1074C00014006A462946FFF7F0FE18B100982060C4
:1074D000012000E0002001B0F0BDD0B502AF82B0C5
:1074E00084460129DCF814001BD007291BD006298B
:1074F00026D1002B4FF0000C4FF0000E08BF4FF0CC
:10750000010C002AC8BF4FF0010E0024B2F1FF3F6A
:107510001ADB1EEA0C0117D10430194611F0CDF91F
:107520000BE003600AE050F8143BDCE901414969D3
:107530000A6889680094FFF7DCFD20B1012403E0AC
:107540006FF0010400E00024204602B0D0BDF0B589
:1075500003AF81B015460E46044655B345F21021DF
:107560003046C0F20301F8F794EF50B146F63151BE
:107570003046C0F20201F8F78CEF70B16FF00104F1
:1075800018E0606929464FF0FF32043011F095F998
:10759000002818BF012001B0F0BD6946284610F050
:1075A00063FD05462DB1009AB2F1FF3F05DA0024D4
:1075B0000CE00024204601B0F0BD6069294604308B
:1075C00011F07BF90446002C18BF01242846FEF771
:1075D00024FCEFE780B56F46006940691430FFF77F
:1075E00061FE002818BF012080BDB0F5667F09DB71
:1075F00046F67020C0F208000168002918BF7047E5
:10760000012101607047D0B502AF8AB0C10872296C
:1076100013D848B100EB40014BF68C12C0F20202C5
:1076200002EBC1018968D1B100EB40004BF68C112F
:10763000C0F2020101EBC0041BE046F67421C0F267
:1076400008010A68A2B103210490089102A90991D6
:1076500008A9104611F014F808B1446809E00024A4
:1076600008206721652200230094FEF741FC00E01A
:10767000002420460AB0D0BDD0B502AF8AB0C10800
:10768000722913D848B100EB40014BF68C12C0F2BE
:10769000020202EBC1018968D9B14BF68C1100EBF3
:1076A0004000C0F2020151F830401CE046F674215F
:1076B000C0F208010A68AAB103210490089102A946
:1076C000099108A9104610F0DBFF10B1406804686A
:1076D00009E0002408206821652200230094FEF7B9
:1076E00007FC00E0002420460AB0D0BDD0B502AFB0
:1076F0008AB0C108722914D848B100EB40014BF69A
:107700008C12C0F2020202EBC1018968E1B100EB08
:1077100040004BF68C11C0F2020101EBC00044683E
:107720001CE046F67421C0F208010A68AAB10321E0
:107730000490089102A9099108A9104610F0A0FF31
:1077400010B14068446809E00024082066216522E1
:1077500000230094FEF7CCFB00E0002420460AB092
:10776000D0BD2DE9F04703AF84B001460029039155
:107770003FD08868F0BB46F67420C0F2080000686D
:1077800040B10022CDE9012101A910F079FF08B133
:1077900040682CE040F6CC780DF10C094FF0000A5F
:1077A00040F25936C0F20308002000243546AA45AD
:1077B00012DA05EB0A0000EBD0704610484608EBE1
:1077C0008604214600F0B8F80028EFDB06F1010A34
:1077D0002E460028EAD100E058B954B120684BF693
:1077E0008C11C0F2020100EB400001EBC000806888
:1077F00000E0002004B0BDE8F0872DE9F04F03AFB2
:1078000089B0814646F67420C0F20800CDF80C908D
:10781000006858B10121019103A9029101A910F05A
:107820002FFF08B1406831E0DDF80C9042F6743A61
:107830004BF68C184FF0000B40F29136C0F2030A61
:10784000C0F20208002000243546AB4517DA05EBEC
:107850000B0000EBD07046105AF826000AEB8604A5
:1078600000EB400058F830104846F8F712EE0028B8
:10787000EADB06F1010B2E460028E5D100E038B91D
:1078800034B1206800EB400008EBC000806800E0E5
:10789000002009B0BDE8F08F2DE9F04F03AF89B0AB
:1078A000814646F67420C0F20800CDF810900068BA
:1078B00058B10221019103A9029101A910F0E0FE43
:1078C00008B1406832E0DDF8109041F6305A4BF6CE
:1078D0008C184FF0000B40F29136C0F2030AC0F250
:1078E0000208002000243546AB4518DA05EB0B00F2
:1078F00000EBD07046105AF826000AEB860400EB25
:10790000400008EBC00041684846F8F7C2ED002887
:10791000E9DB06F1010B2E460028E4D100E038B97E
:1079200034B1206800EB400008EBC000806800E044
:10793000002009B0BDE8F08F09684BF68C1203688F
:10794000C0F2020201EB410102EBC101DA68D1F899
:107950000CC0B2EB0C0018BF7047096918691CF025
:107960000BBED0B502AF0446A06810F051FD2168EF
:107970004840D0BD0A6803689A1A1CBF1046704779
:10798000896880681CF008BE2DE9F04103AF84B01F
:1079900005460C467DB346F67828C0F20808D8F8AC
:1079A000000060B948F6631048F67511C0F2000097
:1079B000C0F2000110F0DCFCC8F80000D8B124F4DB
:1079C000004102950091694610F05AFE98B104F406
:1079D00000454FF0FF366C468DB9416879B10136EC
:1079E000092E08DCC06821460290D8F8000010F08B
:1079F00047FE0028F0D1002004B0BDE8F081C06847
:107A0000FAE72DE9F04303AF81B046F67829054641
:107A1000C0F208099046D9F800000E4660B948F651
:107A2000631048F67511C0F20000C0F2000110F0BA
:107A30009FFCC9F80000F0B146F683011020C0F2A7
:107A4000020100220024FEF709F90146B1B106F453
:107A5000004026F40042C1E90020C1E90258D9F8EB
:107A6000000010F016FD10B1FEF7D7F905E0D9F8C7
:107A70000000C06D08B1002400E00124204601B0E0
:107A8000BDE8F08346F67C23C0F208031A6822B9E9
:107A90004CF26012C0F203021A60126802B1104781
:107AA000704780B546F67C2EC0F2080EDEF800C0A6
:107AB000BCF1000F02BF4CF2601CC0F2030CCEF808
:107AC00000C0DCF80CC0BCF1000F08BF80BDBDE8F1
:107AD0008040604746F67C23C0F208031A6822B94A
:107AE0004CF26012C0F203021A60526802B11047F1
:107AF0004FF0FF30704746F67C23C0F208031A6847
:107B000022B94CF26012C0F203021A60126902B18B
:107B100010474FF0FF30704746F67C21C0F2080155
:107B2000086820B94CF26010C0F203000860406998
:107B300000B1004700207047B0B502AF0C460546C3
:107B40002046F9F78CE802460B4628462146BDE858
:107B5000B04000F035B8002200F088B9D0B502AFCF
:107B600046F6802040F21341C0F20800FEF79FF96C
:107B700046F694600024C0F208001421046046F622
:107B80009860C0F20800046046F6A060C0F20800E9
:107B9000FEF78DF946F6D460C0F20800046046F6A0
:107BA000D860C0F20800046046F6B860C0F2080071
:107BB000C0E9004446F6C060C0F208000470D0BDC1
:107BC0002DE9F04F03AF93B0CDE90123059046F6C0
:107BD000C460C0F208000391007801280AD106AC05
:107BE000204610F044F946F6C8602146C0F208006D
:107BF00010F045F946F6D46046F6D86CC0F208009D
:107C0000C0F2080C46F6986E46F6A06300680DF1C7
:107C10003008DCF80090C0F2080E1190C0F20803A2
:107C2000CDF848904546DEF800A093E8570057C5C8
:107C300040F2FF36039D0AEB0503CEF80030B34255
:107C400015DB41F20500C0F24000A3FB0001581A09
:107C500001EB5000410A8902A1EB5020181ACEF81E
:107C6000000046F69460C0F2080006600BE046F69D
:107C7000946240F2FE30C0F208021668864202DCCE
:107C8000B342C8BF136046F26760C6F2666055FB38
:107C900000F0C11001EBD07000EB8001A5EB810179
:107CA0000029C8BF01304844CCF8000006A8FEF700
:107CB000C7FD012D6EDB46F680244FF0000BC0F2AD
:107CC000080440F2FD36FEF77BFD014606A80022BF
:107CD000A9460546FEF7CBFD284641461422FEF78D
:107CE00011FE4D46A5EB0B09B9F1140FCDF810901C
:107CF000C8BF4FF0140904EB0A0109EB0A00B0F504
:107D0000806F0EDBA0F2FF3806ADA9EB0802284613
:107D1000FEF7F8FD284621464246FEF7F3FDA84649
:107D200005E00DF118084A464046FEF7EBFD059DBB
:107D300040464A462946FEF7E5FD11A9404608227D
:107D4000FEF7E0FD40460DF1300800224146FEF707
:107D5000DBFD12984D4405950130129004980128DE
:107D600013DB039D0020514618F8002001F1010AA1
:107D7000635CB14282EA03026254C8BF4FF0000A5A
:107D8000013051464845EFDB00E0039D0BF1140B39
:107D9000AB4598DB06A8FEF7E7FD46F6A06300209A
:107DA000C0F2080318F800101A5C51401954013051
:107DB0001428F7D146F6B8660023C0F20806C4F2CC
:107DC0004003D6E90054002221462846F9F73EE850
:107DD00038B9DDE9012328462146F8F7A6EDC6E9C2
:107DE000000113B0BDE8F08F012200F03FB8F0B5FC
:107DF00003AF83B001A810F03AF846F6C464C0F2AD
:107E000008042078012807D146F6C86001A9C0F20D
:107E1000080010F034F850B146F6C86001A9C0F26D
:107E2000080010F028F801200025207000E001254E
:107E300046F6C066C0F20806307818B918F076F831
:107E40000120307046F6B8600023C0F20800C4F28A
:107E50004003D0E9000100220026F8F7F8EF0028DF
:107E600018BF012005B9267003B0F0BD2DE9F04F11
:107E700003AF93B00E4601240590012EC0F24C8151
:107E800006A80292FEF7DCFC46F6C860C0F20800C5
:107E90000FF0EDFF46F6C460A6F1010AC0F208003B
:107EA00046F6C065047046F26760C6F26660C0F2CE
:107EB00008055AFB00F0811001EBD074287818B93E
:107EC00018F034F80120287046F6D06046F6B869FC
:107ED000C0F20800C0F2080904EB840BD0F800805F
:107EE000D9E900540023C4F2400321460022284669
:107EF000F8F7ACEF002818BF0120039012D13046EC
:107F0000F8F7ACEE02460B4628462146F8F70AED94
:107F100000220023C9E900010024F8F798EF08B90E
:107F2000C9E90044AAEB4B0AB146B8F1000F17D1DA
:107F300045F2141440F21345C0F203042046142104
:107F400000220023FFF73CFE143D142DF6DC0398BD
:107F5000012801BF012046F6D061C0F20801086087
:107F600046F6946046F6986EC0F2080046F6A06C9D
:107F7000046846F6D460C0F20800C0F2080ED0F8DB
:107F8000008046F6D860C0F20800CDF84480006852
:107F9000C0F2080C12900CA9DEF800B09CE86D004D
:107FA0006DC109F10900A0EB0A0000EB0B014D4681
:107FB000A14205DD084621467646F8F7A0ECB64614
:107FC000CEF8001046F6D461059E08F10100C0F21B
:107FD0000801012D086046F6C4604FF00001C0F2B0
:107FE0000800017060DB46F68029C4F10A000490A5
:107FF0000DF1180AC0F20809FEF7E2FB01465046EF
:108000000022FEF734FC0CA950461422FEF77AFC3D
:1080100011A950460822FEF775FC4FF00A080A2DF8
:10802000B8BFA846504631464246FEF76BFC04985E
:1080300009EB0B01A5EB080505955844012809DB60
:108040000546C5F10A025046FEF75CFC504649461B
:108050002A4601E050460A22FEF754FC0CA950467D
:1080600000224FF0000AFEF74FFC0CAA002312F882
:108070000A0019F80B10484009F80B000BF1010B2E
:10808000A345A8BF9B46C245BEBF02EB0A00807A4B
:1080900006F8010B0AF1010ABAF10A0FE7D1059DB2
:1080A0000DF1180A012DA7DAFEF78AFB06AC01468E
:1080B00000222046FEF7DBFB11A920460822FEF72E
:1080C00021FC0CA920461422FEF71CFC46F6A065F4
:1080D0002046C0F2080514222946FEF713FC20466C
:1080E00029460022FEF710FC2046FEF73DFC0398CF
:1080F00008B1012410E00298002468B9242064210A
:10810000642200230094FDF7F3FE45F229110120BB
:10811000C0F20301FDF7EDFE204613B0BDE8F08F7D
:1081200000F000B8F0B503AF81B046F683014C20F3
:10813000C0F2020100220025FDF790FD04468CB339
:1081400046F6DC66C0F2080635681DB907F0B3FADA
:1081500005463560204600211C2265641BF006EBB5
:1081600004F12000002118221BF000EB0120214621
:10817000A063A86904F13C0520F48060E061082058
:108180002A460FF021FC606C016999B120468847AE
:1081900080B9082021462A460FF025FC2046FDF72D
:1081A0003CFE06E005206921412200230095FDF7F1
:1081B0009FFE0024204601B0F0BDD0B502AF0446BA
:1081C0001CB1A06B0138A06300DDD0BD606C4169BB
:1081D00009B12046884704F13C02082021460FF0EF
:1081E00002FCA06808B1FDF7D6FEE06808B1FDF713
:1081F000D2FE606A08B1FDF7CEFEA06A08B1FDF7B5
:10820000CAFEE06A08B1FDF708FE606B08B1FDF731
:10821000C2FE606908B1FDF7BEFEA06908B1FDF7B6
:10822000BAFE2046BDE8D040FDF7F7BDB0B502AFBD
:1082300046F683010446C0F2020114200022002504
:10824000FDF70CFD48B14FF48061022280E8260062
:10825000012560610C30C4E908022846B0BDB0B504
:1082600002AF0C460546FFF7E1FF48B16169686956
:108270000A6802604A684260896881600120B0BD76
:108280000020B0BD4069002818BFFDF7C6BD70478B
:108290002DE9F04103AF84B0884601464C69C869B6
:1082A00020B101AD284617F031FE00E00025FFF7B0
:1082B00037FF064686B1D4E9001230462B4607F058
:1082C00052FB05462DB140461C21324617F0ECFD0D
:1082D00003E03046FFF771FF0025284604B0BDE8F3
:1082E000F081B0B502AF82B005460C46A86890B1E7
:1082F000FFF716FF0246B2B120461C2117F0D4FD4D
:10830000A968204617F06AFD68B1606902B0BDE84F
:10831000B04007F0CAB900207121009005206B22FF
:108320000023FDF7E5FD002002B0B0BDB0B502AFFF
:1083300082B01546826872B1C06860B14069526906
:1083400043690846194607F0B3F90446002C0ADBD6
:108350002C60012407E00024052070216C220023FA
:108360000094FDF7C5FD204602B0B0BD022911D032
:10837000406941F20203994209D041F20103994256
:1083800002D1B2F5807F04DA6FF0010070474260DD
:1083900000E0026001207047F0B503AF83B00E46E5
:1083A00045F273110446C0F2030130461546F8F752
:1083B00070E858B145F289113046C0F20301F8F770
:1083C00068E878B16FF0010003B0F0BD28461AF0FC
:1083D00088EF00210222CDE9000120461C2141F254
:1083E00001030AE028461AF07CEF00210222CDE9C1
:1083F000000120461C2141F20203FEF739FE03B0C2
:10840000F0BD00F000B8F0B503AF81B046F68301CF
:108410004420C0F2020100220025FDF71FFC0446A3
:108420008CB346F6E066C0F2080635681DB906F062
:1084300035FE0546356000200126E5630021C4E9CC
:1084400000001C22A660E06204F10C001BF08EE923
:1084500026632146286A04F1340520F48060A06276
:1084600007202A460FF0B0FAE06B816999B12046E7
:10847000884780B9072021462A460FF0B4FA2046E3
:10848000FDF7CBFC06E00A2067214122002300957E
:10849000FDF72EFD0024204601B0F0BDD0B502AF9F
:1084A00004461CB1206B0138206300DDD0BDE06BB9
:1084B000C16909B12046884704F1340207202146EA
:1084C0000FF091FAE06808B1FDF765FD206908B189
:1084D000FDF761FD606908B1FDF75DFDA06908B1B8
:1084E000FDF759FDE06908B1FDF755FD206A08B1B7
:1084F000FDF751FD606A08B1FDF74DFD2046BDE86E
:10850000D040FDF78ABCB0B502AF46F68301044601
:10851000C0F20201182000220025FDF79FFB58B190
:108520004FF48061A022456180E8260001250221E8
:1085300060610C30C4E908012846B0BDB0B502AF97
:108540000C460546FFF7DFFF58B1616968690A68A4
:1085500002604A6842608A6882604969416101201C
:10856000B0BD0020B0BD4069002818BFFDF755BC64
:1085700070472DE9F04303AF89B0884601464C6946
:10858000C86928B10DF11809484617F0BFFC01E091
:108590004FF00009FFF735FF05460026B5B194E816
:1085A0000E002846CDE90066CDE90266CDE90469F2
:1085B00007F0B0FA06462EB1404674212A4617F05D
:1085C00073FC03E02846FFF769FF0026304609B038
:1085D000BDE8F083B0B502AF82B005460C46A8688E
:1085E00090B1FFF70EFF0246B2B12046742117F09A
:1085F0005BFCA968204617F0F1FB68B1606902B026
:10860000BDE8B04006F0E5BF0020792100900A20C7
:108610006B220023FDF76CFC002002B0B0BD2DE9F9
:10862000F04303AF83B00D46816840691E46D7F81A
:10863000108091464C69406910B1FEF7D2FA00E013
:10864000402002A9CDE90014314642462B4600F0F5
:10865000F8F80128A2BF0298C9F80000012003B071
:10866000BDE8F0832DE9F04303AF83B0894681680C
:1086700040691D46D7F8108016464C69406910B114
:10868000FEF7AFFA00E04020294642464B46CDE9CE
:10869000006400F0FAF803B0BDE8F083F0B503AF72
:1086A00081B046691C46B1F5805F36DC481E0A2859
:1086B0004CD80125DFE800F006424A4A704A704A69
:1086C0004A4A70002046FEF78CFA402853D02046D4
:1086D000FEF787FA74284ED02046FEF782FA422829
:1086E00049D02046FEF77DFA40F2A321884242D0CD
:1086F0002046FEF776FAB0F5287F3CD02046FEF7FC
:1087000070FA40F2A121884235D02046FEF769FA7E
:1087100040F2A22188422ED041E041F20300814282
:1087200017D041F20200814227D041F2010081427C
:108730000CD1B2F5807F09DB32602CE0002078217B
:1087400000900A2096220023FDF7D2FB6FF001056E
:1087500022E02046FEF745FA40280CD02046FEF7DE
:1087600040FA40F2A321884205D02046FEF739FAAC
:10877000B0F5287F13D174610DE06FF00105DF2A99
:1087800003DC3AB1A02A05D006E0B2F5807F18BF1D
:10879000E02A01D172600125284601B0F0BD002514
:1087A0000A2078216A2200230095FDF7A1FBF3E758
:1087B000F0B503AF83B00E4645F29F110446C0F2F8
:1087C000030130461546F7F764EE98B145F2B11152
:1087D0003046C0F20301F7F75CEEB8B145F2C511BF
:1087E0003046C0F20301F7F754EED8B16FF0010044
:1087F00003B0F0BD28461AF074ED00210222CDE945
:1088000000012046742141F2010316E028461AF0C7
:1088100068ED00210222CDE900012046742141F2D9
:1088200002030AE02846FEF7CCF900210222CDE936
:1088300000102046742141F20303FEF719FC03B037
:10884000F0BDB0B502AF82B00D46144628462146B1
:108850000193FFF717F9FA682846214600F061F8FE
:10886000BD6804466CB145F2D81201A9C0F20302FA
:10887000204611F089F92860204600F066F80120B2
:1088800001E00020286002B0B0BDB0B502AF82B0F8
:1088900014460D46019300F047F8009088B1BA687D
:1088A00045F2D81301A96846C0F2030310F007F897
:1088B00050B1FB682846009A214600F02DF8044686
:1088C00004E04FF0FF3404E04FF0FF34009800F074
:1088D0003CF8204602B0B0BDB0B502AF82B00D4644
:1088E00008B1012415E046F683010820C0F2020118
:1088F00000220024FDF7B2F920B1C0E900440224AF
:10890000286006E00A207221412200230094FDF72E
:10891000EFFA204602B0B0BDD3F83CC0DCF80CC082
:108920006047D36B5B681847D0B502AF46F683014A
:108930000820C0F2020100220024FDF78FF910B1D7
:10894000C0E9004404462046D0BDD0B502AF04467D
:1089500064B1206808B1FDF742FB606808B1FDF71B
:108960003EFB2046BDE8D040FDF757BAD0BDB0B5BC
:1089700002AF46F683010446C0F202012420002221
:108980000025FDF76BF988B14FF480616FF00102AB
:10899000C0E900150121C0E904150221C0E9065211
:1089A0000562012560610830C4E908012846B0BDB0
:1089B000B0B502AF0C460546FFF7D9FF78B1646940
:1089C0006D6920682860606818B1FDF7B4FB6860C5
:1089D00028B120692861606968610120B0BD00206C
:1089E000B0BDD0B502AF446964B1606808B1FDF7AD
:1089F000F6FA206A08B1FDF710FA2046BDE8D0402B
:108A0000FDF70BBAD0BD2DE9F04303AF83B00646A6
:108A100088467469606840B9FDF700FB606080B10A
:108A20004FF00111FDF7FAFB58B100F00FFE0546BB
:108A30003DB1F06938B1E9463146484617F066FA6B
:108A400003E0002613E04FF00009D4E900122846A5
:108A50004B460EF011FE0646012E05DB4046062170
:108A60002A4617F021FA02E0284600F051FE30466F
:108A700003B0BDE8F0832DE9F04F03AF85B00646A3
:108A80008946B1681C4675699046D7F818A0D1F898
:108A900014B06869C0B1FEF7A6F8504522D16869E4
:108AA000FEF79FF85F282AD12869012822D104A85F
:108AB000CDE9000B5F20214652464B4600F075FD84
:108AC000012819DB049807E02869214600905046E8
:108AD0004A465B460EF0D1FA00280DDBC8F80000CC
:108AE000012009E000208E21009004208F22002325
:108AF000FDF7FEF94FF0FF3005B0BDE8F08F2869B3
:108B000001281CD0062829D00528F3D12846314653
:108B100000F0A2FA0028EDD0286A214652461AF049
:108B200014ED6869FEF75DF800F047FB296A01F86B
:108B30000A000520296A00900AF10100C8E7686967
:108B4000FEF74FF803A9CDE9001B214652464B46DC
:108B500000F04FFB0128CFDB0398BDE728463146E4
:108B600000F07AFA0028C5D0D5E90530D5E907210B
:108B7000CDE90002584622460EF082FC0028B9D00A
:108B800058460EF06AFA0322296A0092A0E72DE9FE
:108B9000F04703AF84B00C460146886899464D699A
:108BA0001646D7F81480D0F814A0686988B12A69ED
:108BB000062A1ED0052A3CD0012A37D1FEF711F82B
:108BC000494642462346CDE9006A00F0CDFC064600
:108BD00045E0284600F040FA40B32A6A2146286959
:108BE0005346009030460EF052FA039060BB0026C8
:108BF00035E0284600F030FAC0B12A6A0320009020
:108C00003046214653460EF042FA0026012826DB64
:108C1000D5E90523D5E90701CDE9001050464946BD
:108C20000EF00EFB0028C8BF012618E04FF0FF36FB
:108C300015E003AA0846002123460096002600F00E
:108C400012F801280BDB03980026404507D1296A5A
:108C5000484642461AF01EEC002808BF012630465E
:108C600004B0BDE8F0872DE9F04703AF86B00646B3
:108C7000D7F8149074691D4690468A46606960B3BF
:108C80002169012937D0052932D12046314600F02B
:108C9000E3F968B3B0682946226A43690520009069
:108CA00048460EF0F4F901283FDB451E6069216A51
:108CB0004E5DFDF796FF00F080FA864237D160697D
:108CC000FDF791FF854238D1BAF1000F26D0216A15
:108CD00050462A461AF038EC20E0B0682946524641
:108CE00043692069009048460EF0D1F9054613E02B
:108CF0004FF0FF3515E0FDF774FFB16805AA534644
:108D000049698DE82402002200250391002100F02A
:108D100011FB012805DB059D002D02DBC8F8005082
:108D20000125284606B0BDE8F0870025F9E70025B3
:108D300004208D216422009504E000250420009584
:108D40008D218F220023FDF7D3F8EAE7B0B502AFFB
:108D500082B015460A46816840694C691946006927
:108D60000090B86823460EF083F9002801DB2860E4
:108D7000012002B0B0BDB0B502AF82B015460A46C0
:108D8000816840694C69194600690090B8682346BB
:108D90000EF078F9002801DB2860012002B0B0BD98
:108DA0002DE9F04103AF82B0064641F20100D6F84A
:108DB0001480081A1D461446072810D8DFE800F072
:108DC00038044A5224560424D8F81000062852D1F8
:108DD00041F2070081425CD1D8F81C0048E001391B
:108DE000062900F278800120DFE801F0041C777783
:108DF00077757700D8F81010284600F044F900285D
:108E000045D0C8F8145034E0D8F81000062838D1FE
:108E100041F20800814242D1D8F8180040BBD8F88E
:108E2000140025E000208F210090042094224FE0C0
:108E3000601E052847D8D8F81400214600F023F911
:108E400028B3042C31D0062C3AD1307C10F0180F06
:108E50002FD138E0FF2C25DC00208F21009004204A
:108E6000912235E0BDB3C8F8045002E0D8F81000F4
:108E70002860012031E000208F2100900420922200
:108E800026E000208F21009004209C2220E000207A
:108E900023E014F1020F1EDBC8F81C40E9E7C8F814
:108EA0001850E6E7C8F80040E3E7707C10F0030FC5
:108EB00009D0D8F8140018B9FDF782FCC8F81400DE
:108EC000C8F81040D5E700208F21009004209022A0
:108ED0000023FDF70DF86FF0010002B0BDE8F0814E
:108EE000F0B503AF83B015460E460446DDB345F238
:108EF00048213046C0F20301F7F7CAEAE0B345F271
:108F00006F213046C0F20301F7F7C2EA002873D0A0
:108F100045F27F213046C0F20301F7F7BAEA002894
:108F200076D045F28F213046C0F20301F7F7B0EA60
:108F300000285CD102A800262946029612F0B3FC54
:108F4000002856D002980621042241F20403CDE9FC
:108F500000602046FEF78CF80646002E49DC029899
:108F6000FDF73DF845E000260420902193220023E0
:108F70000096FCF7BDFF3CE047F642512846C0F2A0
:108F80000201F7F786EA00284ED045F2592128461B
:108F9000C0F20301F7F77CEA002847D045F26021D0
:108FA0002846C0F20301F7F774EA002840D045F2E2
:108FB00065212846C0F20301F7F76AEAD0B345F20B
:108FC0006A212846C0F20301F7F762EAA0B349F22A
:108FD000A5112846C0F20201F7F75AEA70B3002043
:108FE00090210090042076220023FCF781FF6FF08F
:108FF0000106304603B0F0BD28461AF072E90021A0
:109000001822CDE900012046062141F202031FE0AB
:1090100028461AF066E900210422CDE90001204625
:10902000062141F2030313E0012008E0022006E0DC
:10903000032004E0042002E0052000E006200021D7
:109040004FF0FF32CDE900012046062141F2010335
:10905000FEF70EF803B0F0BDD0B502AF0446206AAB
:1090600008B10120D0BD886840690DF0F6FF46F6D2
:1090700083010022C0F20201FCF7F0FD206200280B
:1090800018BF0120D0BDD0B502AF82B080B1052994
:1090900007D003290CD10024042000948C218D22B8
:1090A0000DE0FDF79EFD00F088F8B0F1FF3F01D024
:1090B000012407E0002404208C218E220094002348
:1090C000FCF716FF204602B0D0BD2DE9F04103AFFA
:1090D00082B01C46091B154601290ADC00207F21AD
:1090E000009004206E220023FCF702FF4FF0FF30B7
:1090F0001DE08A1E00F101060FD06B23022A0370C7
:1091000007DBA1F103083046BB2142461AF02EEBE3
:109110004644BA2006F8010B01E06A21017030468E
:10912000294622461AF010EACC203055012002B020
:10913000BDE8F081D0B502AF82B0BC689C4213D1CB
:10914000117801F0FE036A2B0ED16B2919D1042C82
:1091500027DBA4F1030C0023D1184C78BB2C13D1CE
:1091600001339C45F8DC12E00020802100900420AF
:1091700089220023FCF7BCFE4FF0FF34204602B0EA
:10918000D0BD511C023C05E0BA2C0AD14BB1ACEB6E
:10919000030402310A5DCC2A09D122461AF0D4E92F
:1091A000ECE700208021009004208A22E1E70020E3
:1091B0008021009004208B22DBE7B0F5287F09DCBA
:1091C000402804BF33207047B0F5287F04BF342007
:1091D00070470BE040F2A121884204BF362070475F
:1091E00040F2A221884204BF352070474FF0FF3083
:1091F00070472DE9F04F03AF8FB0D7F81CB0894608
:10920000B9690446984616469BF83C0010F0400F9A
:109210000CD0DBF80800C56A45B1CDE9001B20463B
:10922000494632464346A84705467FE0722C04D1A2
:10923000242E2ED14FF0240A1DE008A80D902046C0
:10924000FEF7E1F90D99002808603FD0C0680028BA
:1092500042D005200B9000200C900BA8486004A879
:109260000E900DA80021CDF81890049611F01AFA6E
:1092700082464FF0000958460DF0EFFE0646A6F173
:109280000B0082450BDD002504200095752170221E
:1092900049E00025042000957521832243E0722CCB
:1092A00020D046F68301701CC0F202010022002586
:1092B000FCF7D4FC8146B9F1000F30D00DA80AA903
:1092C000CDF8289011F0EEF948460CE00025042076
:1092D00000957521752226E0002504200095752152
:1092E000742220E00020039001200090504649465F
:1092F00042465B460DF0C1FE012803DBB96901253A
:10930000086000E00025DDF80C80722C0ED0711C86
:109310004046FCF7CCFD4046FCF77FFD06E004200C
:109320007521412200950023FCF7E2FD28460FB08D
:10933000BDE8F08F2DE9F04F03AF83B0D7F824805C
:1093400083461E4615460C4640460DF086FE3A6A98
:10935000904213D1D7E906A9BBF1720F17D1B6B16C
:109360000120494600901046324643460DF08FFEDC
:10937000012828DBCAF800000126BFE000260420EF
:109380000096912177220023FCF7B2FDB6E046F665
:1093900083011046C0F20201002201960026FCF76C
:1093A0005DFC824688B1BBF1720F13D1242D11D020
:1093B000002604209121832200230096FCF798FDCB
:1093C000396AD14694E0002698E004209121412298
:1093D0000096D8E7012049460090D146386A4A46AF
:1093E00043460DF054FE82460026BAF1010F7EDBA3
:1093F000BBF15F0F0ED1A046019CBAF1120F26D12E
:1094000099F80000042804BF99F80100102804D03E
:1094100000261CE0A046019C19E009F1020144B1BC
:109420002046102210261AF090E8B869066001263E
:109430000DE0404610221AF02EE80028F7D0002652
:1094400004209121682200230096FCF751FDBBF116
:10945000720F12D1BAF1240F06D148464146242298
:109460001AF018E8002841D0002091210090042033
:1094700068220023FCF73CFD39E002A90020524697
:10948000CDF8089011F008F988B3029909EB0A02A7
:1094900091420CD082460020912100900420682245
:1094A0000023FCF725FD504611F002F91FE001688A
:1094B0008246486828B110F0C5F90528EBD1DAF8E2
:1094C00000100868FEF74DF958451BD0BBF1040F9A
:1094D00008BF082816D0BBF1030F08BF072811D01A
:1094E00000209121009004206422D9E70126396AE6
:1094F0004846FCF7DCFC4846FCF78FFC304603B0DE
:10950000BDE8F08FA4B15846FEF7B6F8FDF759FB59
:10951000D8B1FDF768FBD046024658F8040F016841
:109520008A4216D000209121009004208F22B7E7B4
:10953000DAF804000168A942ADD1816840462A46A4
:1095400019F0A8EF0028A6D10CE0D04658F8040F77
:1095500002688168204619F0F8EFD8F80000B96970
:109560000068086001269EE7B0B502AF84B0D7F866
:109570000CC0D7F808E09CF83C4014F0400F0AD02B
:10958000DCF80840256B002D2C4604D0A44604B01E
:10959000BDE8B04060470024CDE900430023CDE999
:1095A00002ECFFF7C7FE04B0B0BD2DE9F04703AFF2
:1095B00086B004209846CDE9022002A8049100213B
:1095C000002410F0C1FED7F818A0064650460DF052
:1095D00044FDA0F10B018E4204DD042076217022AF
:1095E000009423E000F1010946F68301C0F2020174
:1095F000002248460024FCF731FB054695B102A83D
:1096000001A9019510F0A0FE0120294600903046E6
:10961000424653460DF031FD01280BDB79690124E8
:10962000086008E000940420762141220023FCF722
:109630005FFC07E0002428464946FCF738FC284632
:10964000FCF7EBFB204606B0BDE8F08700F000B861
:10965000F0B503AF81B046F683015820C0F2020195
:1096600000220025FCF7FAFA0446B4B346F6E46695
:10967000C0F2080635681DB90CF007FE05463560D6
:1096800000200021C4E9000004F110002022A560A0
:109690001AF06CE801200021A06304F140001822B8
:1096A0001AF064E8686A04F13005214620F480600D
:1096B000E06306202A460EF087F950B1A068C16920
:1096C00099B12046884780B9062021462A460EF0E7
:1096D0008AF92046FCF7A1FB06E004206A2141221A
:1096E00000230095FCF704FC0024204601B0F0BDE7
:1096F000B0B502AF04460D46A068016A09B1204624
:109700008847A560E96909B1204688470120B0BDB6
:10971000D0B502AF04461CB1A06B0138A06300DDD8
:10972000D0BDA068016A09B12046884704F1300223
:10973000062021460EF057F9206908B1FCF72BFCF2
:10974000606908B1FCF727FCA06908B1FCF723FCAD
:10975000E06908B1FCF71FFC206A08B1FCF71BFCAC
:10976000606A08B1FCF717FCA06A08B1FCF713FCAB
:10977000E06A08B1FCF70FFC206D08B103F0DEF8D9
:10978000606D08B103F0DAF8E06C08B1FCF74BFA51
:109790002046BDE8D040FCF740BB2DE9F04F03AFB9
:1097A00083B00D46816898469246002D4E6911D0CF
:1097B000D0F814B03046DAF80040FCF753FF84428A
:1097C0000CD200251020DA21642200230095FCF73A
:1097D0008FFB1BE03046FCF745FF14E0DBF804008C
:1097E000D7F8189010B1FDF7FCF900E0402002A96D
:1097F000CDE9001641464A462B46FCF76AFF05466E
:10980000012D03DB02980125CAF80000284603B0A9
:10981000BDE8F08F2DE9F04303AF83B0894681683E
:1098200040691D46D7F8108016464C69406810B153
:10983000FDF7D7F900E04020294642464B46CDE9E6
:109840000064FCF77AFF03B0BDE8F083F0B503AF26
:1098500081B006461446B0680D4698B1F16889B1EA
:10986000CDB1486901F08FFF0246B06821684369B5
:10987000002000902846FCF740FB0546002D16DB33
:10988000256013E000251020D9218C2200230095AB
:10989000FCF72EFB0BE0406901F051FF00F017FCD4
:1098A0000730C11700EB5170C01020600125284619
:1098B00001B0F0BDB0B502AF82B005460C46A86855
:1098C000F0B101F05EFD024612B320464FF4CC71B8
:1098D00016F0EAFAA868406901F031FF00F02BFBAE
:1098E0000546ADB16069294601F02BFF80B12846DD
:1098F00000F04FF9606902B0BDE8B04001F087BDEB
:109900000020C721009010208B220023FCF7F0FAE2
:10991000002002B0B0BDB0B502AF46F683010446E8
:10992000C0F20201082000220025FCF797F918B1C7
:10993000C0E90055012560612846B0BD2DE9F04120
:1099400003AF884646F683010646C0F202010820AE
:1099500000220025FCF782F904467CB1C4E90055D9
:109960007461D8F81450286818B100F0E4FA206047
:1099700018B168680125606000E000252846BDE850
:10998000F081D0B502AF446944B1206808B100F05D
:1099900000F92046BDE8D040FCF73FBAD0BDF0B595
:1099A00003AF81B044690D46206880B101F0E9FC45
:1099B0000646C6B12168304601F0C3FE04467CB1BC
:1099C00028464FF4CC71324616F06EFA0CE00024B3
:1099D0001020DB218B2200230094FCF789FA03E09E
:1099E000304601F0F2FC0024204601B0F0BDF0B595
:1099F00003AF81B046691C460B2930D8012540F6DB
:109A0000A40305FA01F0184244D1012927D12046C8
:109A1000FDF7E7F8402820D02046FDF7E2F8B0F542
:109A2000D07F1AD02046FDF7DCF840F2A32188420F
:109A300013D02046FDF7D5F8B0F5287F0DD020468D
:109A4000FDF7CFF840F2A121884206D02046FDF76D
:109A5000C8F840F2A22188421FD174600DE041F2A3
:109A6000010081420BD1104601F0B3FE04464CB117
:109A7000306808B100F08DF8346001250AE06FF01D
:109A8000010507E000251020C5218D220095002347
:109A9000FCF72EFA284601B0F0BD002510200095F5
:109AA000C5218A22F3E7B0B502AF82B0154645F270
:109AB000A122C0F20302044608461146F6F7E8EC7C
:109AC00020B16FF00104204602B0B0BD2846FDF77A
:109AD00094FE18B92846FDF7DFFE60B1002102228E
:109AE000CDE9000120464FF4CC7141F20103FDF7AE
:109AF000BFFA02B0B0BD00241020C6218D22002381
:109B00000094FCF7F5F9DEE7F0B503AF81B0054648
:109B10002DB3A86848B346F68301AC20C0F2020119
:109B200000220026FCF79AF804463CB304F1080032
:109B30006664C4E90056FCF76DFA04F11C00FCF7FA
:109B400069FA0420C4E90C66C4E90E0620462664BE
:109B5000A9688847D0B92046FCF75FF915E00024D2
:109B600010206C216C22009404E00024102000944A
:109B70006C2142220023FCF7BBF907E010206C2186
:109B8000412200230096FCF7B3F90024204601B0DF
:109B9000F0BDB0B502AF04461CB32068C16809B17E
:109BA0002046884704F1440000F01CF865683DB188
:109BB0002868C16A09B1284688472846FCF72DF96C
:109BC00004F10800FCF70BFA04F11C00FCF707FA9B
:109BD000E06B08B1FCF721F92046BDE8B040FCF786
:109BE0001CB9B0BDF0B503AF81B004466CB12568B7
:109BF0004DB1D5E90060E96888472846FCF70DF9C2
:109C00003546002EF5D10020206001B0F0BDD0B562
:109C100002AF04464CB12068C16A09B120468847AA
:109C20002046BDE8D040FCF7F8B8D0BDD0B502AFB3
:109C300004463CB32068016909B9C16809B12046EE
:109C4000884704F1440000F01EF8606808B100F095
:109C50002FF804F10800FCF79EF904F11C00FCF752
:109C60009AF9E06B28B1216CFCF721F9E06BFCF765
:109C7000D4F82046AC21FCF71AF92046BDE8D040C4
:109C8000FCF7CBB8D0BDF0B503AF81B004466CB1E2
:109C900025684DB1D5E90060296988472846FCF759
:109CA000BCF83546002EF5D10020206001B0F0BD93
:109CB000D0B502AF04467CB12068016B09B9C16A16
:109CC00009B12046884720464421FCF7F0F8204699
:109CD000BDE8D040FCF7A1B8D0BD2DE9F04103AFFD
:109CE00082B0054688462868416949B1D8F8001015
:109CF000884211D00026102000966A21652204E0D7
:109D0000002610206A21422200960023FCF7F0F87A
:109D1000304602B0BDE8F081454519D005F1440652
:109D20003046FFF75FFFD8F8444000E024688CB16C
:109D3000D4E9010188470146002952D0D4E9022321
:109D400020690090304600F05CF80028EED148E031
:109D50000126DDE7D8F80410686859B130B9284603
:109D600000F090F86860E0B3D8F8041000F0C1F893
:109D700028B936E018B1FFF79BFF0020686005F1B5
:109D8000080008F10801FCF702FA50B305F11C00C5
:109D900008F11C01FCF7FBF918B3D8F83000286370
:109DA000D8F834006863D8F83800A863E86BD8F8AE
:109DB0003C10C1B108B1FCF730F8D8F8400046F6C5
:109DC0008301C0F2020100220026FBF747FFE8638F
:109DD00000289DD0D8E90F1219F0B6EBD8F8400052
:109DE00006E0002694E708B1FCF717F80020E863C6
:109DF0002864414628684269284602B0BDE8F0411F
:109E000010472DE9F04703AF82B004461D461646C1
:109E100088468CB3D7F814A0206800E0006898B199
:109E20008168B142FAD1C168A94204BF01695145B4
:109E3000F4D14FF000091020D3216C220023CDF87B
:109E40000090FCF755F819E0B8F1000F11D046F674
:109E500083011420C0F2020100224FF00009FBF739
:109E6000FDFE58B1C0E90186C0E9035A21680160CE
:109E700020604FF0010901E04FF00009484602B0B0
:109E8000BDE8F087F0B503AF81B00546BDB12868E5
:109E9000806AD0B146F683014420C0F2020100225C
:109EA0000026FBF7DBFE0446C4B128682060816A07
:109EB00020468847D0B92046FBF7AFFF15E00024C5
:109EC000102079214322009404E000241020009403
:109ED000792142220023FCF70BF807E010207921BA
:109EE000412200230096FCF703F80024204601B02D
:109EF000F0BDD0B502AF82B003685A6B42B10C68B6
:109F0000A34210D00024102000947221652204E0A6
:109F1000002410207221422200940023FBF7E8FF66
:109F2000204602B0D0BD884203D002B0BDE8D04088
:109F300010470124F4E7B0B502AF054665B12868C3
:109F4000FFF7E2FD04463CB120462946FFF7C5FE77
:109F500018B92046FFF71DFE00242046B0BD00685A
:109F60007047406870472DE9F04103AF82B00C465E
:109F700098461646054694B1686820B92846FFF70A
:109F800081FF686000B32146FFF7B3FFE0B105F140
:109F900008006EB13146FCF7FAF860B914E000240D
:109FA00010206F21432200230094FBF7A1FF11E052
:109FB0000021FCF733F905F11C00B8F1000F05D0C2
:109FC0004146FCF7E4F820B9002403E00021FCF747
:109FD00025F90124204602B0BDE8F08140687047B1
:109FE000D0B502AF0C4600F108012046FCF7CFF8CF
:109FF00020B16068002818BF0120D0BD0020D0BD6E
:10A00000D0B502AF044604F11C0208461146FCF725
:10A01000BEF820B1206A002818BF0120D0BD002062
:10A02000D0BD016370472DE9F04103AF05461446EA
:10A03000E86B884620B1FBF7F0FE0020C5E90F0071
:10A04000B8F1000F4FF0010618BF002C10D046F6F3
:10A0500083012046C0F2020100220026FBF7FEFD2C
:10A06000E86328B14146224619F06EEA26462C6480
:10A070003046BDE8F081D0F800C0DCF818C0BCF173
:10A08000000F00D0604780B56F4682B000206D2180
:10A090000090102042220023FBF72AFF002002B08C
:10A0A00080BDD0F800C0DCF818C0BCF1000F00D0B3
:10A0B000604780B56F4682B00020B021009010202C
:10A0C00042220023FBF714FF002002B080BD01688C
:10A0D000096A01B1084780B56F4682B00020AD2102
:10A0E0000090102042220023FBF702FF002002B064
:10A0F00080BDD0B502AF82B0D0F800E0DEF86CC011
:10A10000BCF1000F0BD00C68A64504BF1468A6452F
:10A1100010D00020712100901020652204E0002062
:10A1200071210090102042220023FBF7E1FE002065
:10A1300002B0D0BD02B0BDE8D040604700E000688A
:10A1400070B1D0F808C08C4504BFD0F80CC094455D
:10A15000F5D1D0F810C09C4504BF40687047EEE7C9
:10A1600000207047B0B502AF98B104688CB10546C5
:10A17000204684688C42F8D1C468944204BF0469C4
:10A180009C42F2D1D0E9004090472868FBF745FE99
:10A190002C60B0BDB0B502AF05468DB10846FFF7E3
:10A1A00071FE044664B120462946FFF7A2FE40B97D
:10A1B0002068C16A09B1204688472046FBF72DFE7A
:10A1C00000242046B0BD80B56F4682B00368D3F846
:10A1D00038C0BCF1000F08D00A68934210D00020AC
:10A1E0007F2100901020652204E000207F21009054
:10A1F000102042220023FBF77BFE002002B080BD2E
:10A2000002B0BDE880406047D0B502AF82B0D0F860
:10A2100000E0DEF83CC0BCF1000F08D00C68A64599
:10A2200010D000207E2100901020652204E0002044
:10A230007E210090102042220023FBF759FE0020CF
:10A2400002B0D0BD02B0BDE8D0406047D0B502AF8B
:10A2500082B0D0F800E0DEF844C0BCF1000F08D0B6
:10A260000C68A64510D000207C21009010206522AB
:10A2700004E000207C210090102042220023FBF704
:10A2800037FE002002B0D0BD02B0BDE8D04060472C
:10A29000D0B502AF82B0D0F800E0DEF844C0BCF127
:10A2A000000F08D00C68A64510D00020B9210090FE
:10A2B0001020652204E00020B921009010204222E5
:10A2C0000023FBF715FE002002B0D0BD02B0BDE8B0
:10A2D000D0406047D0B502AF82B0D0F800E0DEF8E1
:10A2E00048C0BCF1000F08D00C68A64510D0002073
:10A2F000742100901020652204E000207421009059
:10A30000102042220023FBF7F3FD002002B0D0BD55
:10A3100002B0BDE8D0406047D0B502AF82B0D0F8FF
:10A3200000E0DEF848C0BCF1000F08D00C68A6457C
:10A3300010D00020B72100901020652204E00020FA
:10A34000B7210090102042220023FBF7D1FD00200E
:10A3500002B0D0BD02B0BDE8D0406047D0B502AF7A
:10A3600082B0D0F800E0DEF858C0BCF1000F0BD08E
:10A370000C68A64504BF1468A64510D000207021C3
:10A3800000901020652204E0002070210090102031
:10A3900042220023FBF7ACFD002002B0D0BD1C68B8
:10A3A000A645EBD102B0BDE8D0406047D0B502AFC2
:10A3B00082B0D0F800E0DEF85CC0BCF1000F0BD03A
:10A3C0000C68A64504BF1468A64510D00020732170
:10A3D00000901020652204E00020732100901020DE
:10A3E00042220023FBF784FD002002B0D0BD02B062
:10A3F000BDE8D040604780B56F4682B0D0F800C05D
:10A40000DCF85C3043B10B689C4510D00020D221B1
:10A4100000901020652204E00020D221009010203E
:10A4200042220023FBF764FD002002B080BDDCF86F
:10A43000603002B0BDE88040184780B56F4682B0FA
:10A440000368D3F864C0BCF1000F08D00A689342D7
:10A4500010D00020762100901020652204E000201A
:10A4600076210090102042220023FBF741FD0020BE
:10A4700002B080BD02B0BDE88040604780B56F4645
:10A4800082B0D0F800E0DEF868C0BCF1000F08D060
:10A490000B689E4510D00020772100901020652287
:10A4A00004E0002077210090102042220023FBF7D7
:10A4B0001FFD002002B080BD02B0BDE880406047B3
:10A4C00080B56F4682B0D0F800E0DEF870C0BCF115
:10A4D000000F08D00B689E4510D000207821009016
:10A4E0001020652204E000207821009010204222F4
:10A4F0000023FBF7FDFC002002B080BD02B0BDE8E8
:10A5000080406047B0B502AF82B0D0F800E0DEF81E
:10A5100074C0BCF1000F0DD041B1002452F824509A
:10A520002D68AE450CD101348C42F7D302B0BDE8A2
:10A53000B04060470020882100901020422204E0B3
:10A54000002088210090102065220023FBF7D0FC1A
:10A55000002002B0B0BDD0F800C0DCF878C0BCF17B
:10A56000000F08BF00F02AB86047B0B502AF86B050
:10A57000D7F808C004ACD7F80CE0002B059305AD64
:10A58000CDF810C0CDE90054CDF808E018BF012384
:10A59000BCF1000F18BF4FF0010C03EA0C03FFF7EA
:10A5A000DAFF06B0B0BD01688A6F1AB1D1F8801029
:10A5B00011B1084700F0D0BE002070472DE9F04FE0
:10A5C00003AF97B006460C4630689A46216890461D
:10A5D00088421AD1D7E90719B8F1000F1491BD6963
:10A5E00008BFBAF1000F1CD0BAF1000F08D000214B
:10A5F00055F821201268904207D101315145F7D317
:10A60000B9F1000F14D0002017E000251020BB2165
:10A61000652200230095FBF76BFC284617B0BDE8C8
:10A62000F08F3046214617B0BDE8F04FFFF7CBBDA5
:10A6300015F0C1FA8146002850D00E90B8F1000FF5
:10A6400025D03046FFF7CAFC8346BBF1000F30D05F
:10A65000706C4BF6AF514BF6B7524BF6F153C0F25C
:10A660000001C0F20002C0F20003FFF767FD06948C
:10A6700000280F96CDF82490CDE904B5CDF84C8094
:10A680001CBF816800292BD10020012135E000206A
:10A69000CDF84C80CDF8249000210F96CDE90554DB
:10A6A0000490002007900020039000200A900020D2
:10A6B00029E04FF000091020BB2171220023CDF8C2
:10A6C0000090FBF715FC00244FF0000A4FF0000B40
:10A6D00000264FF0000800250E9818E200259CE7A0
:10A6E0000169044630464B460A685946FFF701FDAA
:10A6F0000121002800F0FE80002007900020039038
:10A7000000200A9001200D9001EB0A0546F6830413
:10A71000C0F202040B91AE00214630460022FBF746
:10A720009DFA8346304621460022FBF797FA804681
:10A73000042000EB8500214600220895FBF78EFAE5
:10A7400081462146304600225C46C346FBF786FA26
:10A750008046002C00F0A880BBF1000F18BFB9F1B3
:10A76000000F00F0A180B8F1000F00F09D800020E4
:10A770001294CDF830800024CDF854900025C9F80B
:10A7800000000D9810EB0A001090CDF844B055D0A1
:10A79000DDF844900026002500244FF00008D04545
:10A7A0002EBF1398149850F82800FBF7E5FB010919
:10A7B0007C2902D94FF0060B16E04109182902D96D
:10A7C0004FF0050B10E081084A2902D94FF0040B25
:10A7D0000AE0452802D94FF0030B05E04FF0010BCA
:10A7E000132888BF4FF0020B12980021D04509EBC7
:10A7F000060240F828B0159800EB880041605946E1
:10A8000013983CBF149850F8280000F015FB1599D8
:10A810000028885157D0ABF1010001210436CB4606
:10A8200001FA00F059F82810054408F10100A1428E
:10A8300088BF0C46109980468842B0D30B980028F8
:10A8400000F0FC800A9A002A40D0002016900D9952
:10A8500001BB14951298D16816AA40F82A101398D3
:10A8600000F0EAFA8046B8F1000F1AD0169B149D4A
:10A87000A3426DD9079D0B98684383427CD2E818A8
:10A88000294601381E46F5F71CEF0A998968884267
:10A890006FD9002000901020BB2144220023FBF739
:10A8A00027FB4FF000091FE00020BB210090102083
:10A8B00041220023FBF71CFBCA46002600250E9808
:10A8C0004FF0000923E1CB46002617E10D9801283F
:10A8D00000F0B4804FF000091020BB214422002377
:10A8E000CDF80090FBF704FB002600250E98DDF85C
:10A8F000308009E140466568FBF73EFB2946079139
:10A90000F5F7DEEED4E9022123460A9301306369AC
:10A910000139904288BF104600248A40934207D1F3
:10A9200000220D92012202FA01F103910146EBE6A9
:10A930001020BB214422002300260094FBF7D8FA04
:10A940004FF0000900244FF0000A4FF0000BC0E662
:10A9500015990AF10102002041F82A80089241F875
:10A9600022004BF82A300A980C99006941F82A0015
:10A9700064E0334650440890DDF82090CDF808801C
:10A98000D14553D915984646D04600EB8A0004308D
:10A990001390039880000390A9F101000B900A988E
:10A9A000D0F810B00B9880450AD21198AB4240F80D
:10A9B0002850C0F0D6815B1B0D931693284604E007
:10A9C000119840F8283018460D93139A0021154627
:10A9D0000022296046F68301C0F20201FBF73EF92E
:10A9E00045F8040C002800F0A181119D314655F86E
:10A9F000282018F0AAEDDBF80000002800F0A48160
:10AA00000C9A08F1010055F8281042F828B0A1422C
:10AA10008046039A079D88BF0C46139993442E44A1
:10AA2000484501F1040113910D9BBBD3CDF8209053
:10AA30000298FBF7F2F9149DDDF844B0042046F6C5
:10AA4000830100EB8500C0F2020100224FF00008F4
:10AA5000FBF704F90646002E48D0149546F82580E9
:10AA6000354610980D96E0B10D9D4FF0000B4FF05C
:10AA700001080C98002640F82B500F98FFF702FAB7
:10AA8000286040B312980136043550F82B00013885
:10AA900008FA00F08642F0D30BF1010B10988345C1
:10AAA000E7D30D9914980E4601EB8000854266D0DD
:10AAB0004FF000091020BB2144220023CDF8009064
:10AAC000FBF716FA00250E98DDF83080DDF854A06B
:10AAD000DDE911B41BE04FF0000900250E98DDF808
:10AAE00054A0DDE911B4DDE90C8610E01020BB2193
:10AAF00041220023CDF80080FBF7FAF900250E98DB
:10AB0000DDF830804FF00009DDF854A0129C08B148
:10AB100015F070F8B9F1000F1CBF4846FFF777F841
:10AB200014B12046FBF779F9BBF1000F1CBF584662
:10AB3000FBF773F9BAF1000F0DD0DAF8000038B165
:10AB40000AF10404FBF769F954F8040B0028F9D161
:10AB50005046FBF762F95EB1306830B1341DFFF743
:10AB6000A7F854F8040B0028F9D13046FBF755F943
:10AB7000B8F1000F1CBF4046FBF74FF94DE50F98A9
:10AB8000FFF780F9DDF844B08146002800F0C3806B
:10AB90001098002848D000254FF001080C98554522
:10ABA00050F8250000682EBF0499059951F825102A
:10ABB000FFF79FF9002800F0B180129850F82500A7
:10ABC00002282DD30C984946099B50F825000268AD
:10ABD0000F98FFF7EBFB002800F0A080129850F8C8
:10ABE000250001281CD000260C984B4650F8250063
:10ABF00050F8262000EB86004168099800900F98D5
:10AC0000FFF7ACFB002800F089801298711CB21C81
:10AC10000E4650F82500013808FA00F08242E3D3CE
:10AC2000013510988542B9D30D9A0F981499099B54
:10AC30001646FFF767FC00283FF457AEA4F1010A5F
:10AC4000CDF85090BAF1000F5DDB4FF00009012004
:10AC50006FF00308012510F0010F09D106990F9834
:10AC6000099B0A46FFF7A2FB0025002800F085801B
:10AC70000898E0B300265BF82600504533D91598B4
:10AC800050F8260010F90A40002C2CD004F0800067
:10AC9000B8BF6442B9EBD01F0ED035B90F980699F2
:10ACA000099AFFF7A8FB002866D0B9F1000F4FF012
:10ACB000000908BF4FF001090C9908EA4400002D73
:10ACC00051F826100B5804D006981946FFF711F9D1
:10ACD00006E00998009006990F980A46FFF73EFB98
:10ACE0000025002849D0013608988642C3D328465B
:10ACF000AAF1010A002D18BF0120BAF1000FAADA4B
:10AD00000D9E002D40D00F980699FFF75CFA0028A1
:10AD100043D1002542E04FF00009E6E500250E98FA
:10AD2000DDF854A0129CDDE90C86F0E60020BB2182
:10AD30000090102041220023FBF7DAF80298FBF77D
:10AD40006CF8DDF844B0ACE50020BB210090102089
:10AD500044220023FBF7CCF80298FBF75EF8AB46E1
:10AD60009FE50020BB210090102044220023FBF728
:10AD7000BFF8DDF844B094E500250E98DDF854A046
:10AD8000129CDDE90C860FE0B9F1000F05D00F9899
:10AD90000699099AFFF72FFBB9E701250E98DDF810
:10ADA0003080DDF854A0129CDDF85090AFE6816948
:10ADB000013181617047B0B502AF04461CB1A06992
:10ADC0000138A06100DDB0BD216961B1086838B10A
:10ADD0000D1DFEF71CFF55F8040B0028F9D1216961
:10ADE0000846FBF71AF82046BDE8B040FBF715B857
:10ADF000B0B502AF04461CB1A0690138A06100DD06
:10AE0000B0BD25697DB1286850B1FEF751FF2846D5
:10AE10000421FBF74CF855F8040F0028F5D12569FB
:10AE20002846FAF7FAFF20461C21FBF740F8204697
:10AE3000BDE8B040FAF7F1BF2DE9F04F03AF87B09E
:10AE40000546914668680E46002800F08780701E0F
:10AE500007287DD2E9684FF0FF3A28684FF0FF38A5
:10AE6000002908BF4FF0010A002871D02846FBF7DF
:10AE700083F8014600F1010B059146F68301C0F20B
:10AE80000201584600220024FAF7E8FE002874D098
:10AE9000CDE9019B0121069001FA06F4286808EB30
:10AEA00044014FEA44084FF00009006800EA010B32
:10AEB0004810039060420490BBF1000F23D01BF0B8
:10AEC000010F28D058461BEA040F0AD0039806EB5E
:10AED0000901059A013100EA0B00914238BFABEB42
:10AEE0000800A0422ADA0499884227DD10F0010107
:10AEF00024D0ABEB000BA34518BFBBF1000F0BD068
:10AF0000C34509D01AE006EB0900059901308842D3
:10AF100041D24FF0000B002000FB0AF0069901F827
:10AF2000090006EB0900411C2846FBF795FAB040E2
:10AF300000EB6B0B09F10109C345BDDD00208F213A
:10AF40000090102044220023FAF7D2FF069C1BE059
:10AF50000024102000948F21442212E046F6830141
:10AF60000120C0F20201002201250024FAF776FE3A
:10AF700018B10470C9F800500AE010208F21412256
:10AF800000940023FAF7B4FF2046FAF746FF0020AA
:10AF900007B0BDE8F08F02988145CFD80198C0F87E
:10AFA00000900698F4E72DE9F04F03AF8DB081468D
:10AFB00009F1440A4BF6B7524BF6F1530D464BF6E6
:10AFC000AF51C0F20001C0F20002C0F200035046CF
:10AFD000FFF7C8F8B9F1000F20D046F683011C2016
:10AFE000C0F2020100224FF00008FAF737FE0446D3
:10AFF000BCB108200421C4E9009048460122C4E9FC
:10B000000281C4E90488A261FEF7E8FF8046B8F136
:10B01000000F0FD0FDB100200C9023E04FF000088E
:10B020008FE11020C42141220023CDF80080FAF7DF
:10B030005FFF86E100261020BC21712200230B95C2
:10B040000096FAF755FF4FF000094FF0000B00256E
:10B050004FF0000850E114F0AEFD0146054600280F
:10B060000C912AD0284614F0EDFD284614F05BFE22
:10B070000646C6B1484631462A46FEF7B1FF90B1B2
:10B08000706810B33046FAF777FF01097C294FF05A
:10B09000060B4FF006010B952FD8410918291FD92F
:10B0A0004FF0050B2DE04FF00008284600254FF02B
:10B0B000000B4FF000090C9E20E14FF00008002526
:10B0C0004FF0000B4FF000091FE14FF00008102077
:10B0D000BC2172220023CDF80080FAF709FFE4E7D3
:10B0E00081084A2901D9042107E0452801D9032113
:10B0F00003E00121132888BF0221052938BF4FF042
:10B10000040B0730ABF1010107910022C00800FADF
:10B1100001F60990042046F6830100EB8600C0F298
:10B120000201FAF79BFD0546002D00F0B1800020DA
:10B13000CDF814B00A9545F826004846FEF7A2FE61
:10B14000834676B100250A98BBF1000F40F825B080
:10B1500000F0BB8048460135FEF794FE8346B542B9
:10B16000F1D30496BBF1000F00F0A1804846FEF732
:10B1700089FE002800F09B8041460890FEF7B9FE4A
:10B18000002800F0B3800998002854D007990120C6
:10B190000B9E4FF0000888400690099801380190F6
:10B1A0000A980390089A484659463346FFF7FEF836
:10B1B000002800F09B80039D08992868FEF799FEFF
:10B1C000002800F0938004350798CDF8088090B1EE
:10B1D0004FF0010855F8043C484629685A46009645
:10B1E000FFF7BCF8002800F0818008F10108043561
:10B1F00006988045EED30395DDE90108804515D218
:10B20000089948460B9B5A46FFF7D0F8002800F0F3
:10B210009C800225089948460B9B0A46FFF7C6F812
:10B22000002800F092800135072DF3D908F10108BC
:10B2300009988045B6D3049E48460A9D0B9B31462B
:10B240002A46FFF75FF94FF00008002851D0082088
:10B2500004F10C01C4E900904BF6AF5209984BF68B
:10B26000B753A060C0F200020598C0F2000361C1AC
:10B270004BF6F150C0F20000009050462146FEF718
:10B28000C0FD00281CBF444601200025804630E058
:10B290000020BC210090102041220023FAF728FE54
:10B2A0004FF0000B4FF000084FF0000923E04FF083
:10B2B00000091020BC2141220023CDF80090FAF7AC
:10B2C00017FE4FF000080A9D15E04FF0000910200E
:10B2D000BC2141220023CDF80090FAF709FE4FF07F
:10B2E000000B4FF000080C9E0A9D05E04FF000088F
:10B2F0000A9DDDF820900C9E0B9808B114F0E9FC33
:10B3000016B1304614F076FC14B12046FFF753FD19
:10B310005DB1286830B12C1DFEF779FC54F8040BA0
:10B320000028F9D12846FAF778FDBBF1000F1CBFC1
:10B330005846FEF76CFCB9F1000F1CBF4846FEF7FB
:10B3400066FC40460DB0BDE8F08F4FF000080C9E43
:10B350000A9DDDF82090CFE780B56F46406C4BF634
:10B36000AF514BF6B7524BF6F153C0F20001C0F2A9
:10B370000002C0F20003FEF7E1FE002818BF012022
:10B3800080BDD0B502AF82B046F683012420C0F262
:10B39000020100220024FAF761FC60B101210422BD
:10B3A0000462C0E90014C0E90244C0E90442C0E9F3
:10B3B0000614044606E01020B62141220023009422
:10B3C000FAF796FD204602B0D0BDD0B502AF0446D4
:10B3D0001CB1A0690138A06100DDD0BD606808B172
:10B3E000FEF7D7FBA06808B1FEF711FCE06808B1D2
:10B3F000FAF7D1FD04F12000FEF7F4FB20462421EA
:10B40000FAF755FD2046BDE8D040FAF706BD2DE914
:10B41000F04703AF82B00546002D45D0686800288C
:10B4200042D0FAF7FBFD8146B9F1000F45D014F088
:10B43000C2FB8046B8F1000F4BD0EE6826B9FAF790
:10B44000EDFD0646002E46D0686849464246FEF7A6
:10B45000C7FDA0B33046494613F0C5FA78B370680B
:10B460000028F7D0D5F808A0BAF1000F06D1686817
:10B47000FEF708FD8246BAF1000F20D0686800246C
:10B48000514632460023CDE90048FFF76EF810B16F
:10B490000124C5E902A64846FAF7A1FDA86890B9BB
:10B4A0005046FEF7B4FB0EE000241020B3214322E7
:10B4B00000230094FAF71CFD17E0002415E048462D
:10B4C000FAF78DFD0024E86848B93046FAF787FDA1
:10B4D00005E04FF000084846FAF781FD0024B8F176
:10B4E000000F1CBF404614F085FB204602B0BDE8AB
:10B4F000F0872DE9F04303AF83B0054665B1686876
:10B5000050B1A96841B1FEF798FF88B1002610201C
:10B510000096B1216A2204E000261020B1214322C6
:10B5200000960023FAF7E4FC304603B0BDE8F08350
:10B5300014F041FB044684B36868FEF7A3FC804620
:10B54000B8F1000F26D0D5E901012246FEF796FF9B
:10B5500028B36868C16841B3AB684146002200F176
:10B560000809CDE900940026FEF7FFFFD0B3686814
:10B570004146FEF762FF38B1E868002840D04946EE
:10B58000FAF7FCFE002816DB002610200096B121F9
:10B5900082222BE0204614F02DFB0026C4E7002673
:10B5A00010200096B1216B2220E00026102000968A
:10B5B000B1217A221AE068680026EA684146002331
:10B5C000CDE90064FEF7D1FF60B1D5E90102414643
:10B5D0002346FEF78EFD98B1002610200096B1217B
:10B5E0007B2203E01020B121102200960023FAF7FD
:10B5F0007FFC204614F0FEFA4046FEF708FB93E776
:10B600000126F6E72DE9F04F03AF83B00646144656
:10B610000D46A6B39CB395B3706880B314F0CBFA13
:10B620008146B9F1000F36D07068FEF72BFC8046DA
:10B63000B8F1000F2CD07068FEF791FCFEF791FC7A
:10B640008246484614F06FFB8346484614F06BFB75
:10B65000029040F2971170688A451ED141462A46F1
:10B660002346CDF80090FEF713FEE8B3706841461C
:10B67000029B5A46CDF80090FEF74EFE1DE00024D6
:10B680001020E521432200230094FAF731FC32E038
:10B69000484614F0AFFA00242DE041462A462346DE
:10B6A000CDF80090FEF7D2FDF0B170684146029BE4
:10B6B0005A46CDF80090FEF70DFEA8B1284659462F
:10B6C000FAF75CFE20B902992046FAF757FEB0B1AE
:10B6D00000241020E521922200230094FAF708FCB0
:10B6E000484614F087FA03E0484614F083FA002431
:10B6F0004046FEF78CFA204603B0BDE8F08F304696
:10B70000414600F00BF838B13046FFF7F2FE044630
:10B71000002C18BF0124E3E70024E1E7B0B502AF35
:10B7200004460D46A06808B1FEF771FA6168284624
:10B73000FEF730FDA060002818BF0120B0BD4068B2
:10B740007047B0B502AF04460D46606808B1FEF719
:10B7500020FA2846FEF7EFFB6060002818BF0120A2
:10B76000B0BDC0687047B0B502AF04460D46E06892
:10B7700008B1FAF710FC2846FAF7DDFCE060002873
:10B7800018BF0120B0BD80687047006AFEF7D6BCC4
:10B790002DE9F04703AF82B00646D7F814A056F85B
:10B7A000200F99461546884629464A465346FEF7D5
:10B7B000C5FC04463CB9304641462A464B46CDF8C6
:10B7C00000A0FEF71EFB204602B0BDE8F087C0696E
:10B7D00070472DE9F04F03AF89B00446012C0EDB12
:10B7E00045F2B4200021C0F20300043050F8042CCC
:10B7F000A24207D0013110304329F7D337E14FF08F
:10B80000000A3EE1D0E9008B14F0D5F9002862D09F
:10B8100007900022D8E9010905904946404400F10B
:10B82000100A5046FAF712FD054600266DB30AEBE2
:10B830000900494600220026FAF708FD28B306460B
:10B840000AEB490049460022CDF80CA0FAF7FEFCAD
:10B85000D8B1089606460495BBF1000F069646D06F
:10B86000D847FEF751F98246BAF1000F00F09F80E9
:10B87000DAF8000033460499089A85690798009021
:10B880005046A847002848D191E00020AF210690FB
:10B89000002000901020032200230896FAF728FBCE
:10B8A0004FF0000A5046FEF774F9079814F0A2F919
:10B8B0004FF0000A002D28464FF000014FF0000B1A
:10B8C0004FF000094FF000064FF000084FF0000560
:10B8D00040F0A980ADE00020AF210090102041226F
:10B8E0000023FAF705FB0020FEF753F9BFE0D8F874
:10B8F0000000B0F5CB7F06D1049832460899079B2B
:10B9000000F0C3F805E0049832460899079B00F060
:10B91000F9F88246BAF1000F5FD05046FEF7B2FA4E
:10B92000002844D0039E4946019009EB4900304469
:10B9300000224FF0000BFAF789FC0290002840D05B
:10B9400006EB890049460022FAF780FC0346C3B3A0
:10B95000079E504600961D46DDE90112FEF776FC73
:10B9600000283FD0039909EB890000224FF0000B1B
:10B9700008444946FAF76AFC8146B9F1000F36D00F
:10B98000D8F80C100298FAF749FC80B30199504698
:10B99000029B4A46FEF7E7FA78B3059A2AB1039864
:10B9A000811A5046FEF73FFB38B3AB4633E0002028
:10B9B00000901020AF2110220023FAF799FA049D7D
:10B9C00070E71020AF2103220023CDF800B0FAF772
:10B9D0008FFA4FF00009079E18E04FF0000ACDF8EB
:10B9E00000A0E6E74FF00009CDF8009007E0CDF8A1
:10B9F00000B01020AF21032204E0002000901020AE
:10BA0000AF2110220023FAF773FAAB465046FEF737
:10BA1000C0F84FF0000A0198FEF7F9F8304614F02C
:10BA2000E9F8049802990D46FAF7D9FA2E46D84655
:10BA30004D46089808B1FAF7D2FA069808B1FAF715
:10BA4000CEFA15B12846FAF7CAFA16B13046FAF717
:10BA5000C6FAB8F1000F1CBF4046FAF7C0FABAF1B7
:10BA6000000F04D050462146FEF7DBFA09E04FF004
:10BA7000000A1020AE2181220023CDF800A0FAF7A1
:10BA800037FA504609B0BDE8F08F2DE9F04303AF17
:10BA900081B01D4690468946064604F06FFEFEF7CB
:10BAA00033F804464CB3204631464A464346009597
:10BAB000FEF7E1FA10BBFAF71EFA00F07F41B1F190
:10BAC000805F17D16FF31F308738022812D2FAF740
:10BAD00011FA2046FEF7AAF800F075FDFEF714F8FB
:10BAE000044654B1204631464A4643460095FEF787
:10BAF000C2FA18B92046FEF799F80024204601B092
:10BB0000BDE8F0832DE9F04303AF81B01D469046B8
:10BB10008946064600F014F8FDF7F6FF044654B1D6
:10BB2000204631464A4643460095FEF7BAFA18B910
:10BB30002046FEF77BF80024204601B0BDE8F083E4
:10BB400048F63450C0F203007047D0B502AF044647
:10BB500004F14800FAF75EFA04F17400FAF75AFAB1
:10BB600004F18800FAF756FA0120D0BDD0B502AF33
:10BB7000044604F14800FAF732FA04F17400FAF7C7
:10BB80002EFA04F18800BDE8D040FAF728BAD0B503
:10BB900002AF044604F14800FAF7FDF904F174001D
:10BBA000FAF7F9F904F18800FAF7F5F904F15C0005
:10BBB0000021142217F0DAED4FF0FF302067D0BDDE
:10BBC0002DE9F04103AF0D46044604F1480005F1AC
:10BBD0004801FAF7DCFA002855D004F1740605F1A3
:10BBE00074013046FAF7D3FA00284CD004F18808E3
:10BBF00005F188014046FAF7CAFA002843D0E86DFB
:10BC0000E065296E2166696E6166A96EA166E96EBE
:10BC1000E166296F216700F11F01CA1701EBD261AC
:10BC2000E26F4911914204DD3046FAF797FA50B3BA
:10BC3000E06D1F30C11700EBD1604111D4F89000C6
:10BC4000814203DD4046FAF789FAE0B1D4E91E01EA
:10BC5000884207DA3168002241F820200130E36F82
:10BC60009842F9DBD4E92301884209DAD8F80010B8
:10BC7000002241F820200130D4F890309842F8DBBF
:10BC80000120BDE8F0810020BDE8F0812DE9F047FA
:10BC900003AF82B0044604F1480698461546304684
:10BCA000FAF775FA002854D004F15C0A30460622EF
:10BCB000514602F0EFFD40F0020006284BD104F19E
:10BCC000740929465246484602F0D4FC002840D068
:10BCD000E06DE26F1F30C11700EBD160411191425E
:10BCE00004DD4846FAF73AFA98B3E26FA06F904243
:10BCF00008DAD9F80010002241F820200130E36F63
:10BD00009842F9DB04F1880541465246284602F084
:10BD1000B1FCF0B1E06DD4F890201F30C11700EBFA
:10BD2000D1604111914205DD2846FAF717FA80B13A
:10BD3000D4F89020D4F88C00904208DA29680022C8
:10BD400041F820200130D4F890309842F8DB0124EB
:10BD500009E0002407E000241020C32183220023EF
:10BD60000094FAF7C5F8204602B0BDE8F087F0B5B8
:10BD700003AF81B01C461646054631B105F14802B5
:10BD800008461146FAF703FA78B12EB105F17401AD
:10BD90003046FAF7FCF940B12CB105F18801204694
:10BDA000FAF7F5F908B1012000E0002001B0F0BD7C
:10BDB00080B56F464830FAF7DFF8013880BD2DE9CD
:10BDC000F04103AF82B00C46064614B14FF00008B4
:10BDD00005E013F0F0FE0446002CA04622D02046D9
:10BDE00013F030FF204613F09EFF054665B106F1C3
:10BDF000880106F15C02284602F03CFC20B16E6826
:10BE0000002E18BF012600E00026204613F061FF37
:10BE1000B8F1000F1CBF404613F0ECFE304602B0F4
:10BE2000BDE8F081002610209F21412200230096CA
:10BE3000FAF75EF8F2E7D0B502AF0446201DFAF734
:10BE4000E9F804F11800FAF7E5F804F12C00FAF724
:10BE5000E1F80120D0BDD0B502AF0446201DFAF7AD
:10BE6000BEF804F11800FAF7BAF804F12C00BDE8A6
:10BE7000D040FAF7B4B8D0B502AF0446201DFAF7A7
:10BE80008AF804F11800FAF786F804F12C00FAF7A2
:10BE900082F800202064D0BDB0B502AF0D46044644
:10BEA000201D291DFAF773F988B104F1180005F176
:10BEB0001801FAF76CF950B104F12C0005F12C01CE
:10BEC000FAF765F918B1286C20640120B0BD002094
:10BED000B0BD80B56F460020086401F12C00002140
:10BEE000FAF79CF9012080BD2DE9F04303AF81B042
:10BEF0001E4689464AB346B309F10404114620465A
:10BF0000FAF745F9002540B320460021FAF7DDFA9B
:10BF100009F1180831464046FAF739F9E8B14046C8
:10BF200000210025FAF7D1FAF9F7F9FF09F12C06FB
:10BF300001463046FAF72BF978B130460021FAF77E
:10BF4000C4FA0125C9F8405007E000251020A321BC
:10BF5000432200230095F9F7CBFF284601B0BDE846
:10BF6000F083F0B503AF81B01C4616460D46FEF7D0
:10BF700064FA28B100241020A2216A2200940CE067
:10BF8000F9F7CDFF014605F12C00FAF7F7F950B1AA
:10BF9000002410200094A22142220023F9F7A8FFD8
:10BFA000204601B0F0BD46B1291D3046FAF7EFF842
:10BFB00080B130460021FAF788FA4CB105F118013A
:10BFC0002046FAF7E4F828B120460021FAF77DFA76
:10BFD0000124E5E70024E3E72DE9F04F03AF89B042
:10BFE00092460E4651469B460446FEF726FA10B18D
:10BFF0003046594606E020465946FEF71EFA58B12B
:10C0000030465146FDF775FF0446002C18BF012449
:10C01000204609B0BDE8F08FBD690DB1002004E0F5
:10C0200013F0C9FD0546002851D00890284613F0AA
:10C0300009FE284613F077FE8046284613F073FE6B
:10C040000790284613F06FFE8146284613F06BFEDA
:10C050000690284613F067FE0490284613F063FE0E
:10C060000390284613F05FFE0590284613F05BFE10
:10C07000002878D00290DAF8400060B10AF104019B
:10C080004046FAF784F800286DD007980AF11801A5
:10C09000FAF77DF806E0079B204651464246009598
:10C0A000FEF73AF900285ED0DBF8400088B1CA46B6
:10C0B0000BF104015046FAF76AF8002853D00BF14F
:10C0C0001801DDF818B05846FAF761F80BE00024C3
:10C0D0009EE75946DDF818B0CA46204652460095FC
:10C0E0005B46FEF719F9F0B340465146FAF72AF9D4
:10C0F000002845D002984146524602F068FADDF821
:10C10000149080B3079948465A4602F060FA50B33B
:10C1100020684946029B4A46D0F88CC020460095CC
:10C12000E04700B320684A46DDF810802B46D0F87F
:10C1300088C020464146E047A8B104F17402404659
:10C14000414602F044FA70B1404641464A4602F088
:10C150003EFA40B1029A4046414602F038FAC146E2
:10C16000DDF8208043E00024DDF82080284613F02D
:10C17000B0FDB8F1000F1CBF404613F03BFD47E790
:10C1800007985946FAF7DEF8DDF820800028DDF838
:10C19000149054D1DAF80400002850D020684946A1
:10C1A0005A465346D0F88CC020460095E0470028F8
:10C1B0004ED048464946524602F009FA002847D078
:10C1C00020684A46DDF810902B46D0F888C02046FB
:10C1D0004946E047E0B3059A4846494602F0F7F978
:10C1E000B0B304F174024846494602F0F0F978B35E
:10C1F0005146DDF80CA04A46504602F0E8F938B343
:10C2000020685146059B5246D0F884C020460095D0
:10C21000E047D146E0B1049A4846494602F0D7F9D2
:10C22000B0B1484649465A4602F0D1F980B1049A65
:10C23000204631464B460095FEF72AF803E020469B
:10C240003146FDF7C0FF0446002C18BF01248DE7DE
:10C2500000248BE780B56F4682B000931346FFF74A
:10C26000BBFE02B080BDF0B503AF81B015460C46F1
:10C270000646FEF7E2F880B9E06970B13046214623
:10C280002A46FEF71DF958B104F11800211D024697
:10C2900001B0BDE8F04002F09AB9012001B0F0BD54
:10C2A0000020FBE7096B0020002908BF0120704730
:10C2B0002DE9F04F03AF83B014460D460646FEF756
:10C2C000BCF808B101256AE0286C002865D0306808
:10C2D000002CD0E9219B02D04FF0000806E013F0BB
:10C2E0006AFC8046B8F1000F444656D0204613F051
:10C2F000A9FC204613F017FD0290204613F013FD11
:10C300008246BAF1000F3CD0CDF804B005F1040B21
:10C3100006F174025046594602F059F988B3304686
:10C32000514652465B460094C84750B318355046B4
:10C3300051462A4602F04BF918B330465146524650
:10C340005B460094C847E0B106F18802504651466A
:10C3500002F03DF9A8B1DDF808903046019E2A466A
:10C3600023464946B04760B1504651464A4602F01E
:10C370002EF930B1DAF804000025002808BF0125A5
:10C3800001E04FF0FF35204613F0A3FCB8F1000F99
:10C390001CBF404613F02EFC01E04FF0FF3528464D
:10C3A00003B0BDE8F08F2DE9F04F03AF83B099469D
:10C3B00092460D460446FEF740F806462046514692
:10C3C000FEF73BF826B10024002808BF012401E055
:10C3D00020B10124204603B0BDE8F08F286CA8B13D
:10C3E000DAF8400090B1281D0AF10401F9F7C6FF00
:10C3F000002440B905F118000AF11801F9F7BEFF51
:10C40000002808BF012484F00104E3E7B9F1000F1C
:10C4100001D0002005E013F0CEFB8146B9F1000FFA
:10C4200046D00290484613F00DFC484613F07BFCC2
:10C430008346484613F077FC0646484613F073FCE3
:10C440000190484613F06FFC8046B8F1000F23D0EE
:10C45000294620465A463346CDF800905D46FDF702
:10C460005BFFC8B12046019C51464346CDF8009081
:10C470002246FDF751FF78B128462146F9F77EFFA5
:10C48000002430B930464146F9F778FF002808BF4C
:10C49000012484F0010401E04FF0FF344846029D7E
:10C4A00013F017FC002D95D0284613F0A3FB91E75D
:10C4B0004FF0FF348EE72DE9F04703AF82B00E4610
:10C4C0000546306C144620B928463146FDF7B5FFC5
:10C4D00020B10125284602B0BDE8F08714B14FF025
:10C4E000000806E013F067FB8046B8F1000F4446F1
:10C4F00035D0204613F0A6FB204613F014FC8246EC
:10C50000204613F010FC8146B9F1000F1CD02846DC
:10C51000314652464B460094FDF7FEFEA0B1301D59
:10C520005146F9F734FE78B106F118004946F9F79B
:10C530002EFE48B106F12C000121F9F76FFE0546E9
:10C54000002D18BF012500E00025204613F0C1FB97
:10C55000B8F1000F1CBF404613F04CFBBAE70025B2
:10C56000B8E72DE9F04303AF81B00E4698469146F7
:10C5700004465EB100252068424659F82510036F35
:10C580002046984720B10135B542F4D3012000E0A0
:10C59000002001B0BDE8F08300F15C0C08461146B4
:10C5A0001A46634602F0AFB900F15C0C084611462A
:10C5B000624602F076BA00F1480C084611461A4667
:10C5C000634602F0AEBC48F6D050C0F2030070479C
:10C5D000D0B502AF044614F07FF80021C4E9281159
:10C5E000D0BDD0B502AF0446D4F8A00020B101F010
:10C5F00004FF0020C4F8A000D4F8A40020B1F9F78B
:10C60000EEFC0020C4F8A4002046BDE8D04014F0A1
:10C6100077B8D0B502AF0446D4F8A00020B101F03D
:10C62000ECFE0020C4F8A000D4F8A40020B1F9F773
:10C63000B2FC0020C4F8A4002046BDE8D04014F0AD
:10C6400070B8B0B502AF04460D46D4F8A00020B1D2
:10C6500001F0D3FE0020C4F8A000D4F8A40020B15B
:10C66000F9F799FC0020C4F8A4002046294614F0EC
:10C6700069F8B0B1D5F8A00048B101F095FEC4F852
:10C68000A00070B1D5F8A01001F063FF60B1D5F83B
:10C69000A40020B1F9F74FFDC4F8A40020B1012592
:10C6A00000E000252846B0BDD4F8A00000250028F1
:10C6B000F8D001F0A2FEC4F8A050F3E72DE9F04F46
:10C6C00003AF83B005469846D5F8A00091468A4648
:10C6D00020B101F092FE0020C5F8A000D5F8A4001A
:10C6E000BC6920B1F9F77BFC0020C5F8A40014B1A7
:10C6F0004FF0000B05E013F05EFA0446002CA34651
:10C700004AD001F051FE064686B3304651462246D5
:10C7100001F08DFE68B3CDF80880F9F77FFC804604
:10C72000B8F1000F23D0F9F7FAFB321D014640465D
:10C730003346009401F00CFDC8B1C5E928682846CD
:10C74000029B51464A46009414F01DF80446002608
:10C75000BCB9D5F8A00001F050FEC5F8A060D5F82E
:10C76000A400F9F73CFCC5F8A46000E00026002412
:10C7700007E000241020BD21032200230094F9F7D4
:10C78000B7FBBBF1000F1CBF584613F033FA26B1BC
:10C79000304601F032FE00E00024204603B0BDE840
:10C7A000F08FD0F8A0C0BCF1000F05D008461146AC
:10C7B0001A46634601F0CCBC80B56F4682B00020BB
:10C7C0008321009010206F220023F9F791FB0020B5
:10C7D00002B080BD80B56F4682B09C46D0F8A030D4
:10C7E0003BB108461146CDF800C001F0B1FC02B0E3
:10C7F00080BD00208421009010206F220023F9F7D3
:10C8000077FB002002B080BD80B56F4682B09C46A9
:10C81000D0F8A03053B1CDF800C003F1040C0846A5
:10C820001146624601F094FC02B080BD00208621D2
:10C83000009010206F220023F9F75AFB002002B06D
:10C8400080BDD0F8A0C0BCF1000F04D0084611464E
:10C85000624601F085BD80B56F4682B0002085211B
:10C86000009010206F220023F9F742FB002002B055
:10C8700080BDD0B502AF82B0D0F8A42042B1084646
:10C880001146F9F784FC0446002C18BF012407E088
:10C8900000241020D1216F2200230094F9F728FBF7
:10C8A000204602B0D0BD2DE9F04303AF81B00E4663
:10C8B00046F6830190460546C0F202012C20002274
:10C8C0004FF00009F9F7CAF9044634B320460021B5
:10C8D0002C2216F04CEF25B12846F9F72CFC2060ED
:10C8E00020B326B13046F9F726FC6060F0B140462F
:10C8F000F9F721FCE060C8B198F8101011F0040FAE
:10C900001EBF016941F0040101614FF0FF30E06199
:10C9100004F114000BF0ABFA0CE003206621412275
:10C920000023CDF80090F9F7E3FA02E0204600F08A
:10C9300005F80024204601B0BDE8F083D0B502AF71
:10C940000446A4B1206808B1F9F749FB606808B152
:10C95000F9F745FBA06808B1F9F741FBE06808B1B9
:10C96000F9F73DFB2046BDE8D040F9F756BAD0BDF7
:10C970002DE9F04103AF82B0044688462068F8B143
:10C980006168E9B1254655F81C1FB1F1FF3F22D07F
:10C9900001312960202920D1A168F1B194F820103B
:10C9A00011F0020F19D10026204600210022434633
:10C9B000CDE9006600F033F8002818BF012625E015
:10C9C0000026032067216B2200230096F9F790FAD6
:10C9D00004F11C051AE00121296094F8201011F0DF
:10C9E000010F10D1E36801460246CDF800800EF039
:10C9F00056FD50B16068E368CDF8008001460246FC
:10CA00000EF04DFD08B1012600E000262868202820
:10CA100004BF00202860304602B0BDE8F0812DE957
:10CA2000F04303AF83B0814698460E464C46B9F1B9
:10CA3000000F07D1002000210025FFF734FF044636
:10CA4000002C63D0206820B9F9F7E8FA20600028AC
:10CA500044D0606818B9F9F7E1FA6060F0B3A068F3
:10CA600036B108B1F9F7BBFA3046F9F764FBA060BC
:10CA7000A0B3D7E9041001B1A16200B160622068DF
:10CA8000E16811F0B0FF48B302AE6FF02005D4E9C1
:10CA900000104346E268009600F04AF950B9029847
:10CAA000E0B1013512D02068E16811F09CFF002848
:10CAB000EDD113E0A66AB6B1616AA1B12068D4E9EC
:10CAC0000223CDE900810146B04714E00020802117
:10CAD0000090032071220023F9F70AFAB9F1000F40
:10CAE0000ED17CB90CE02068D4E90223CDF8008097
:10CAF000014600F03FFCB9F1000F08BF002801D04B
:10CB0000254603E02046FFF719FF0025284603B01D
:10CB1000BDE8F0832DE9F04103AF82B0164605462B
:10CB2000306898460C4660B1706850B1F069B0F159
:10CB3000FF3F0FD030464146FFF71AFF60B900248F
:10CB400020E00024032064216B2200230094F9F7E5
:10CB5000CFF917E00020F06144B171682046F9F781
:10CB600016FB0446002C18BF012400E001243268A3
:10CB70002846F3682946CDF800800EF090FC002886
:10CB800008BF0446204602B0BDE8F08180B56F467C
:10CB900082B08C46BCF1000F04BFD2F804C0BCF1D7
:10CBA000000F09D0D2F80CE00146009362467346AC
:10CBB0000EF075FC02B080BD0020652100900320BE
:10CBC0006B220023F9F794F9002002B080BD1430E5
:10CBD00070472DE9F04F03AF81B099468046484633
:10CBE00092468B4613F02EF8484613F09CF8064602
:10CBF000484613F098F805460024002E7CD0002DFE
:10CC00007AD030465946F9F7C2FA00285BD0284658
:10CC10005146F9F7BCFA002400286DD03046294669
:10CC2000F460EC60F9F7AAFBB2460028BCBFAA4644
:10CC300035462E4656F8040F002855D000242BE028
:10CC40002846294611F0A0FFE8B33068013418BB2C
:10CC50003BE0012804DB2868007810F0010F02D1C6
:10CC60002846294607E0504651462A4611F0B7FDAE
:10CC700048B35046514611F087FF20B3504629462D
:10CC8000F9F77CFB00282846BCBF5046AA4605465B
:10CC90002E4656F8040FDAE7DAF80410012905DB0E
:10CCA000DAF80010097811F0010FD2D1012804DB65
:10CCB0002868007810F0010FDBD15046514611F082
:10CCC00063FF0028BCD1002416E054B15046514601
:10CCD000224611F09DFF0024BAF1000F0CD018B9C4
:10CCE0000AE0BAF1000FEED040465146F9F74FFA8C
:10CCF0000446002C18BF0124484612F0EAFF2046E3
:10CD000001B0BDE8F08FD0B502AF82B001AC0094A5
:10CD100000F00EF80446019838B100206E21009012
:10CD200003206C220023F9F7E3F8204602B0D0BDBF
:10CD30002DE9F04F03AF93B08A46B9691C4605460A
:10CD400009B1002008609AF81000049210F0040F56
:10CD5000CDE9075404BF107C10F0040F00F0BC8034
:10CD6000204612F06FFF204612F0DDFF834620467A
:10CD700012F0D9FF0646204612F0D5FF8146204624
:10CD800012F0D1FF0590204612F0CDFF069020460C
:10CD900012F0C9FF8046204612F0C5FF002800F0BF
:10CDA0008F802846002D04D1F9F738F9002800F0CB
:10CDB0008780039048460121F9F730FA4446002164
:10CDC00020460025F9F72AFA30465146F9F7DFF9EF
:10CDD000002871D004995846F9F7D9F900250028A0
:10CDE0006AD0CBF80C50F06830B930465946F9F7A4
:10CDF000A9FA002814DBF06831685A460991716875
:10CE00000A91B168CDE90B1006213069089B61F3E6
:10CE1000020009A90D9030460EF0DDFA00284AD034
:10CE200006984FF0FF31354682466868002800F0CA
:10CE30000A8206914E46DBF8000051460E90D84615
:10CE4000DBF804002B460F90DBF808001090DBF8AD
:10CE50000C001190DBF81000129A20F00700DDF8AA
:10CE6000149002F00102DDF820B010430EAA40F049
:10CE7000060012904846CDF800B010F02BFC0028B8
:10CE800000F006824046494632465B4611F070FA91
:10CE9000D946002800F0F98140464146224611F06B
:10CEA00065FB0699002820463446C1F10001C146C1
:10CEB000AB465646B7D10025DDF82090039903E034
:10CEC000DDF82090002100250798284304BF08467C
:10CED000F9F785F84846F2E12046564612F0B2FED0
:10CEE000204612F020FF8346204612F01CFF254604
:10CEF0008246284612F017FF8146284612F013FF9B
:10CF00000590284612F00FFF8046284612F00BFFCE
:10CF10000690284612F007FF0446002C00F0CD8052
:10CF2000079820B9F9F77AF8002800F0C680039036
:10CF300048460121F9F772F9069800210025F9F712
:10CF40006DF950463146F9F722F9002800F0AD811D
:10CF500004995846F9F71BF90025002800F0A5812F
:10CF6000CBF80C50DAF80C0028B950465946F9F7BE
:10CF7000E9F9002808DB089B504651465A460EF056
:10CF80002AFA002800F09081049A50680128C0F223
:10CF900099801068007810F0010F00F0938010461F
:10CFA000F8F7EAFF049AB0F5006F00F38B80DAF827
:10CFB00004000028069800F0B9810024504621465C
:10CFC000F9F74AFAD0B9D9F8040001280DDBD9F8ED
:10CFD0000000007810F0010F07D0049A4846494637
:10CFE00011F0A6FB002800F05F8148464946013455
:10CFF00011F0CAFD00250028E0D156E1012C07DB25
:10D0000050465146224611F07DFE002800F04C812A
:10D01000002458462146F9F71FFAC8B9069D6868EA
:10D0200001280CDB2868007810F0010F07D0049A63
:10D030002846294611F07CFB002800F0358128465F
:10D040002946013411F0A0FD00250028E1D12CE192
:10D05000069D012C07DB58465946224611F052FE28
:10D06000002800F0218150465946F9F76BF9002855
:10D070000BDB484649462A4611F05AFB002800F0CF
:10D080001381504651465A460AE0284629464A46E8
:10D0900011F04EFB002800F00781584659465246D1
:10D0A00011F096FA002800F0FF80DAF8040000285A
:10D0B0007FF483AF069D049AEFE0DDF820A0002105
:10D0C0000025F5E00699DAF80400002800F0E48075
:10D0D0004FF0FF304646019450E0606801280DD1C2
:10D0E00020680068042810D0022816D0012804BF48
:10D0F000E068002813D14846294621E048462146E9
:10D100002A46534611F034F915E0E06838B948462C
:10D110002946022211F07CFD0DE0E06848B3484644
:10D120002946F9F734F8002800F08B802068016860
:10D1300048460DF0D0FF002800F08380484649465D
:10D14000424611F013FA00287BD0029A5B467168C0
:10D15000B24650424646002929460FD1CBE0204630
:10D160000121F9F75BF81FE020460221F9F756F894
:10D1700063E04846294611F0CAFCDCE7CDF8189078
:10D18000D946029048468846D346F8F7F5FE05464C
:10D190005846F8F7F1FE85420ED1059C0121204644
:10D1A000F9F73CF8DDF820A000284AD0304649467F
:10D1B0005A4611F014FB40E04846F8F7DDFE0546FC
:10D1C0005846F8F7D9FEDDF820A00130059C8542CD
:10D1D0002BD1019D5946284611F099FC88B3484649
:10D1E0002946F9F7AFF8B0F1FF3FB8DD30464946C0
:10D1F0002A4611F0F4FA20B3204629465A4611F087
:10D20000B5F9F0B148462146F9F79CF8B0F1FF3F77
:10D21000AADD20460321F9F701F8069D88B13046C2
:10D2200031465A4611F0DBFA08E0204631464A46BC
:10D230005B46CDF800A010F04DFA069D00287FF463
:10D240004CAF002533E0DDF82090B1F1FF3F05DC65
:10D2500004992046024611F0C2FAB0B1DBF804008E
:10D26000012808D1DBF800000068012804BFDBF8C2
:10D270000C00002829D0002503208B216C220023DC
:10D280000095F8F735FE03991EE6002503991BE685
:10D2900000250399D94617E60D46114628462A4629
:10D2A00011F09DFA049A50BB0025DDF820A00399E7
:10D2B0000798284304BF0846F8F791FE504612F03D
:10D2C00008FD284613B0BDE8F08FE06830B9049936
:10D2D0002046F9F737F8B0F1FF3F3FDD039E2146C6
:10D2E000049A4B4630460EF076F8002814BF3546B7
:10D2F00000253146E8E5012A049A9B46CDDADDF89F
:10D3000020A0DBF80400012808D1DBF80000006849
:10D31000012804BFDBF80C00002809D0BA690025F9
:10D320000399002A1CBF01201060C1E70546B4E73D
:10D33000E86838B928461146F9F704F8049AB0F1BC
:10D34000FF3F11DD039C2946534620460EF043F86B
:10D35000002814BF254600252146A9E7039E214643
:10D360003046F8F714FFC0E7039C29462046F8F73B
:10D370000EFFEDE780B56F4682B0D3F804C0BCF174
:10D38000010F06DBD3F800C09CF800C01CF0010FB1
:10D3900004D102B0BDE8804000F024BBD1F804E025
:10D3A000D7F808C0BEF1010F04BFD1F80CE0BEF100
:10D3B000000F0ED192F810E01EF0040F09D1096899
:10D3C0004FF0000E0968CDE900CE00F00AF802B077
:10D3D00080BD4FF0000ECDE900CE00F079F902B02B
:10D3E00080BD2DE9F04F03AF8BB0934606469BF806
:10D3F00010000C4610F0040F12D15868012804DB0D
:10D400001968096811F0010F18D14FF000080320C6
:10D41000752166220023CDF80080F8F769FD09E048
:10D42000002075210090032042220023F8F760FDC0
:10D430004FF0FF3840460BB0BDE8F08FFA69012885
:10D440000592BD69069303D12046F3F7B4E90C4673
:10D450005846F8F791FD8146B9F1000F00F0E080E1
:10D46000002C00F0E48028460794029612F0EAFBB4
:10D47000284612F058FC8246284612F054FC044616
:10D480002846099512F04FFCBAF1000F06464FF0FE
:10D49000000818BF002C00F01781002E00F0148146
:10D4A0000598099D002801460DD100F07DFF002858
:10D4B00000F0E18006992A46824600F0B8FF002875
:10D4C00000F0DC805146A9F102000A96002808917C
:10D4D000C0F2B480081D0390A9F10105DDF81C908D
:10D4E000012609FB09FA49465046F3F7EAE84845A0
:10D4F00006D106B3DDF828904FF001080A9447E002
:10D5000020464946002E04951CD0F8F787FEDDE939
:10D510000956002800F0CF8000952046039A214646
:10D52000089B00F015FE002800F0C580B1464FF0C2
:10D53000010A264604E004952646DDF82890099D58
:10D54000089B17E00DF0C7FD0028DDE9090600F093
:10D55000B28000900020069B314622464FF0000822
:10D5600010F0B8F8002800F0A8804FF0010AA1469A
:10D57000DDE9083530463146324600950A9600F01E
:10D58000E7FD049D4FF000080026002800F095807C
:10D59000013D58464C462946F8F75EFF08B3079907
:10D5A0000AFB01F94846F3F78CE850451AD0B8F168
:10D5B000010F1ED10A9E51463046F8F72FFE002873
:10D5C00079D00998314600903046039A089B00F0C4
:10D5D000BFFDDDF81C9031460A9400260C4620B9A8
:10D5E00069E0D1460A980A940446002D3FF779AFC6
:10D5F00027E0DDF82890514648460DF06CFD0028E4
:10D6000059D00998214600900020069B4A464FF0C9
:10D61000000810F05FF8DDF81C900028E5D14CE020
:10D62000304601210BB0BDE8F04FF8F7F7BD3046AA
:10D630000021F8F7F3FD4FF00108FBE60126DDF8C5
:10D640001C90B9F1010F06D1099D56B30298012132
:10D65000F8F7E4FD2BE0204649469EB1F8F7DEFDE1
:10D66000099D40B300952046089B21461A1D00F0F5
:10D670006FFDB0B91FE04FF0000825E04FF0000843
:10D6800051461BE00DF027FD099DA0B100952246F3
:10D690000A9C0020069B4FF00008214610F01AF863
:10D6A00058B102982146089A2B4600F059FE10B155
:10D6B0004FF0010801E04FF000080899059818B9EB
:10D6C00011B1084600F099FE099812F002FBB1E68C
:10D6D0002DE9F04F03AFA9B015460646287C8B46CE
:10D6E000D7E906419A4610F0040F14D1DAF8040085
:10D6F000012805DBDAF80000007810F0010F17D1DF
:10D700004FF0000803206D2166220023CDF8008031
:10D71000F8F7EEFB08E0CDE90041304659462A46CD
:10D72000534600F0A1FA8046404629B0BDE8F08F8C
:10D730002846F8F721FC002861D00590204607967E
:10D7400012F080FA204612F0EEFA0646204612F059
:10D75000EAFA8146204612F0E6FA02464FF0000847
:10D760000992002E069600F03481B9F1000F18BF1F
:10D77000002A00F02E81DDF81C80F869CDF81090A9
:10D78000002808900DD1164600F00EFE002842D069
:10D7900051462246089000F04AFE002800F00D8114
:10D7A0003246DBF80C0038B9584651461646F8F7B1
:10D7B000C9FD324600280BDB104616465946524634
:10D7C00023460DF008FE32460028934600F0F5800F
:10D7D000DBF80400C0B1089B16461046594603F119
:10D7E000040A0094524600F0B3FC002800F0E580E3
:10D7F0000598B0F5287F11DB062031461BE0304646
:10D800000121F8F70BFD8EE740460021F8F706FDF1
:10D810004FF00108D3E04FF00008DAE03146EF287E
:10D8200001DD052007E04F2801DD042003E0182872
:10D83000C0F2D38003200390DDF820900A460698BA
:10D8400000944B4600F084FC002800F0AE80039862
:10D8500001215646013801FA00FABAF1020F21DB24
:10D860000DF124080024D7F8189008EB840B4846E3
:10D8700012F059FACBF80400002800F09D80CDF892
:10D880000090DDF8209058F82410069A4B4600F0DE
:10D890005FFC002800F08C80601CA11C51450446F0
:10D8A000E1DBBC69B246F8F73AFB01460498524600
:10D8B0004B46009400F04CFC002876D005980126D9
:10D8C000A0F1010A01E0AAF1010A28465146F8F741
:10D8D000C3FD68B946B904984B4600940146024618
:10D8E00000F036FC002860D0BAF1000FEBD14FE019
:10D8F0000398069602281CDBAAF101044FF00008E9
:10D900004FF001094FF0010B002C16DB2846214691
:10D91000F8F7A2FD30B1A9EB0800C8460BFA00F0F9
:10D9200040F0010B013C09F1010903988145EBDB53
:10D9300003E04FF0010B4FF00008DDF8209006984F
:10D9400080B9B8F1000F0DDB4FF0FF34B8694B46DA
:10D95000009004980146024600F0FAFB40B30134FF
:10D960004445F3DB6FF0030009A900EA4B00BC69F2
:10D970004B4600940A580498014600F0E9FBA0B118
:10D98000AAF101000026A0EB080ABAF1FF3F9CDCD7
:10D9900007984A460499234600F0E2FC8046B8F115
:10D9A000000F18BF4FF001080BE04FF0000808E02F
:10D9B0004FF00008BC6904E04C464FF00008DDF869
:10D9C0002090F86928B9B9F1000F1CBF484600F053
:10D9D00014FD204612F07DF9A6E6DDF82090012026
:10D9E000039060E72DE9F04F03AFB1B0164604464F
:10D9F000307C98468A4610F0040F33D13046F8F751
:10DA0000BBFA8146B9F1000F37D00394BC692046B8
:10DA100012F018F9204612F086F98346204612F0DB
:10DA200082F904460025BBF1000F119418BF002CA9
:10DA300000F0108104A80DF073FBD8F80C0010B3AF
:10DA400058464146F8F7A3FB0025002800F0028164
:10DA5000BA6904A85946CBF80C500DF084FB012894
:10DA600019DAF7E000207D210090032042220023F4
:10DA7000F8F73EFA4FF0FF35F2E020460121F8F7C3
:10DA8000CDFB0546ECE0BA6904A841460DF06BFBFE
:10DA90000128C0F2DE80BD692046514642462B4631
:10DAA0000DF099FC002800F0D480606820B1B9F531
:10DAB000287F07DB062013E003980021F8F7AEFB70
:10DAC0000125C7E0B9F1EF0F01DD052008E0B9F14C
:10DAD0004F0F01DD042003E0B9F1180F34DB032000
:10DAE00004ABCDE900505846214622460DF052FBCA
:10DAF000002800F0AE80019C0121601E01FA00F0B8
:10DB00000228029021DB11AD0024D7F818A005EB04
:10DB10008408504612F007F9C8F80400002800F005
:10DB2000988055F8241004AB5A46CDF800A00DF0AB
:10DB300031FB002800F08D80601C029AA11C044675
:10DB40009142E2DB019C00E0012403980121F8F7F7
:10DB500065FB00287DD0A9F101090DF1100B4FF0F4
:10DB6000010A019430464946F8F776FC039CB8B99F
:10DB7000BAF1000F09D1B86921460090204622462B
:10DB80005B460DF007FB002863D0B9F1000F97D07A
:10DB9000A9F1010930464946F8F75EFC0028E7D0B4
:10DBA000019C022C1DDBA9F1010501204FF00008AA
:10DBB0004FF0010B0290002D17DB30462946F8F795
:10DBC0004BFC40B10299ABEB0800D84601FA00F0DB
:10DBD00040F0010002900BF1010B013DA345EADB8F
:10DBE00003E001204FF000080290BAF1000FD7F8CF
:10DBF00018A0039C0DF1100B10D1B8F1000F0DDB34
:10DC00004FF0FF352046214622465B46CDF800A066
:10DC10000DF0C0FAE8B101354545F3DB02996FF02C
:10DC200003005B46CDF800A000EA410011A90A58A4
:10DC3000204621460DF0AEFA58B1A9F101004FF08F
:10DC4000000AA0EB08090125B9F1FF3F3FF78AAFB1
:10DC500000E00025B86912F03CF804A80DF06DFA58
:10DC6000284631B0BDE8F08F2DE9F04F03AF95B0F5
:10DC70009B468246DBF800001546007810F0010F45
:10DC80000CD182B04FF0000A03207C2166220023D1
:10DC9000CDF800A0F8F72CF902B010E247F8481CC4
:10DCA000DBF8040047F8400C2846F8F765F9804691
:10DCB000B8F1000F18D0D7E90696484611F0C2FF18
:10DCC00034465EB900F070FB0446ECB1204659467C
:10DCD0004A4600F0ACFB002800F0B98040F2A930C1
:10DCE000804507DD062217E050460121F8F796FA35
:10DCF0008246E4E1B8F5997F01DD05220CE0B8F138
:10DD0000590F04DD042207E04FF0000AD4E101229C
:10DD1000B8F1160FC8BF032257F8401C012000FAC3
:10DD200002F947F8502C47F8445C480048454846FB
:10DD300047F85CACC8BF480091400144402000EB6C
:10DD40008100890047F84C1CB1F5406F06DA0730B6
:10DD500020F00700ADEB0005AD460BE046F6830171
:10DD60000022C0F202014FF0000AF7F777FF0546E4
:10DD7000002D67D005F03F0047F8580C57F84C6C61
:10DD8000C0F1400047F8608C05EB000800214FF01F
:10DD9000000A4046324615F0EAEC57F8401C57F8A6
:10DDA000502C88009040404447F8240C00EB810040
:10DDB00047E90E0A022047E908A147E90C1A47F88B
:10DDC00018AC47F8280C47F8140CF8F7A8F80146E7
:10DDD00082B02346B8691C1D0090A7F1240047F8C3
:10DDE0003C3C224600F0B4F902B0B6F5406F2E4636
:10DDF0003146B8BF0021002847F8541C00F0F180DC
:10DE000057F8482CD06838B910465946F8F79AFAAE
:10DE100057F8482C002823DB82B0B869A7F13801F5
:10DE20005B464FF0000A0546002000950FF052FCBB
:10DE300002B0002800F0D58082B0A7F1380000952C
:10DE4000014613E000254FF00008FE6923E10020A1
:10DE50004FF0000A002547F84C0C4FF000081AE17B
:10DE600082B0B86911460090A7F1380057F83C3CE1
:10DE7000224600F06DF902B0002800F0B08057F89B
:10DE8000400C57F8201C57F850BC47F8488C81428A
:10DE9000A8BF01460020B0EB810F0BD057F8483CDB
:10DEA0008900002257F8245CAD5C01321D704B44A0
:10DEB0008A42F7D357F8402C57F8341C9142A8BF38
:10DEC0001146B0EB810F0ED0880057F8581C002285
:10DED000C1F14101314457F8383C9B5C01320B7071
:10DEE00049448242F7D3BBF1020F60D382B0B869D4
:10DEF000A7F1380157F83C3C0090A7F124000A46EE
:10DF000000F026F902B04FF0000A002800F0BC80B3
:10DF100057F8401C57F8200C8842A8BF0846BAEBB7
:10DF2000800F0ED057F8581C80000022C1F142012A
:10DF3000314457F8243C9B5C01320B7049448242C7
:10DF4000F7D3B9F1040F32DB57F8580CA7F13808B2
:10DF5000A7F124050324C0F143004FF0000A064452
:10DF600082B057F83C3C4146B8692A4600902846A2
:10DF700000F0EEF802B0002800F0848057F8401C52
:10DF800057F8200C8842A8BF0846BAEB800F0AD089
:10DF900080000021324657F8243C5B5C013113704D
:10DFA0004A448142F7D3013401364C45D8DB57F857
:10DFB000600C5946451E2846F2F7A0EC002914DBF8
:10DFC00057F8448C4E1C002440462946F8F744FA82
:10DFD000013E00EB4404013D002EF5DC06E04FF06D
:10DFE000000AFE6957F83C4C53E0002482B057F811
:10DFF000401CA7F1240057F8482C2346CDF8009088
:10E0000000F075F802B0E8B3A7F12408002D5CDB3E
:10E01000D7F818A00024002682B057F83C3C4046B0
:10E0200041464246CDF800A000F092F802B048B355
:10E0300057F8440C2946F8F70FFA013400EB46066E
:10E04000013D5C45E8DB82B0A7F1380457F8401C7D
:10E0500057F8482C33462046CDF8009000F047F89A
:10E0600002B078B182B057F83C3C40464146224667
:10E07000CDF800A000F06CF802B04FF0000A0028C4
:10E08000C4D101E04FF0000AFE6957F83C4C57F844
:10E09000488C57F8545C1EB914B1204600F0ADF915
:10E0A000B8F1000F08D057F84C1C4046F7F7FFFEB8
:10E0B00015B12846F7F7B1FEB86911F00AFE5046CF
:10E0C000A7F10C04A546BDE8F08F57F83C4CA7F12A
:10E0D000240157F85C0CBB69224600F041F9FE6947
:10E0E0008246BAF1000F18BF4FF0010ACFE72DE9C1
:10E0F000F04103AF05469846A8680C461646A04274
:10E1000004DA28462146F8F729F8F0B10020B0EBF0
:10E11000840F0CD0D7F80CC006EB0802A100002336
:10E120002E6810786244F05401339942F8D16C6043
:10E13000012C07DB2868043850F8241009B9013C89
:10E14000FADC6C600120BDE8F0810020BDE8F081C0
:10E150002DE9F04703AFD7F814A08146984614463E
:10E160000E46504611F06EFD504611F0DCFD05469E
:10E17000B5B128463146A64204D02246534610F097
:10E18000F7F802E052460DF0B1FB48B14846294687
:10E19000424600F00CF80446002C18BF012400E0B1
:10E1A0000024504611F095FD2046BDE8F0872DE98A
:10E1B000F04F03AF83B090460E46D8F81C9004464B
:10E1C000B9F1000F00F0C480B0684FEA490B8345F5
:10E1D00006DD30465946F7F7C1FF002800F0BC8045
:10E1E0000294D8F82400F1684840F060D6E9005164
:10E1F0005945D8F818A008DA4FEAC90205EB8100A2
:10E20000A2EB8102002115F0B2EA00240196C6F8C3
:10E2100004B0B9F1010F20DBD8F840804E462868E1
:10E2200051464A4600FB08F328460DF0D1FC55F84C
:10E2300029102044421845F829208A424FF0000155
:10E2400005F1040598BF0121002818BF0120013EF7
:10E2500040EA040000EA0104E1D1029DA86881457A
:10E2600005DD28464946F7F779FF002874D0C5F840
:10E270000490524601994B46C868E8600E68D5F88C
:10E2800000B006EB8908584641460DF055FE201AAD
:10E290004FF0000A08EA00012BEA000040EA010EF4
:10E2A000B9F1050F26DBA9F1040C00960023002626
:10E2B0000EEB030408EB0301D4E9012004365EF8F9
:10E2C0000350664548F803A0E468C1F804A04BF881
:10E2D00003500BEB030503F11003C1F808A06A60BB
:10E2E000C1F80CA0C5E90204E2DBA9F10101009E1E
:10E2F00021F0030ACA4512DA0AEB0901A9EB0A0266
:10E300000BEB8A030EEB8A0006EB8101002650F826
:10E31000045B013A43F8045B41F8046BF7D1019EBA
:10E32000029B7068012807DB3168043951F820200E
:10E330000AB90138FADC7060586801280ADB1968EC
:10E34000043951F820200AB90138FADC586001E09C
:10E3500000206060012000E0002003B0BDE8F08FE5
:10E360002DE9F04303AF81B01C468146204690461C
:10E370000D4611F067FC204611F0D5FC06465EB153
:10E3800030462946F7F703FF30B14846314642464A
:10E39000FFF70DFF054600E00025204611F099FC2F
:10E3A000284601B0BDE8F083B0B502AF46F6830160
:10E3B0004C20C0F2020100220025F7F74FFC044672
:10E3C0002CB1204600F005F801202546A06428461F
:10E3D000B0BDB0B502AF0446201D00252560F7F79B
:10E3E00019FE04F11800F7F715FE04F12C00F7F7F9
:10E3F00011FEC4E91055A564B0BDD0B502AF044606
:10E400007CB1201DF7F7EBFD04F11800F7F7E7FDED
:10E4100004F12C00F7F7E3FD94F8480010F0010F29
:10E4200000D1D0BD2046BDE8D040F7F7F6BC2DE9BD
:10E43000F04F03AF89B01446824620460D4611F0D6
:10E4400001FC204611F06FFC8346BBF1000F78D031
:10E450000AF1180829464046F7F799FE00260028D9
:10E4600070D004A80AF10409CAF82460F7F7D2FDB5
:10E4700002A804900220CDE906062846F7F77CFDA5
:10E480001F30C11700EBD160002120F01F00CAF837
:10E4900000004846F7F7C2FE48462021F7F7A8FFDC
:10E4A00000284ED02868002104AA23460068029064
:10E4B0000391002818BF0120494605905846FEF7F1
:10E4C00022FCF0B358465946202210F0A1FBC0B3FD
:10E4D000DBF8040020B1584601210CF0C1FD04E036
:10E4E00058464FF0FF31F7F799FE50B304AB58464A
:10E4F00000215A4600940FF0EDF810B3DBF8040049
:10E500000026002101284FF00000A4BFDBF8000026
:10E510000068CAE910064846F7F780FEDAF80000FE
:10E5200041004846F7F764FF60B1002049464A467B
:10E53000434600940FF0CEF80646002E18BF012681
:10E5400000E00026204611F0C4FB304609B0BDE8CB
:10E55000F08FB0B502AF0D460446AC421AD0201D74
:10E56000291DF7F714FEA0B104F1180005F11801F8
:10E57000F7F70DFE68B104F12C0005F12C01F7F757
:10E5800006FE30B128682060286C2064686C6064E6
:10E5900000E000242046B0BD2DE9F04103AF044661
:10E5A0009846256816467DB9FFF7FEFE05462DB153
:10E5B000284631464246FFF73AFF08B1256003E09E
:10E5C0002846FFF71AFF25682846BDE8F0812DE9A7
:10E5D000F04303AF81B08946804650681646D9F8AB
:10E5E00004108142BCBF4E469146D8F80800D9F8C5
:10E5F0000410814203DD4046F7F7B0FDB0B3706808
:10E60000012811DBD8F8001000203268D9F800305A
:10E6100053F8204052F82050654041F82050013016
:10E620007568A842F4DB00E00020D9F804108842A5
:10E630000CDAD8F80020D9F8003053F8201042F84E
:10E6400020100130D9F804108842F6DBC8F8041015
:10E65000012909DBD8F80000043850F821200AB954
:10E660000139FADCC8F80410012000E0002001B0F4
:10E67000BDE8F0832DE9F04F03AF81B09346054626
:10E68000DBF800000E4600B37168AE4222D0A868E5
:10E69000814206DD2846F7F761FD002800F0D980A9
:10E6A000716801290ADB28680023326852F82310B8
:10E6B00040F82310013371688B42F7DB284640F89D
:10E6C000041F0090DBF8000006E028460021F7F761
:10E6D000A5FDBAE02A1D0092C2174B1E00EBD260C6
:10E6E00029684FEA601EB3EB601F53DD4FF000084E
:10E6F00051F8230000284AD0A3EB0E0AAAF1010921
:10E7000041F82380DBE900252DB30826551BEA17C5
:10E7100005EBD264A3EB641224F01F042D1B51F807
:10E7200022C020FA05F484EA0C0441F822401FBFFD
:10E73000C5F1200500FA05F501EB820252F8044C00
:10E740001CBF654042F8045C5BF806500436DBF8F9
:10E750000020002DDAD1D51751F82A6002EBD565DB
:10E7600025F01F05521B20FA02F586EA050641F83E
:10E770002A601FBF51F82960C2F12002904070400A
:10E7800018BF41F8290051F823000028B8D1013BF7
:10E790007345ADDC73454DD1DBF8000051F82E30E8
:10E7A000C21700EBD26222F01F02851A23FA05F28B
:10E7B000002A3FD00BF1080CC5F12006002D03FA0A
:10E7C00006F318BF23FA06F541F82E500B685340A4
:10E7D0000B60DBF804506346F5B1EE1705EBD66429
:10E7E000661124F01F042D1B51F8260002FA05F4CF
:10E7F00080EA040041F826001EBFC5F1200022FA7D
:10E8000000F5002D04D001EB860044686C404460A4
:10E8100053F8045B002DE0D1DBF8002051F82E30D6
:10E82000D61702EBD66626F01F06951B23FA05F2D3
:10E83000002AC1D1009B1868012806DB043951F871
:10E8400020200AB90138FADC1860012001B0BDE8C7
:10E85000F08F0020FAE7B0B502AF88B00C4602A9ED
:10E8600005461046062200F015F840B1072806DAE2
:10E8700002AA28462146FFF7FDFE044607E00024D1
:10E88000032083216A2200230094F7F731FB2046FE
:10E8900008B0B0BD8446DCF8043093B32DE9F041F4
:10E8A00000204FF0FF3E0EEB43173C46012B1EDBD2
:10E8B000DCF80050013BA4F1200755F82360002E3E
:10E8C000F3D04FF01F084FF0004705E055F82360E4
:10E8D000013C7F08A8F101083E4204D09042B8BF35
:10E8E00041F820400130B8F1010FEFDADBE7904248
:10E8F000BDE8F041BEBF4FF0FF3241F820200130AB
:10E900007047002070472DE9F04F03AF91B0D7F862
:10E9100018A0994614468846A04500F0B38002909E
:10E92000504611F08FF9504611F0FDF90546002DC3
:10E9300000F0AF806068D8F804100844061DA8688D
:10E94000864206DD28463146F7F708FC002800F02D
:10E95000A080CDF80490012E6E6004DB2868B20020
:10E96000002114F004EF6068012874DB0BAE4FF057
:10E97000000C311D069106F10801059106F10C010C
:10E9800004910394216851F82C200A924CF0010262
:10E99000824214BF51F8221000210991D8F80410C6
:10E9A000012954DBDDE909200024E346CDF820C02D
:10E9B00050400790D8F8000044F001028A4250F815
:10E9C000249014BF50F822A04FF0000ADDE90401A2
:10E9D000099B524600F0D3FA069831460A9B4A46F4
:10E9E00000F0CDFA079B8AEA090210A80FA900F0EF
:10E9F000C6FA0CAB10980ECB4840DDF820C058404A
:10EA000050400D9081EA02000B990F9A4840504007
:10EA10000C902A6804EB0C0052F82030594042F860
:10EA2000201002EB8B00012156F8212050F82130F4
:10EA30005A4040F8212001310429F5D1D8F80410BA
:10EA400002340BF1020B8C42B4DB039C60680CF1C6
:10EA5000020C844596DBBE696868019AB2460128BB
:10EA600007DB2968043951F820300BB90138FADC8A
:10EA7000686002982946FFF7FDFD0446002C18BF88
:10EA8000012407E041464A46534600F00AF804468E
:10EA900003E00024504611F01CF9204611B0BDE8F7
:10EAA000F08F2DE9F04F03AF81B09A468146504672
:10EAB00014468B4611F0C6F8504611F034F98046E2
:10EAC000B8F1000F67D0DBF80400D8F80820410047
:10EAD000914206DD4046F7F741FB00286AD0DBF89B
:10EAE0000400002859DDD8F8001048F66C63DBF804
:10EAF0000020A64601EBC001C0F203030439043A2A
:10EB00004FF03C0C52F82060C6F30364350F53F805
:10EB1000255053F82440240444EA0565C6F3035401
:10EB2000C6F3034653F8244053F8266045EA04250B
:10EB30002E430E6052F820600138C6F30335C6F349
:10EB4000032453F8244053F825504FEA044444EA80
:10EB500005650CEA960406F00F061C5953F826606A
:10EB600045EA042546EA050641F8046CA1F10801CE
:10EB7000C8DCDBF80410744601294FEA4100C8F8EC
:10EB800004000DDBD8F80010043951F820202AB910
:10EB90000138FADC02E0002510E04000C8F804006B
:10EBA000484641462246FFF765FD0546002D18BF41
:10EBB000012500E00025504611F08BF8284601B0F1
:10EBC000BDE8F08F2DE9F04F03AF81B01C468246BF
:10EBD000204690468946F7F7CFF9461C46F6830152
:10EBE000C0F202010022B0000025F7F737F8834693
:10EBF000BBF1000F1DD0204659463246FFF74AFEB2
:10EC000005465DB1B54209DCB869494600905046F9
:10EC100042465B46FFF777FE054607E00020852168
:10EC2000009003206A220023F7F762F95846F7F7AD
:10EC3000F4F8284601B0BDE8F08F2DE9F04F03AF9E
:10EC40008FB01D46804628460D920C4610F0FAFF04
:10EC5000284611F068F80646002E00F093802846FA
:10EC600011F061F8002800F08D800890284611F01E
:10EC70005AF8002800F086808246284611F053F8A2
:10EC8000079000287ED021460D9CD146484622465A
:10EC9000FFF7E1FD002875D0D9F80400002871D0F5
:10ECA000DDF81CB021465846F7F771FA002869D004
:10ECB000D1464846F7F760F90E905846F7F75CF9E9
:10ECC0000990CC46D4F80490DCF80800814504DDB6
:10ECD00060464946F7F742FAD446DCE900B1894577
:10ECE000DDF838E00ADD0BEB8100A9EB01018A00B9
:10ECF000002114F03CEDDDF838E0D446CDE9018583
:10ED00004D46CCF80490B068814506DD3046294672
:10ED1000F7F724FADDF838E0D446D6F80090012061
:10ED2000022DC9F800000BDB6FF0030000EB850239
:10ED300009F10400002114F01AEDDDF838E0D446A2
:10ED400003967560089881688D4206DD2946F7F7BD
:10ED500005FADDF838E0D44608980668012D08DB8E
:10ED6000AA003046002114F002EDDDF838E0D44668
:10ED700008980596691E45600E9107990C950A68DA
:10ED800004920FE00024284610F0A3FF20460FB0A5
:10ED9000BDE8F08F60466546F7F7EEF88646AC466C
:10EDA000414650460890BEF1000FCDE906C150D053
:10EDB0000C9D0BF104000B9009F104000A90DBF8A4
:10EDC00000A01AF0010F48D12168022DD9F8006087
:10EDD00006F001030A68C3F1000302EA030282EAB3
:10EDE000060C27DB0E1DDDE90A21DDF838800D68F1
:10EDF000B8F101084FEAC57444EA5A0441F8044CDA
:10EE000056F8044B01F104011068AA4604EA030411
:10EE100084EA00044FEAC47040EA5C0042F8040C43
:10EE200002F10402A446E2D10E99AA46A446DDE905
:10EE30000C5400E000214FEA5A00BEF1010E4BF8DD
:10EE400021004FEA5C0049F82100B8D14FF0000ED4
:10EE500006E04FF0000E0C9D02E0BEF1200F03DC37
:10EE6000DBF80000012847D0099EB64512DADDF82C
:10EE70000CA0DDF81880DAF80000D8F80010CDF802
:10EE800024E0B646DDE904B9CDE90410DDE907C0A8
:10EE9000039003E0DDF820A0DDE906C8012D14DBB6
:10EEA0000C984946059A5B46049E56F8045B013867
:10EEB0001C6885EA040543F8045B52F8045B0C689F
:10EEC00085EA040541F8045BEFD1099841460D9CA1
:10EED000864550467FF466AFDCF804000128FFF653
:10EEE00059AFDCF80010043951F820200AB9013874
:10EEF000FADCCCF804004DE703994B68DDE9010525
:10EF0000012B07DB0A68161F56F823200AB9013BBC
:10EF1000FADC4B60F7F73BF90446002C18BF0124DC
:10EF200031E72DE9F04703AF82B0D7F814A081464E
:10EF30001D4614468846504610F084FE504610F098
:10EF4000F2FE06469EB1304621462A465346FFF75A
:10EF500074FE60B14846414632462B46CDF800A0CB
:10EF6000FFF730FE0546002D18BF012500E0002503
:10EF7000504610F0AEFE284602B0BDE8F0872DE9FD
:10EF8000F04F8CB00025CDE90201049522F04045F8
:10EF9000940005954FEA450E85EA450CCDF818E03A
:10EFA000CDF81CC0089485EA82048EEA8205099493
:10EFB0000A958CEA82050B951C2505EA53050DF18F
:10EFC000100E5EF805000190C3F382155EF825105F
:10EFD0000091C3F342268C0E990F5EF826A0C3F36E
:10EFE000023784EA50745EF827B0C3F3C23584EA6E
:10EFF000DA545EF825C0C3F3824684EA1B545EF8F7
:10F000002660C3F3425784EA5C445EF82770C3F37A
:10F01000026584EA96345EF82550C3F3C26884EA38
:10F02000D7245EF8288003F007005EF8211084EAF8
:10F03000152484EA58145EF8200084EA9109019CA2
:10F0400080EAC400009C80EA841080EA4A2080EABA
:10F050000B3080EACC3080EA864080EA4750970F38
:10F0600080EA056080EAC86080EA817E012010EABB
:10F07000927F1CBF89EA93098EEA837E17F0020F04
:10F080001CBF89EA53098EEAC37E0298C0F800903B
:10F090000398C0F800E00CB0BDE8F08F4CF22830C7
:10F0A000C0F2030070472DE9F04F03AF8FB08146E7
:10F0B00008A84FF0000B15468846CDE90DBBF6F7C2
:10F0C000A9FF03A8F6F7A6FFE86800287CD0286906
:10F0D000002876D06869002873D0F6F79FFF0646AF
:10F0E000002E00F0938010F066FD82460024BAF1F5
:10F0F000000F00F0938000202A6A0190002A1CBFB4
:10F10000696A00290BD1E86B0EAA0DAB51468468E1
:10F110002846A047002400287BD0002004E00120DE
:10F120000E922C620D916C6202902869F6F724FF12
:10F130000730C11700EB5170B8EBE00F08DD28690C
:10F14000F6F71AFF0730C11700EB51704FEAE008DD
:10F1500008AA48464146F7F779F8002859D02B69A4
:10F1600003A8E9690D9ACDF800A00CF098F90028E1
:10F170004FD003A908AA30460FF0F8F9002848D06C
:10F1800029693046F7F7FAF8012805DB2A69304685
:10F1900031460FF024FBE0B32B6930460E9A31461E
:10F1A000CDF800A00CF07BF998B3F9F7BDFB90B354
:10F1B0000D9A516809B1716891BB029900299BD0E1
:10F1C00030E00024652201E06522002400260A20A8
:10F1D00070210023CDF800B0F6F78AFE0D98F6F7FF
:10F1E000FEFE3046F6F7FBFE14B1204610F002FD9D
:10F1F00008A8F6F7D0FE03A8F6F7CDFE0E9808B1E2
:10F20000F6F7C9FE58460FB0BDE8F08F0024032280
:10F21000DCE7019830B903225446D8E70322D6E749
:10F22000C0E9002683465446DEE72DE9F04F03AFE0
:10F230008FB006469A46F06893460C4600285ED08A
:10F24000306900285BD07069002858D00AA8F6F70A
:10F25000E1FE05A8F6F7DEFEA0462CB910F0ABFCE7
:10F260008046B8F1000F53D0F6F7D8FE8146B9F1C9
:10F27000000F4FD00AAD316928460FF0B4FB0028CB
:10F2800000F08A800B980028F5D0B06A10F0020FC9
:10F2900002BF0E9941F004010E9110F0010F09D048
:10F2A000F26806F12C0008214346FFF775F90028A3
:10F2B00072D0B06A10F0020F35D105A80AA9F6F78E
:10F2C00066FF002868D005A8326901460FF04EF9A4
:10F2D000002861D005AD2846F6F74EFE049030694F
:10F2E000F6F74AFE0499AC4681421EDC05AD326950
:10F2F000284629460FF03AF9AC46B0B94CE0002553
:10F300000A206B21652200230095F6F7F1FD58E0F5
:10F310004FF0000800250A206B21032200230095EE
:10F32000F6F7E6FD43E00DF1280CF16BF368726926
:10F330004D69F06A3DB1CDE900384946029030464A
:10F340006346A84706E0CDE900801146484662467C
:10F35000FEF7BEF900B33369002049464A46CDF8AE
:10F3600000800EF0B7F9B8B132690AA9002043460F
:10F37000FDF7C9FC05467DB1DBF8000008B1F6F7E2
:10F380000AFECBF80050DAF8000008B1F6F703FEE9
:10F39000CAF8009001250AE000250A206B2103220B
:10F3A00000230095F6F7A4FD4846F6F7F4FD14B9DE
:10F3B000404610F01FFC0AA8F6F7EDFD05A8F6F789
:10F3C000EAFD28460FB0BDE8F08F2DE9F04F03AFFE
:10F3D00095B01E460546F06891468A46E0B1306910
:10F3E000D0B17169C1B1F6F7C7FD8346BBF1A00F7B
:10F3F00005D0BBF1E00F18BFBBF5807F1AD1F068D4
:10F40000F6F7BAFD42F21171884219DB0020712132
:10F4100000900A20672204E00020712100900A2059
:10F4200065220023F6F764FD4FF0FF34204615B047
:10F43000BDE8F08F0020712100900A206622F0E7DD
:10F4400010A8F6F7E7FD0BA8F6F7E4FD06A8F6F717
:10F45000E1FD10F0B0FB8046B8F1000F16D0D9F8EE
:10F46000000000220024416819B3C16861B9316904
:10F47000F6F768FFB0F1FF3F19DCD9F8040000226D
:10F48000416809B1C16861B1002412E00020712116
:10F4900000900A2003220023F6F72AFD4FF0FF34E4
:10F4A00011E03169F6F74EFFB0F1FF3F15DD0024A2
:10F4B000002200920A20712103220023F6F718FD92
:10F4C000404610F097FB10A8F6F789FD0BA8F6F759
:10F4D00086FD06A8F6F783FDA8E732690BA8D9F8E0
:10F4E00004104346FDF70FFC00285DD04FEAEB0007
:10F4F0005045B8BF4FEAEB0A10AA28465146F6F726
:10F50000A5FE002850D0336910A80BAACDF80080C2
:10F5100001460BF0C4FF002846D00BAC3369D9F884
:10F52000001020462246CDF800800BF0B8FFD8B37B
:10F5300096F8280010F0010F01D1002007E0F268D2
:10F5400006F12C0008214346FFF726F860B3F16866
:10F55000D6E90523F56B2D694DB1CDE9003410AB2B
:10F56000CDE9021806A904903046A84709E010AD7D
:10F57000CDE90041CDE9028006A811462A4612F0E5
:10F58000F0FF88B1336910A906AA0020CDF80080E9
:10F590000EF0A0F840B1D9F8001010A8F6F7D2FE8E
:10F5A00028B10024009485E74FF0FF3480E7012460
:10F5B00086E7816A41F00101816201207047C06ADB
:10F5C00028B180B56F46FEF718FFBDE880400120E6
:10F5D00070472DE9F04303AF87B00546E86BC16A79
:10F5E00021B1284607B0BDE8F043084710F0E3FA20
:10F5F0008146B9F1000F42D0EE691EB9F6F70EFD53
:10F600000646F6B3296930460FF0EDF900283FD0E1
:10F6100070680028F6D0D5F81880B8F1000F05D131
:10F62000F6F7FCFC8046B8F1000F31D095F82800C1
:10F63000344610F0020F15D102AC2046F6F7EAFC72
:10F640003068029070680390B0680490F06805908C
:10F650003069069920F0070001F00101084340F0ED
:10F6600006000690EB68404669692246CDF8009096
:10F67000FDF780FE38B1C5E90686012409E00024C3
:10F680000FE000240AE0A86910B94046F6F7A7FC8D
:10F690000024E86910B93046F6F7A1FC484610F09E
:10F6A000A9FA204607B0BDE8F083416C49680847D5
:10F6B000536C9B6818474CF25830C0F203007047F7
:10F6C0002DE9F04F03AF89B0064610F074FA814679
:10F6D0004FF0000800240025B9F1000F78D0B5697B
:10F6E00015B14FF0000B06E0F6F798FC0546002D2B
:10F6F0006AD04FF0010B746924B9F6F78FFC044609
:10F70000002C64D0307F10F0010F02D14FF0000ABE
:10F710000AE0B26806F120001A214B46FEF73CFFD2
:10F720008246BAF1000F53D0BBF1000F1FD0716AAF
:10F7300069B9316919B9B068F6F71EFC411E28464F
:10F74000002200230FF08FF888B941E0716A284643
:10F750000FF049F9E0B368680028F7D0012806D116
:10F7600028680068012804BFE8680028EED0307FD0
:10F77000AB4610F0020F16D10DF1100B5846F6F7FC
:10F7800049FC2868049068680590A8680690E868B5
:10F7900007902869089920F0070001F0010108434B
:10F7A00040F006000890D6E902025B46716CD1F881
:10F7B0000CC021468DE801063046E04740B1C6E95D
:10F7C00005454FF001080BE00024002500E000246F
:10F7D0000520672103220023CDF80080F6F788FB7F
:10F7E00024B1706910B92046F6F7F9FB25B1B0696C
:10F7F00010B92846F6F7F3FB484610F0FBF94046EF
:10F8000009B0BDE8F08F2DE9F04703AF84B015468D
:10F810008046A8680E46F6F7AFFB42F211718842A7
:10F8200008DB002066210090052067220023F6F700
:10F830005FFB13E010F0BFF904467CB1204610F0E6
:10F8400001FA204610F06FFA8146A86948B1287F76
:10F8500010F0010F0BD14FF0000A1CE04FF0FF3504
:10F8600049E00020662100900520642238E0AA6863
:10F8700005F120001A212346FEF78EFE8246287FDE
:10F8800010F0020F01BFA869016941F00401016194
:10F89000BAF1000F27D003AA2846314600F004F938
:10F8A00098B1039888B9696C3246A868AB69D1F8F9
:10F8B0000CC049468DE811042846E04758B1484637
:10F8C0004146F6F71BFD05460FE00020662100903B
:10F8D0000520662204E00020662100900520032216
:10F8E0000023F6F705FB4FF0FF35204610F0F1F945
:10F8F000204610F07FF9284604B0BDE8F087B0B587
:10F9000002AF82B05568D7F810E0D7E902C4012DE4
:10F9100003D1007F10F0020F09D1084611461A46A4
:10F920006346CDE9004EFDF7D3FE02B0B0BD1068CE
:10F9300002680846CDE9004E11461A466346FDF7B7
:10F9400050FD02B0B0BDC16941F00101C1610120AB
:10F950007047006A28B180B56F46FEF74EFDBDE8DE
:10F960008040012070472DE9F04F03AF83B005467A
:10F970009946686C16460C46D0F820C0BCF1000FC2
:10F9800007D02846214632464B4603B0BDE8F04F2B
:10F99000604710F010F98046B8F1000F35D04046AE
:10F9A00010F050F9404610F0BEF98246404610F083
:10F9B000BAF98346BAF1000F18BFBBF1000F15D09A
:10F9C000A86818B9F6F72AFBA86078B1E86818B9F2
:10F9D000F6F724FBE86048B1012E22DC00206A2102
:10F9E0000090052065220023F6F782FA0024052006
:10F9F0006A21032200230094F6F77AFA404610F0B9
:10FA000068F9404610F0F6F807E0002405206A2166
:10FA1000032200230094F6F76BFA204603B0BDE8FA
:10FA2000F08F5046052E0ED0022E19D11821F6F770
:10FA3000F5FB0028DAD058460B21F6F7EFFB00283B
:10FA4000D4D0022617E00A21F6F7E8FB0028CDD033
:10FA500058460321F6F7E2FB0028C7D005260AE046
:10FA60000221F6F7DBFB0028C0D058460121F6F74B
:10FA7000D5FB0028BAD0A868214601225346CDE91B
:10FA800000B912F01CFA0028B0D048460321002229
:10FA900012F0F6F90028A9D0E8683146F6F7BEFB67
:10FAA0000028A3D00124A9E72DE9F04303AF81B0DA
:10FAB00014460026894680462660F6F7AFFA0546CA
:10FAC00025B328460121F6F7A9FB48462946F6F753
:10FAD00055FC002803DC206840F001002060D8F8C5
:10FAE00008102846F6F753FB284601210BF0B8FA18
:10FAF00048462946F6F742FC002803DB206840F020
:10FB0000020020602846F6F76AFA0126304601B066
:10FB1000BDE8F0832DE9F04F03AFB5B081466FF03B
:10FB2000130000EBD2000C464FF0000813930C2892
:10FB300000F27882012101FA00F041F2011108423D
:10FB400000F07082D7E906854FEAD20A139810B9FF
:10FB5000F6F736FE13900020AA4588BF0120002D3D
:10FB6000294618BF0121AA4538BF5546B4F5007F84
:10FB700038BF4FF40074B8F1000F06D0084004D12C
:10FB80002CA841462A4613F0E0EC10F014F8064683
:10FB9000002E00F09281FEF707FC002800F0908113
:10FBA000109004F13F0020F03F0B304610F04AF86F
:10FBB000304610F0B8F80E90304610F0B4F80990C6
:10FBC000304610F0B0F80F90304610F0ACF81190BD
:10FBD000304610F0A8F80B90304610F0A4F80A90C8
:10FBE000304610F0A0F880463046129610F09BF890
:10FBF0000646F6F794F9ABF1010401463046224679
:10FC00000FF006F8002800F0FE814CF6CD40CDE95B
:10FC10000786CCF6CC40AAF10106A4FB00010DF149
:10FC2000700BCDF814904FF000090694C8090C90A1
:10FC30004FEACA000D9035E115B100252CAC08E063
:10FC40002CAC51462046F7F756FF0028C0F2DB8166
:10FC5000012558462146524613F076EC14A8214659
:10FC6000524613F072EC5046BAF1000F0CD00BEB79
:10FC7000000111F8012C013201F8012C12F0FF0FE4
:10FC800002D101380128F2DA4FF00008139824AAB3
:10FC9000CDE90008204651460023F6F715FF00285D
:10FCA00000F0B381139814AACDE9000858465146D4
:10FCB0000023F6F709FF002800F0A781BAF1000F32
:10FCC0000BD014A824A9524610F8013B013A0C7835
:10FCD00083EA040301F8013BF6D19DF8900040F05F
:10FCE00080008DF8900024A8815D41F001018155CC
:10FCF0005146119C2246F6F7A9FA002800F08381AC
:10FD0000129A3221F86A2B460090204609F1010927
:10FD100012F095FA002806DC4FF000054FF00008BD
:10FD200000F0C08071E1F86A022100224FF0000863
:10FD300012F0A6F8002800F06881F86A032100227A
:10FD40004FF0000812F09CF8002800F05E810020BF
:10FD50000396049048B1F86A0021049A4FF0000815
:10FD600012F08EF8002800F050810F980021002535
:10FD7000F6F754FA2C46504601280ADB411E584437
:10FD800010F8012C013200F8012C084612F0FF0F88
:10FD9000F2D04FF00008139824AACDE90008584685
:10FDA00051460023F6F790FE002800F02E810E9DAC
:10FDB00024A851462A46F6F749FA002800F0238184
:10FDC0000D98294600FB04F228460EF021FF00287A
:10FDD00000F019810F9E2A46304631460EF0C6FBD0
:10FDE000002800F01081651C0C988442C2DB069943
:10FDF0003046F6F743FB002800F005810B9D3146A5
:10FE00002846F6F7C4F9002800F0FD80089A284635
:10FE100029460EF0ABFB002800F0F5800E9C1199EE
:10FE200020460EF074FE002800F0ED800A992A4664
:10FE300012982346009000204FF000080DF04AFC75
:10FE4000039E002800F0E180F6F769F80E9D024657
:10FE50000A9928460EF0C3FC002800F0D480079CC5
:10FE60002A460B9920460EF0BAFC002800F0CB8001
:10FE700008992046F6F782FA00280BDBF86A32214F
:10FE8000009001230798129A12F0D9F900281BDC80
:10FE900040F0B980049A002540F6FE71501C8A4259
:10FEA0007FF757AFF86A00214A464FF0000811F07B
:10FEB000E7FF00287FF4C0AEA7E04FF00008B1E0F4
:10FEC0004FF000080024A3E0F86A0221012211F09B
:10FED000D7FF002800F09780F6F721F80246DDE909
:10FEE00007100EF07CFC002800F08D801298002195
:10FEF00000904FF000080E98089A119B0DF0EAFB55
:10FF0000002800F0828008980221F6F787F900287F
:10FF100079D010980799129AFEF789FA002872D0C2
:10FF2000129800901098019009980E9ADDE9073117
:10FF3000FDF7CEFB002866D002244FF00008099997
:10FF4000486801281DD108680068012804BFC868F6
:10FF5000002816D1F5F7E3FF0246089801460EF097
:10FF600005FB00284FD01298009010980190099836
:10FF70000E9ADDE90731FDF7ABFB01340028DED135
:10FF800043E0F86A0321012211F07AFF8146B9F1BA
:10FF9000000F18BF4FF0010935D00598C06808B1AF
:10FFA000F6F71DF80598006908B1F6F718F80598F6
:10FFB000406908B1F6F713F80798F6F7BCF8059D05
:10FFC000E8601198F6F7B7F828610998F6F7B3F8E2
:10FFD0006861E968B9B14FF00008B0B105980069EF
:10FFE00098B1786A10B1786A04990160B86A08B16A
:10FFF000B86A0460386A20B1386A2CA9524613F0F6
:020000021000EC
:10000000A4EAC84601E04FF00008129E109C2EB1F1
:1000100030460FF05EFE30460FF0ECFD14B1204686
:10002000FEF7EBF9404635B0BDE8F08F2DE9F04F13
:1000300003AF85B03C6A9B4692460D46804600263B
:100040004FF0000934B90FF0B6FD0446002CA1466C
:1000500000F09480D7E90621BBF1010F504688BF1C
:100060000126BAF1000F18BF0120BBF1020F0BD817
:10007000304009D1BBF1000F11D140461646FAF7C6
:1000800092FAF969324650B1CDE90021404629463D
:1000900052465B460294FAF791FA044683E04046E2
:1000A0000395F9F7EFFE0546002D72D04046F9F7AB
:1000B000E9FE0146002969D040460E46FAF783F86A
:1000C00000285DD0BAF1000F20D0D8F804304046A7
:1000D00029465246009400F070F8002850D0DAF813
:1000E0000C0040B1D8F8000029462246036E404675
:1000F0009847002844D0D8F8000031460A462B46DD
:10010000D0F858C040460094E047C8B3049535463F
:10011000BBF1000F29D00026B869D7F81CA00499BC
:1001200050F8263040465AF82620009400F045F852
:1001300088B35AF82600DDF810A0C06838B1D8F8A6
:10014000000051462246036E4046984718B3D8F83F
:10015000000029462A465346D0F858C0404600942D
:10016000E047C0B101365E45D6D303982946F9F77A
:10017000C0FE0446002C18BF01240DE0002418E046
:100180002846F9F744FD0024354609E02846F9F7EA
:100190003EFD002407E000240498F9F738FD15B16E
:1001A0002846F9F734FDB9F1000F1CBF48460FF09F
:1001B00021FD204605B0BDE8F08F2DE9F04F03AFDB
:1001C0008BB098460D4692460646454517D0BAF183
:1001D000000F0DD0B8F1000F1CBFDAF804000028A2
:1001E00006D0B86941460A903046FAF726F990B130
:1001F000304629460BB0BDE8F04FF9F7E4BF0025C3
:100200001020D021702200230095F5F771FE2846BA
:100210000BB0BDE8F08FD8F84000002865D00A9CEC
:1002200020460FF00FFD20460FF07DFD834620464F
:100230000FF079FD0446002C00F0CB8108F1040991
:1002400006F15C0258464946FEF714FA002800F011
:10025000C08120460121F5F7E1FF002800F0B981B7
:1002600009945A46306805F1180B5946D0F888C0F1
:10027000304608920A9C2346E047002800F0A981F6
:10028000CDF8189005F1040930685A4649462346CE
:10029000D0F888C03046CDF81CB0E047002800F008
:1002A000988106F1880248464946FEF790F90028F1
:1002B00000F08F81CDF814904FF00043DAE900018F
:1002C0004C1E50F824204FEA530B13425B46FAD0E1
:1002D000BBF1000F08BF8C1E079B002C43DBBBF15A
:1002E000000F08BF4FF0004B06E000258FE7DAF85B
:1002F0000000013C4FF0004B039450F824000490A0
:1003000004981BEA000F0AD0059C9946CDE90043EA
:100310000A98029030460699089A099B0AE0089CC0
:100320000094DDF82490CDF804900A9802903046AD
:10033000DDE9052100F05BF9002800F04A810A9B05
:10034000304621464A4600F0BCF9002800F04181C1
:10035000079B4FEA5B000021B1EB5B0F8346CFD1D7
:10036000039C012CC3DA09984068002800F0F08053
:10037000DDF814B008F11808E869002800F0FA80E8
:100380000A9C20460FF05EFC20460FF0CCFC814614
:1003900020460FF0C8FC049020460FF0C4FC8246B3
:1003A000BAF1000F00F0E08050460121CDF80C803A
:1003B000F5F734FF002800F0D78030684946D0F8C0
:1003C00084400A9800903046DDF82480079B42461E
:1003D000A047002800F0C880306841464246D0F867
:1003E00084400A9800903046069BA047002800F001
:1003F000BB80089A40464146FEF7E9F8002800F025
:10040000ED803068D0F884400A9800903046079913
:10041000069B0A46A047002800F0E0803068D0F82C
:1004200084400A9800903046DDE907210B46A0473A
:10043000002800F0D3800798059A0146FEF7C7F818
:10044000002800F0CB803068D0F884400A980090F3
:1004500030460799099B0A46A047002800F0BE8055
:1004600030680499069AD0F8884030460A9BA04725
:10047000002800F0B3800498039A0146FEF7A7F81D
:10048000002800F0AB8030684B46D0F884400A98D2
:100490000090304604990A46A047002800F09E804C
:1004A0000498079A0146FEF792F8002800F096801B
:1004B000306849460A46D0F884400A980090304691
:1004C000069BA047002800F08980306849465246C4
:1004D0000B46D0F88C400A9800903046A047002880
:1004E0007CD030684A46D0F884400A980090304664
:1004F00004990B46A047002870D030684B46D0F8CE
:1005000084400A98009030460599089AA047002830
:1005100064D00798DDE90512FEF759F800285DD090
:100520003068D0F884400A98009030460799049BC0
:100530000A46A047002851D00798039A0146FEF7C3
:1005400046F88046B8F1000F18BF4FF0020847E0A8
:10055000DDF814B000211C465846F5F75FFE204632
:100560000021F5F75BFE1CE04FF000080A980FF041
:10057000B0FB10E0069C58462146F5F708FE40B354
:10058000079821464246FEF722F88046B8F1000F50
:1005900018BF4FF00208B8F1000F1AD0B8F1010FE0
:1005A00005D130462946F9F70EFE40B911E005F1B4
:1005B0002C0001210126F5F731FE50B12E6458467A
:1005C0000021F5F782FF07980021F5F77EFF01254E
:1005D00000E000250A980FF07CFB18E64FF00008B9
:1005E000DDF814B0C2E7FAF7DEBCFAF7B5BE2DE9C4
:1005F000F04F03AF81B0D7F820B00546994690463A
:100600000C4658460FF01EFB58460FF08CFB8246F6
:1006100058460FF088FB0646002E4AD05046214629
:10062000F5F7B5FD002844D028684146FB694246ED
:10063000D0F884402846CDF800B0A047C8B3286859
:100640004946BB694A46D0F884402846CDF800B0F8
:10065000A04770B32868314642464B46D0F88440E4
:100660002846CDF800B0A04718B348464946424650
:10067000FDF7ADFFE8B1286849464A465B46D0F829
:1006800088402846A047A0B1286841464A465346BC
:10069000D0F884402846CDF800B0A04748B1404685
:1006A00041463246FDF793FF0546002D18BF012550
:1006B00000E0002558460FF00CFB284601B0BDE8CD
:1006C000F08F2DE9F04703AF82B01C460546204667
:1006D000914688460FF0B6FA20460FF024FB82467A
:1006E000BAF1000F42D02868414642462346D0F86E
:1006F00088602846B047C8B3286851464A46234612
:10070000D0F888602846B04780B3286849464246FA
:100710005346D0F8846028460094B04730B3286828
:10072000414642462346D0F888602846B047E8B1A3
:100730002868514652462346D0F888602846B0477C
:10074000A0B12A46514652F8880B5346D0F884602F
:1007500028460094B04748B1404641465246FDF70E
:1007600036FF0546002D18BF012500E00025204674
:100770000FF0AFFA284602B0BDE8F08748F6D46023
:10078000C0F203007047D1F8A820C0F8A8200FF0ED
:10079000D9BF2DE9F04703AF82B07C6998469146F6
:1007A0000E4682460CB1002505E00FF004FA04461F
:1007B000002C254634D020460FF044FA20460FF096
:1007C000B2FA30B30EF00AFB3146F5F7BBFD10B3B9
:1007D0000EF009FB3146F5F7B5FD18B30EF008FB36
:1007E0003146F5F7AFFD10B30EF007FB3146F5F7D4
:1007F000A9FD08B30EF006FB3146F5F7A3FD00B3E3
:1008000000261020CA21872200230096F5F770FBEE
:1008100025E0002623E04FF60F60C0F2010014E04F
:10082000002623E040F20F00C0F202000DE040F28B
:100830009F20C0F2020008E040F20B60C0F202000C
:1008400003E040F65320C0F20200CAF8A800504668
:1008500031464A46434600940FF095FF064620462F
:100860000FF037FA15B128460FF0C4F9304602B040
:10087000BDE8F0872DE9F04703AF82B08246994684
:1008800016460C46BAF1000F18BF002C08D03EB136
:10089000B9F1000F04D07D695DB14FF000080EE0A2
:1008A00000241020C821432200230094F5F720FBE8
:1008B00020E00FF080F90546002DA8461ED0204606
:1008C00031464A462B460DF053FD60B1DAF8A86078
:1008D0000AF14802204621462B46B0470446002C28
:1008E00018BF012400E00024B8F1000F1CBF4046EF
:1008F0000FF080F9204602B0BDE8F0870024F9E748
:100900002DE9F04303AF81B006461D4691460C46E3
:100910003EB134B1B9F1000F03D05DB14FF0000822
:100920000EE000241020C921862200230094F5F750
:10093000DFFA1FE00FF03FF90546002DA8461DD055
:10094000204649462A460AF0D1FF60B1D6F8A8C031
:1009500006F14802204621462B46E0470446002C7B
:1009600018BF012400E00024B8F1000F1CBF40466E
:100970000FF040F9204601B0BDE8F0830024F9E70C
:100980004CF27C30C0F2030070472DE9F04F03AF0A
:100990008DB0D7F81890834600241D460B920E4662
:1009A00048460C94F5F7E8FD80464846FAF7C7FE3E
:1009B00082464846FAF7D5FEB8F1000F18BFBAF1E3
:1009C000000F00F0C080002800F0BD800790F5F710
:1009D000EBFE0446002C00F0BB80606806900FF030
:1009E000EAF8089000284FF0000009904FF000004E
:1009F0000A9000F0BD80F5F711FB014600280A912E
:100A000000F0AF80F5F70AFB01460028099100F0DD
:100A1000AD80F5F703FB002800F0AA80CDE9045073
:100A200050460A9DDDF820A029465246F9F7D8FA2B
:100A3000002800F0CA802846F5F79EFA8246F000AA
:100A40005045C1BF0AF10700C11700EB5170C61035
:100A5000059D584631462A46F5F7F8FB002800F078
:100A6000C080F00050450ADD0AF00700C0F108021E
:100A7000059801460EF046F9002800F0BC80049A63
:100A800000210020002A08BF01210B9B002B08BF7A
:100A9000012008430390002A1046194618BF012080
:100AA000002B18BF012108400290DDE908A6039839
:100AB00001280DD1D8F80C000CAA514623468568B0
:100AC0004846A847002800F0C980DDF830B008E0AB
:100AD00020680499F5F75BFBDDF82CB0002800F0E6
:100AE000C38022683046CDF800A0DDF828A0079921
:100AF00053460AF0D4FC002800F08880069D314659
:100B0000059E5346284632460AF09DFC002800F018
:100B10008B8008982946009028465A4653460AF08A
:100B2000BEFC002800F08B806868002840F09180AF
:100B30000298DDE908A60128B9D1002065210090BE
:100B40002A206A2295E02A2065214322009404E0AD
:100B500000242A200094652141220023F5F7C8F9DA
:100B60002FE00020099000200A9001E00020099069
:100B70004FF000082A20652141220023CDF8008093
:100B8000F5F7B6F90A9DDDE908A62046F5F712FE4D
:100B90000024BAF1000F1CBF50460FF02BF8B8F13B
:100BA000000F1CBF4046F5F7F6F916B13046F5F7D1
:100BB000F2F915B12846F5F712FA0C9808B1F5F7D5
:100BC000EAF920460DB0BDE8F08F002065210090C5
:100BD0002A2010220023F5F78BF9DDF81480099EF6
:100BE000D3E70020652100902A2003220023F5F797
:100BF0007FF9A846C6E70020652100902A2003223D
:100C00000023F5F775F9DDF81480BBE700206521B6
:100C100000902A2003220023F5F76AF95546DDF8F3
:100C20001480DDF820A0B0E70020652100902A2084
:100C300003220023F5F75CF9B0465546A3E70020F0
:100C4000652100902A2003220023F5F751F9B046D0
:100C500098E7B0460A9DDDE908A69AE700206521DD
:100C600000902A202A2204E00020652100902A20FA
:100C700041220023F5F73CF9DDF814800A9D84E752
:100C80002DE9F04F03AF87B01D4614468946002872
:100C900000F0B380FAF753FD8246BAF1000F00F07E
:100CA000AC804846B9F1000F04D10EF084FF002853
:100CB00000F0C1800590F5F7B1F90646F5F7AEF9F9
:100CC0000690F5F7ABF98046F5F7A8F98346002EB4
:100CD00000F09C800698002800F09880B8F1000F82
:100CE00018BFBBF1000F00F091805046F9F7CAF829
:100CF0000490002800F09080059A50464146F9F78C
:100D00006FF9002800F09D80304641460DF06BFEE3
:100D1000002800F08A8070680028F5D030463146FF
:100D200042460DF023FC002800F093803046F5F792
:100D300023F903904046F5F71FF90399814207DC38
:100D40003046314642460DF011FC002800F081800B
:100D500000200499009032460598002301905046E7
:100D6000F9F703FC00286CD05046CDE9029BF9F757
:100D7000F6F8F9F7F6F8B0F5CB7F0BD1DDF814B043
:100D80005046CDF800B00023DDE903914A46F9F75B
:100D9000A1FA0AE0DDF814B05046CDF800B0002307
:100DA000DDE903914A46F9F7B7FA002876D04946BB
:100DB000DDF8189042465B4648460AF00CFB0028D6
:100DC00078D0D9F80400DDE9029B00289CD0059B6F
:100DD000304631464246FBF796FF002878D0286817
:100DE00008B1F5F7D8F8206808B1F5F7D4F80698F7
:100DF000286026600126049C36E000262A20672110
:100E0000432200960023F5F773F843E000242A20DC
:100E100067214122009404E000242A2000946721E5
:100E200010220023F5F764F814E0002067210090F9
:100E30002A2068220AE000262A2000966721412203
:100E4000E0E70020672100902A2010220023F5F718
:100E50004FF8049C069D16B13046F5F79CF815B185
:100E60002846F5F798F80026B9F1000F04BF059859
:100E70000EF0C0FEB8F1000F1CBF4046F5F7AFF80A
:100E800014B12046F8F7C3FEBBF1000F1CBF584653
:100E9000F5F781F8304607B0BDE8F08F00206721F4
:100EA00000902A2010220023F5F722F8CB46049C5C
:100EB000069D0AE00020672100902A2003220023DB
:100EC000F5F716F8DDE903B44D46DDF80890C2E702
:100ED0000020672100902A200322B7E72DE9F04F78
:100EE00003AF89B01D4693460C46064685B1284699
:100EF000FAF725FC8046B8F1000F09D02846FAF72A
:100F000042FC8146BBF1000F18BFB9F1000F0DD1B3
:100F10000020662100902A2067220023F4F7E8FFD2
:100F20004FF0FF34204609B0BDE8F08F0EF043FECD
:100F30008246BAF1000F41D050460EF083FE504673
:100F40000EF0F1FE054650460EF0EDFE06905046BE
:100F50000EF0E9FE089050460EF0E5FE0790504670
:100F60000EF0E1FE002800F09680049040462946ED
:100F700052460595F9F734F830B3DBF800004168C4
:100F800091B1C16881B90599F5F7DCF9B0F1FF3F7E
:100F90000ADCDBF80400416831B1C16821B9059968
:100FA000F5F7D0F9002815DB00242A2066216422F9
:100FB00000230094F4F79CFF002576E000206621D2
:100FC00000902A204122A8E7002500952A206621CA
:100FD000102265E0059D5346DBF8041008982A4668
:100FE000FBF791FE002856D02846F4F7C5FFE10034
:100FF0008142C1BFC21DD11702EB5171CC10079DB8
:10100000039030462A462146F5F720F9002842D0C1
:101010000399E000884208DD01F007002946C0F18D
:10102000080228460DF06EFEA8B32946089D059CCF
:1010300006982A46CDF800A023460AF030FA50B3AD
:10104000DBF8001028462A462346CDF800A00AF017
:1010500026FA00B34046F8F715FF054695B3089801
:101060002946CDE9000A4046069A4B46F9F77DFA33
:1010700070B34046F8F773FFF8F773FFB0F5CB7F16
:1010800029D1049A404629460023CDF800A0002427
:10109000F9F720F928E0002500952A20662103228F
:1010A0000023F4F725FF4FF0FF3450460EF011FEF9
:1010B00050460EF09FFD002D3FF434AF2846F8F760
:1010C000A6FD2FE700252A20009566214122E7E7AB
:1010D000002000907AE7049A404629460023CDF884
:1010E00000A00024F9F718F980B106985346DDE90D
:1010F00004120AF070F958B1DBF800100698F5F701
:1011000021F90024002808BF0124CEE700945DE700
:1011100000200090C1E7F0B503AF81B0044604F1B0
:1011200018000021582212F022EB49F6D8604DF247
:1011300007514DF6175245F6391340F6313C41F24E
:10114000115E48F6A77544F6A476CCF20510C3F2FA
:101150007C61C3F27002CFF20E73CFF6C07CC6F68C
:10116000580E84E80F50C6F2F945CBF6FA661C20FB
:10117000C4E90656E066012001B0F0BDF0B503AF4A
:1011800081B0044604F118000021582212F0EEEA62
:101190004EF267604AF685614FF272324FF23A536F
:1011A00045F27F2C46F68C0E4DF6AB154CF61956D3
:1011B000C6F60920CBF66731C3F66E42CAF24F532A
:1011C000C5F20E1CC9F6053E84E80F50C1F68375C2
:1011D000C5F6E0362020C4E90656E066012001B0DD
:1011E000F0BD2DE9F04303AF81B0144688460546B3
:1011F000002C48D0D5E90821012302EBC40090421D
:1012000028BF00230BB10131696201EB5471C5E9BC
:101210000801A96EC9B105F128060A197018224300
:10122000402A29D3C1F1400941464A4612F08CE9CF
:1012300028463146012200F0B0F830460021442211
:1012400012F094EAA4EB0904C8440020B0EB941F08
:1012500009D0A60928464146324600F09EF8A4EB84
:10126000861408EB861874B105F128004146224621
:10127000AC6612F06AE906E04146224612F064E9E3
:10128000A86E2044A866012001B0BDE8F0832DE9D6
:10129000F04103AF0C4604F12808A16E05468020FA
:1012A0004E1C08F80100392E0CD308EB0600C1F1E2
:1012B0003F020021002612F05AEA20464146012250
:1012C00000F06BF808EB0600C6F13802002112F0BE
:1012D0004EEA606A0122010E84F86010010C84F865
:1012E0006110010A84F8621084F86300206A010E1C
:1012F00084F86410010C84F86510010A84F8661003
:10130000414684F86700204600F047F84046002137
:10131000442212F02CEAE06E1C2812D0202821D1A1
:10132000002054F820100A0E0B0C05F8202005EBC5
:101330008002013053700B0A93700828D170F0D1ED
:1013400028E0002054F820100A0E0B0C05F820208D
:1013500005EB8002013053700B0A93700728D1709F
:10136000F0D117E002D90020BDE8F081042811D3A4
:10137000002054F820100A0E0B0C05F8202005EB75
:101380008002013053700B0A9370D170E16EB0EBA4
:10139000910FEED30120BDE8F0812DE9F04FA4B00C
:1013A0000090002A00F01C860098D0E9006AD0E97D
:1013B0000253D0E90494D0E906C79B4605EA0A0324
:1013C000139585EA0A0535402CEA09006B404FEA7F
:1013D000B60585EA7635019285EAB655A6462B44D0
:1013E00004EA090568404FEAB91585EAF92585EA56
:1013F00079657A194D7810440A788F78CDF844E0F1
:101400002D0445EA0262CC7842EA07220AEA060580
:1014100022431492104442F69872C4F28A22104475
:1014200003EB000808EA0A0408EA06036C4000EB34
:101430000B0563404FEAB80484EA783405EA0907EB
:1014400084EAB8544FEAB510E218109232462EEAF8
:10145000050412927C404F7980EAF5200E7980EAEB
:10146000756B8B7964443F04C87947EA06668E46FB
:1014700046EA0323184344F291431590204458440C
:10148000C7F237131844109B1E1886EA080406EAB0
:101490000803144063404FEAB60484EA763484EAD1
:1014A000B654E2181092139A9EF80BC0871829EAD6
:1014B000070407EA05034FEAB71083EA040B80EA42
:1014C000F7200C7A80EA7762487A8B7A11990004C7
:1014D00040EA046040EA032040EA0C001690084409
:1014E0004FF6CF315844CBF2C05110440844109904
:1014F00001EB000C8CEA06040CEA060304EA08047B
:1015000063404FEABC0484EA7C3484EABC54E118AA
:1015100000EB0A04139125EA04034FEAB4109EF885
:101520000CB080EAF4209EF80E2080EA746104EA90
:10153000070080EA030A9EF80D009EF80F300004B1
:1015400040EA0B6040EA02204DF6A532184317909E
:101550004844CEF6B512504408441399104401444F
:10156000139181EA0C0301EA0C0233405A404FEA1E
:10157000B10383EA713383EAB15399181191129937
:101580009EF810B008449EF8131027EA00024FEAB4
:10159000B01383EAF02383EA706900EA040383EA64
:1015A000020A9EF811209EF81230120442EA0B62E1
:1015B00042EA0322139B1143189129444CF25B2207
:1015C0005144C3F6561249441144119A02EB0109E1
:1015D00089EA030509EA030205EA0C056A404FEAB5
:1015E000B90585EA793585EAB9552A4401EB08053C
:1015F000129224EA05024FEAB5119EF814B081EA6E
:10160000F5219EF8173081EA756805EA000181EA44
:10161000020A9EF815109EF81620090441EA0B6193
:1016200041EA022141F2F112194319913944C5F6F8
:10163000F1125144139F41441144129A0E4402EB9B
:10164000010888EA090308EA09023B404FEAB6119B
:101650005A404FEAB80383EA783306EA050783EA7B
:10166000B85381EAF6211A4412929EF8192020EA12
:10167000060387EA030A9EF8187081EA766B9EF8E3
:101680001A1012049EF81B3042EA076242EA012156
:1016900048F2A42219431A912144C9F23F2251442D
:1016A00059441144129A5718614487EA080307EA1B
:1016B000080203EA090325EA01045A404FEAB70386
:1016C00083EA773383EAB7531A444FEAB11312928D
:1016D00083EAF12383EA716A9EF81D3001EA06026B
:1016E0009EF81FC082EA040B9EF81C409EF81E2044
:1016F0001B0443EA046343EA022242EA0C021B92FF
:10170000104445F6D5625844CAF61C325044104481
:10171000129A02EB000A8AEA07030AEA070203EABE
:1017200008035A404FEABA0383EA7A3383EABA538A
:101730001A441292139A104426EA00044FEAB01396
:1017400083EAF02383EA706213929EF8213000EA64
:10175000010282EA040B9EF820409EF822201B041E
:101760009EF823C043EA046343EA0222139B42EA41
:101770000C021C922A445A441A444AF69823CDF685
:1017800007031A44129B9D1885EA0A0405EA0A0316
:101790003C4063404FEAB50484EA753484EAB554AA
:1017A0002344139302EB090321EA03044FEAB31223
:1017B00082EAF32282EA7362129203EA00029EF83E
:1017C00024B082EA04099EF825209EF826409EF85F
:1017D00027C0120442EA0B6242EA042242EA0C02E7
:1017E0001D923244129E4A44324445F60136C1F2FB
:1017F00083263244139E06EB020989EA050409EAAE
:10180000050604EA0A0466404FEAB90484EA79341A
:1018100084EAB9542644139602EB080620EA06042B
:101820004FEAB61282EAF62282EA7662129206EA5B
:1018300003029EF828B082EA04089EF829209EF848
:101840002A409EF82BC0120442EA0B6242EA0422AC
:1018500042EA0C021E921144129A4144114448F289
:10186000BE52C2F231421144139A02EB01083944CC
:1018700088EA090408EA09022C404FEAB1176240DD
:101880004FEAB80484EA783487EAF12784EAB85446
:101890002244139287EA7162129223EA010401EA58
:1018A000060282EA040B9EF82D709EF82C409EF8EA
:1018B0002E203F049EF82FC047EA046444EA022227
:1018C00042EA0C021F921044129A5844104447F600
:1018D000C352C5F20C521044139A1418504484EAAF
:1018E000080704EA080207EA09077A404FEAB40742
:1018F00087EA743787EAB4573A444FEAB01787EA61
:10190000F027139287EA7062129226EA000200EA38
:10191000010787EA020A9EF831209EF830B09EF84F
:10192000327012049EF833C042EA0B6242EA072288
:1019300042EA0C0220921A44129B52441A4445F681
:101940007453C7F2BE231A44139B02EB050C03EB3E
:10195000020A4FEABC128AEA04070AEA040307EA09
:10196000080782EAFC227B404FEABA0787EA7A3707
:1019700082EA7C6287EABA5712923B4413939EF83C
:10198000352021EA0C070CEA00039EF834B083EA04
:1019900007059EF8363012049EF8377042EA0B6253
:1019A00042EA0322129B3A43219232442A441A44C7
:1019B0004BF2FE13C8F2DE031344139AD5184B44BE
:1019C00005EA0A02CDE912A28AEA050A0AEA040631
:1019D000119556404FEAB50282EA7532CDF808E01B
:1019E00082EAB55232444FEAB31686EAF3261092E1
:1019F00086EA736920EA030203EA0C069EF839704E
:101A000086EA020B9EF838609EF83A209EF83B501A
:101A10003F0447EA0666E64646EA02229C462A4317
:101A20002292114440F2A7625944C9F6DC3249447B
:101A30001144109A5318109303EA0A074FEAB302AD
:101A400082EA733282EAB352139B5F40029BD5193C
:101A500001EB08022EEA020702EA0C064FEAB21175
:101A6000904681EAF22186EA070A81EA726993F8D0
:101A70003D2093F83C6093F83E10120493F83F70B9
:101A800042EA066242EA01213943239108444FF2B7
:101A900074115044CCF29B1148444FF0000A0844A2
:101AA00005EB000904440AF1190014AB00F0090029
:101AB00053F820100AF1100000F0080053F820201D
:101AC00011440AF1110202F0090253F822704FEAA0
:101AD000B74686EAD70686EAF71739440AF11E07A1
:101AE00007F00E05139553F825704FEAF74686EA7E
:101AF000972686EA7746314443F8201007910AF189
:101B00001A0101F00A0153F8226053F82110314400
:101B10000AF1120606F00A0753F827604FEAB645A5
:101B200085EAD60585EAF6150D440AF11F0101F094
:101B30000F010F9153F821604FEAF64181EA962197
:101B400081EA7641294443F822100C910AF11B01E5
:101B500001F00B0153F8272053F82110114440F0F5
:101B6000030253F822204FEAB24585EAD20585EAFE
:101B7000F21211440AF1200202F0080B53F82B2054
:101B80004FEAF24585EA922585EA724211440AF14C
:101B900013020A9102F00B0543F827100AF11C0109
:101BA00001F00C0153F8252053F8211011440AF1DB
:101BB000140202F00C0253F822604FEAB64787EA9B
:101BC000D60787EAF61631440AF1210606F009061F
:101BD00053F826604FEAF64787EA962787EA764663
:101BE000314443F8251008910AF11D0101F00D015F
:101BF00053F8225053F82110294440F0050540F0D5
:101C0000070053F825504FEAB54686EAD50686EA1E
